S01C00005354345F537065637472756D5F576F726B696E672E737265633B
S31508008000000002202D6603087D6603087D660308C6
S315080080107D6603087D6603087D6603080000000088
S315080080200000000000000000000000007D66030854
S315080080307D660308000000007D660308895E030864
S315080080407D6603087D6603087D6603087D6603086A
S315080080507D6603087D6603087D6603087D6603085A
S315080080607D6603087D6603087D6603087D6603084A
S315080080707D6603087D6603087D6603087D6603083A
S315080080808D5E0308995E03087D6603087D6603080E
S315080080907D6603087D6603087D660308355F030869
S315080080A07D6603087D6603087D6603087D6603080A
S315080080B0A55E0308B15E03087D6603087D660308AE
S315080080C07D6603087D6603087D6603087D660308EA
S315080080D07D660308BD5E0308C95E03087D6603085E
S315080080E0655F03087D6603087D6603087D660308E9
S315080080F07D6603087D6603087D660308D55E03086A
S315080081007D660308E15E03087D660308ED5E0308E5
S315080081107D6603087D6603087D6603087D66030899
S315080081207D6603087D660308F95E0308055F030894
S315080081307D66030800000000000000007D66030855
S315080081407D6603087D6603087D660308115F0308DC
S315080081507D6603081D5F0308295F03087D6603081B
S315080081607D6603087D6603087D6603087D66030849
S315080081707D6603087D6603087D6603080000000027
S31508008180000000007D6603080000000000000000F3
S315080081907D66030800000000000000007D660308F5
S315080081A00000000000000000000000007D660308D3
S315080081B07D6603087D6603087D6603087D660308F9
S30D080081C07D6603084433221111
S315080081D010B5054C237833B9044B13B10448AFF3F3
S315080081E000800123237010BD6011002000000000EC
S315080081F0984E040808B5034B1BB103490348AFF36F
S31508008200008008BD0000000064110020984E040894
S3150800821010F8012B11F8013B012A28BF9A42F7D022
S31508008220D01A7047034613F8012B002AFBD1181AF7
S315080082300138704700000000000000000000000040
S3150800824001F0FF01102A2BDB10F0070F08D010F8F9
S31508008250013B013A8B422DD010F0070F42B3F6D1FD
S31508008260F0B441EA012141EA014122F007047FF016
S3150800827000070023F0E80256083C85EA010586EA6D
S31508008280010685FA47F5A3FA87F586FA47F6A5FAA9
S3150800829087F68EB9EED1F0BC01F0FF0102F00702B5
S315080082A032B110F8013B013A83EA010313B1F8D160
S315080082B00020704701387047002D06BF3546033841
S315080082C0073815F0010F07D1013015F4807F02BF7A
S315080082D0013015F4C03F0130F0BC0138704700BFCB
S315080082E081F0004102E000BF83F0004330B54FEA59
S315080082F041044FEA430594EA050F08BF90EA020FC6
S315080083001FBF54EA000C55EA020C7FEA645C7FEA58
S31508008310655C00F0E2804FEA5454D4EB5555B8BF7B
S315080083206D420CDD2C4480EA020281EA030382EAEC
S31508008330000083EA010180EA020281EA0303362D7E
S3150800834088BF30BD11F0004F4FEA01314FF4801C51
S315080083504CEA113102D0404261EB410113F0004F63
S315080083604FEA03334CEA133302D0524263EB43031A
S3150800837094EA050F00F0A780A4F10104D5F1200EB8
S315080083800DDB02FA0EFC22FA05F2801841F1000113
S3150800839003FA0EF2801843FA05F359410EE0A5F1E7
S315080083A020050EF1200E012A03FA0EFC28BF4CF018
S315080083B0020C43FA05F3C01851EBE37101F00045CE
S315080083C007D54FF0000EDCF1000C7EEB00006EEBDB
S315080083D00101B1F5801F1BD3B1F5001F0CD3490865
S315080083E05FEA30004FEA3C0C04F101044FEA4452BC
S315080083F012F5800F80F09A80BCF1004F08BF5FEA43
S31508008400500C50F1000041EB045141EA050130BD22
S315080084105FEA4C0C404141EB0101013C28BFB1F534
S31508008420801FE9D291F0000F04BF01460020B1FA7F
S3150800843081F308BF2033A3F10B03B3F120020CDA52
S315080084400C3208DD02F1140CC2F10C0201FA0CF030
S3150800845021FA02F10CE002F11402D8BFC2F1200C95
S3150800846001FA02F120FA0CFCDCBF41EA0C0190404B
S31508008470E41AA2BF01EB0451294330BD6FEA040494
S315080084801F3C1CDA0C340EDC04F11404C4F120027F
S3150800849020FA04F001FA02F340EA030021FA04F391
S315080084A045EA030130BDC4F10C04C4F1200220FAE8
S315080084B002F001FA04F340EA0300294630BD21FA26
S315080084C004F0294630BD94F0000F83F4801306BFEC
S315080084D081F480110134013D4EE77FEA645C18BFE0
S315080084E07FEA655C29D094EA050F08BF90EA020F77
S315080084F005D054EA000C04BF1946104630BD91EA6F
S31508008500030F1EBF0021002030BD5FEA545C05D171
S315080085104000494128BF41F0004130BD14F58004B0
S315080085203CBF01F5801130BD01F0004545F0FE4124
S3150800853041F470014FF0000030BD7FEA645C1ABF59
S31508008540194610467FEA655C1CBF0B46024650EA90
S31508008550013406BF52EA033591EA030F41F40021BC
S3150800856030BD00BF90F0000F04BF0021704730B542
S315080085704FF4806404F132044FF000054FF0000117
S3150800858050E700BF90F0000F04BF0021704730B5D8
S315080085904FF4806404F1320410F0004548BF4042AD
S315080085A04FF000013EE700BF42004FEAE2014FEA02
S315080085B031014FEA02701FBF12F07F4393F07F4FDD
S315080085C081F06051704732F07F4208BF704793F0E0
S315080085D07F4F04BF41F40021704730B54FF46074F3
S315080085E001F0004521F000411CE700BF50EA0102F6
S315080085F008BF704730B54FF000050AE050EA01029F
S3150800860008BF704730B511F0004502D5404261EB0E
S3150800861041014FF4806404F132045FEA915C3FF44F
S31508008620D8AE4FF003025FEADC0C18BF03325FEAEC
S31508008630DC0C18BF033202EBDC02C2F1200300FA9D
S3150800864003FC20FA02F001FA03FE40EA0E0021FAC2
S3150800865002F11444BDE600BF70B54FF0FF0C4CF4B0
S31508008660E06C1CEA11541DBF1CEA135594EA0C0F62
S3150800867095EA0C0F00F0DEF82C4481EA030621EA9D
S315080086804C5123EA4C5350EA013518BF52EA0335D8
S3150800869041F4801143F4801338D0A0FB02CE4FF08A
S315080086A00005E1FB02E506F00042E0FB03E54FF0BA
S315080086B00006E1FB03569CF0000F18BF4EF0010EB2
S315080086C0A4F1FF04B6F5007F64F5407404D25FEAAE
S315080086D04E0E6D4146EB060642EAC62141EA555161
S315080086E04FEAC52040EA5E504FEACE2EB4F1FD0CA3
S315080086F088BFBCF5E06F1ED8BEF1004F08BF5FEA21
S31508008700500E50F1000041EB045170BD06F00046D2
S3150800871046EA010140EA020081EA0301B4EB5C047F
S31508008720C2BFD4EB0C0541EA045170BD41F4801177
S315080087304FF0000E013C00F3AB8014F1360FDEBF9C
S31508008740002001F0004170BDC4F10004203C35DA78
S315080087500C341BDC04F11404C4F1200500FA05F3FB
S3150800876020FA04F001FA05F240EA020001F000429C
S3150800877021F0004110EBD37021FA04F642EB060112
S315080087805EEA430E08BF20EAD37070BDC4F10C043C
S31508008790C4F1200500FA04F320FA05F001FA04F200
S315080087A040EA020001F0004110EBD37041F10001EC
S315080087B05EEA430E08BF20EAD37070BDC4F12005F7
S315080087C000FA05F24EEA020E20FA04F301FA05F25F
S315080087D043EA020321FA04F001F0004121FA04F207
S315080087E020EA020000EBD3705EEA430E08BF20EAD7
S315080087F0D37070BD94F0000F0FD101F00046400011
S3150800880041EB010111F4801F08BF013CF7D041EA92
S31508008810060195F0000F18BF704703F00046520096
S3150800882043EB030313F4801F08BF013DF7D043EA67
S315080088300603704794EA0C0F0CEA135518BF95EA1D
S315080088400C0F0CD050EA410618BF52EA4306D1D1A4
S3150800885081EA030101F000414FF0000070BD50EAC3
S31508008860410606BF1046194652EA430619D094EA4D
S315080088700C0F02D150EA013613D195EA0C0F05D137
S3150800888052EA03361CBF104619460AD181EA03018B
S3150800889001F0004141F0FE4141F470014FF0000043
S315080088A070BD41F0FE4141F4780170BD70B54FF0DE
S315080088B0FF0C4CF4E06C1CEA11541DBF1CEA13555E
S315080088C094EA0C0F95EA0C0F00F0A7F8A4EB050440
S315080088D081EA030E52EA03354FEA013100F0888037
S315080088E04FEA03334FF0805545EA131343EA126300
S315080088F04FEA022245EA111545EA10654FEA0026B5
S315080089000EF000419D4208BF964244F1FD0404F56D
S31508008910407402D25B084FEA3202B61A65EB0305C9
S315080089205B084FEA32024FF480104FF4002CB6EB86
S31508008930020E75EB030E22BFB61A754640EA0C0006
S315080089405B084FEA3202B6EB020E75EB030E22BF46
S31508008950B61A754640EA5C005B084FEA3202B6EB87
S31508008960020E75EB030E22BFB61A754640EA9C0046
S315080089705B084FEA3202B6EB020E75EB030E22BF16
S31508008980B61A754640EADC0055EA060E18D04FEAD4
S31508008990051545EA16754FEA06164FEAC30343EA74
S315080089A052734FEAC2025FEA1C1CC0D111F4801F41
S315080089B00BD141EA00014FF000004FF0004CB6E73A
S315080089C011F4801F04BF01430020B4F1FD0C88BFD9
S315080089D0BCF5E06F3FF6AFAEB5EB030C04BFB6EBE4
S315080089E0020C5FEA500C50F1000041EB045170BDD7
S315080089F00EF0004E4EEA113114EB5C04C2BFD4EB04
S31508008A000C0541EA045170BD41F480114FF0000E87
S31508008A10013C90E645EA060E8DE60CEA135594EA03
S31508008A200C0F08BF95EA0C0F3FF43BAF94EA0C0F06
S31508008A300AD150EA01347FF434AF95EA0C0F7FF47B
S31508008A4025AF104619462CE795EA0C0F06D152EACF
S31508008A5003353FF4FDAE1046194622E750EA4106B3
S31508008A6018BF52EA43067FF4C5AE50EA41047FF4C4
S31508008A700DAF52EA43057FF4EBAE12E74FF0FF3C29
S31508008A8006E000BF4FF0010C02E000BF4FF0010CFA
S31508008A904DF804CD4FEA410C7FEA6C5C4FEA430C73
S31508008AA018BF7FEA6C5C1BD001B050EA410C0CBFC2
S31508008AB052EA430C91EA030F02BF90EA020F002024
S31508008AC0704710F1000F91EA030F58BF994208BF8B
S31508008AD090422CBFD8176FEAE37040F00100704748
S31508008AE04FEA410C7FEA6C5C02D150EA013C07D19F
S31508008AF04FEA430C7FEA6C5CD6D152EA033CD3D0EA
S31508008B005DF8040B704700BF8446104662468C46E3
S31508008B101946634600E000BF01B5FFF7B7FF002816
S31508008B2048BF10F1000F01BD4DF808EDFFF7F4FF3F
S31508008B300CBF012000205DF808FB00BF4DF808EDCA
S31508008B40FFF7EAFF34BF012000205DF808FB00BFED
S31508008B504DF808EDFFF7E0FF94BF012000205DF80F
S31508008B6008FB00BF4DF808EDFFF7CEFF94BF0120C4
S31508008B7000205DF808FB00BF4DF808EDFFF7C4FFBD
S31508008B8034BF012000205DF808FB00BF4FEA410C06
S31508008B907FEA6C5C02D150EA013C0AD14FEA430CE9
S31508008BA07FEA6C5C02D152EA033C02D14FF0000026
S31508008BB070474FF0010070474FEA410212F5001264
S31508008BC015D211D56FF47873B3EB625212D94FEA06
S31508008BD0C12343F0004343EA505311F0004F23FAF0
S31508008BE002F018BF404270474FF00000704750EA45
S31508008BF0013005D111F0004008BF6FF00040704702
S31508008C004FF00000704700BF4A0011D212F500125B
S31508008C1011D20DD56FF47873B3EB62520ED44FEAC6
S31508008C20C12343F0004343EA505323FA02F0704746
S31508008C304FF00000704750EA013002D14FF0FF3084
S31508008C4070474FF0000070474FEA4102B2F1E04327
S31508008C5024BFB3F5001CDCF1FE5C0DD901F0004C15
S31508008C604FEAC0024CEA5070B2F1004F40EB830065
S31508008C7008BF20F00100704711F0804F21D113F191
S31508008C803872BCBF01F00040704741F480114FEACA
S31508008C905252C2F11802C2F1200C10FA0CF320FA53
S31508008CA002F018BF40F001004FEAC1234FEAD32370
S31508008CB003FA0CFC40EA0C0023FA02F34FEA4303DA
S31508008CC0CCE77FEA625307D150EA01331EBF4FF063
S31508008CD0FE4040F44000704701F0004040F0FE407E
S31508008CE040F40000704700BF53B94AB9002908BFCD
S31508008CF000281CBF4FF0FF314FF0FF3000F0AAB933
S31508008D00ADF1080C6DE904CE00F03CF8DDF804E09E
S31508008D10DDE9022304B0704738B500220023044673
S31508008D200D46FFF70BFF28B920462946BDE838400F
S31508008D3000F00AB8204605F1004100F005F8404267
S31508008D4061EB410138BD00BFD0B50C4B0022064689
S31508008D500F46FFF781FCFFF757FF0446FFF702FCB3
S31508008D60074B0022FFF778FC02460B463046394689
S31508008D70FFF7BAFAFFF748FF2146D0BD0000F03DDD
S31508008D800000F0412DE9F047089D04468E46002B69
S31508008D904DD18A42944669D9B2FA82F252B101FAA1
S31508008DA002F3C2F1200120FA01F10CFA02FC41EAB1
S31508008DB0030E94404FEA1C48210CBEFBF8F61FFA36
S31508008DC08CF708FB16E341EA034306FB07F19942D1
S31508008DD00AD91CEB030306F1FF3080F01F81994284
S31508008DE040F21C81023E63445B1AA4B2B3FBF8F05E
S31508008DF008FB103344EA034400FB07F7A7420AD9E5
S31508008E001CEB040400F1FF3380F00A81A74240F20C
S31508008E1007816444023840EA0640E41B00261DB177
S31508008E20D4400023C5E900433146BDE8F0878B42AC
S31508008E3009D9002D00F0EF800026C5E9000130466B
S31508008E403146BDE8F087B3FA83F6002E4AD18B4245
S31508008E5002D3824200F2F980841A61EB03030120EF
S31508008E609E46002DE0D0C5E9004EDDE702B9FFDEDB
S31508008E70B2FA82F2002A40F09280A1EB0C014FEA86
S31508008E801C471FFA8CFE0126200CB1FBF7F307FBE3
S31508008E90131140EA01410EFB03F0884208D91CEB86
S31508008EA0010103F1FF3802D2884200F2CB80434623
S31508008EB0091AA4B2B1FBF7F007FB101144EA014402
S31508008EC00EFB00FEA64508D91CEB040400F1FF3191
S31508008ED002D2A64500F2BB800846A4EB0E0440EA7F
S31508008EE003409CE7C6F12007B34022FA07FC4CEA88
S31508008EF0030C20FA07F401FA06F31C43F9404FEA7B
S31508008F001C4900FA06F3B1FBF9F8200C1FFA8CFE8F
S31508008F1009FB181140EA014108FB0EF0884202FAE3
S31508008F2006F20BD91CEB010108F1FF3A80F08880A4
S31508008F30884240F28580A8F102086144091AA4B261
S31508008F40B1FBF9F009FB101144EA014100FB0EFEE2
S31508008F508E4508D91CEB010100F1FF346CD28E4511
S31508008F606AD90238614440EA0840A0FB0294A1EBA2
S31508008F700E01A142C846A64656D353D05DB1B3EBFF
S31508008F80080261EB0E0101FA07F722FA06F3F1402F
S31508008F901F43C5E9007100263146BDE8F087C2F1D6
S31508008FA02003D8400CFA02FC21FA03F3914001434E
S31508008FB04FEA1C471FFA8CFEB3FBF7F007FB103687
S31508008FC00B0C43EA064300FB0EF69E4204FA02F433
S31508008FD008D91CEB030300F1FF382FD29E422DD986
S31508008FE0023863449B1B89B2B3FBF7F607FB1633BB
S31508008FF041EA034106FB0EF38B4208D91CEB01013B
S3150800900006F1FF3816D28B4214D9023E6144C91ABA
S3150800901046EA004638E72E46284605E70646E3E6CA
S315080090201846F8E64B45A9D2B9EB020864EB0C0ED4
S315080090300138A3E74646EAE7204694E74046D1E7E3
S31508009040D0467BE7023B614432E7304609E7644491
S31508009050023842E7704700BF13B50446084659B1BF
S315080090600191FFF7DFF8236801995B6802462046FD
S3150800907002B0BDE81040184702B010BD08B5024955
S31508009080FFF7EAFF08BD00BF18C2040838B5054651
S31508009090FFF7E2FF04462846FFF7F0FF204438BDF5
S315080090A0FFF7F4BF07B503688DF807105B68012260
S315080090B00DF10701984703B05DF804FB4FF0FF3048
S315080090C07047704710B54FF0FF331446006992B2E7
S315080090D031F0EFFD204610BD07B54FF0FF330122F2
S315080090E00DF10701006931F039FE9DF8070003B05C
S315080090F05DF804FB10B50446006837F057FB2046B8
S3150800910010BD10B50446006808B137F04FFB0023C0
S31508009110C4E90133236010BD38B504460D4600681E
S31508009120013138F0DDF810B1C4E90005012038BD79
S31508009130036810B5044623B143688B4201D3012066
S3150800914010BD2046FFF7E8FF0028F9D0A368002BDA
S31508009150F5D122681370F2E770B50E46114604463B
S315080091601546FFF7E5FF20B92046FFF7CAFF204658
S3150800917070BD2068A560314638F07EF9F7E7002310
S3150800918013B5C0E900330446836041B1084601912E
S31508009190FFF748F8019902462046FFF7DDFF20460B
S315080091A002B010BD38B5054600680C4668B16A6855
S315080091B08B689A4207D3096838F05EF9A368AB60F2
S315080091C00023A36038BD37F0F1FA23682B60636883
S315080091D06B60A368AB600023C4E90033F1E710B500
S315080091E00023C0E9003304468360FFF7DBFF20460F
S315080091F010BD884210B5044605D00B682BB18A68A5
S315080092001946FFF7A9FF204610BDFFF77AFFFAE7D0
S3150800921010B500230446C0E900338360FFF7E9FF71
S31508009220204610BD884210B5044601D0FFF7BAFFA4
S31508009230204610BD13B5044659B108460191FEF7FC
S31508009240F1FF019902462046FFF786FF204602B045
S3150800925010BDFFF756FFF9E770B505460E4609B982
S31508009260002070BD6AB1846814442146FFF760FF88
S315080092700028F5D02868AB683146184438F0FCF861
S31508009280AC600120EDE707B500238DF80410012234
S3150800929001A98DF80530FFF7DFFF03B05DF804FB81
S315080092A0826808B53AB921B10878B0FA80F0400961
S315080092B000E0012008BD006809B90078F5E7FEF767
S315080092C0A7FFF2E783688B4201D9006818B90348FB
S315080092D00023037070470844704700BF7C110020C4
S315080092E08368934210B506D90468A01838F0B7F811
S315080092F008B1001B10BD4FF0FF30FBE72DE9F04128
S315080093009A420E461F460F4988BF134614468046A2
S3150800931084BF3C461F46FFF732FFB568A5420DD904
S31508009320BD42336828BF3D4600225F5D5A55316805
S3150800933040462144FFF77EFF33685F554046BDE847
S31508009340F08100BF709B0408006808B137F0F7B9D0
S315080093507047FF2808D9B0F5007F07D3B0F5407FDE
S3150800936034BFA520A7207047A1207047A3207047C7
S3150800937030B540F2FE3385189D4285B004460EDCB2
S31508009380FFF7E7FF0E23CDE9012300910123C1B2C0
S31508009390E2B204482EF0CEFB012005B030BD002015
S315080093A0FBE700BFBC1B0020FFF7E2BF30B540F269
S315080093B0FE330D468118994287B0044613DCFFF741
S315080093C0C8FF0E23CDE9012305AB0093C1B20123E3
S315080093D00648E2B22EF0AEFBBDF814305BBA2B801D
S315080093E0012007B030BD0020FBE700BFBC1B0020F2
S315080093F0FF2808D9B0F5007F07D3B0F5407F34BF02
S31508009400A420A6207047A0207047A220704700001D
S3150800941030B540F2FE3385189D4285B0044611DC0E
S31508009420FFF7E6FF0E23CDE9012300910123C1B220
S31508009430E2B205482EF0EEFA04202DF071F901206B
S3150800944005B030BD0020FBE7BC1B002030B540F25C
S31508009450FE3385189D4285B0044611DCFFF7C8FF28
S315080094600E23CDE9012300910123C1B2E2B20548DA
S315080094702EF0D0FA04202DF053F9012005B030BDA6
S315080094800020FBE7BC1B002010B50B8886B0190A24
S315080094908DF814108DF81530811840F2FE33994274
S315080094A0044612DCFFF7A4FF0E23CDE9012305AB22
S315080094B0C1B20093E2B2012305482EF0ABFA0420AC
S315080094C02DF02EF9012006B010BD0020FBE700BFE5
S315080094D0BC1B002008B501464C2200F5FC7037F08D
S315080094E06DF908BD10B5C46B091BC0F85012016CA4
S315080094F0521AC0F85422426C9B1AC0F8583210BD52
S31508009500838D10B50446F3B1B0F824229A4207D0E9
S31508009510A0F8F431D0F8F811D0E97F23FFF7E2FF7D
S3150800952094F8483094F877209A1A5342534184F8AD
S315080095304A3094F8492094F897309A420CBF012390
S31508009540002384F84B3010BD10B5C47B8361013409
S3150800955014F0FF04029B838308BF0124C0E90412A8
S31508009560C47310BD044B828D198891421ABF01201D
S315080095701A800020704700BF7E1100204B780878BB
S315080095801B0443EA0063C8784340887843EA00200E
S31508009590704710B50446FFF79DFF04F5197120467C
S315080095A0FFF7ECFFD4F85032E0631844206004F566
S315080095B01A712046FFF7E2FFD4F8543220641844A3
S315080095C0606004F51B712046FFF7D8FFD4F85832BF
S315080095D060641844A06004F51C712046FFF7CEFFAE
S315080095E004F51D71E0602046FFF7C8FF94F878225D
S315080095F094F87932206143EA0223238394F87A2285
S3150800960094F87B3243EA0223638394F87C2294F825
S315080096107D3243EA0223A383B4F87E32A384B4F8E6
S315080096208032E384B4F88232E385D4F88432236343
S31508009630D4F888326363D4F88C32A36304F52371B3
S315080096402046FFF79BFF94F8902294F891326061C8
S3150800965043EA0223A385B4F89232A4F8483094F872
S315080096609432803B236294F89532803B07EE903A19
S31508009670F8EEE77AF2EE046A87EEA67A204684EDDB
S315080096800A7AFFF73DFF012384F85C3210BD00001B
S31508009690012908D1144B90F82E205878904220D0F2
S315080096A05A7001207047022907D10F4B90F82F20D6
S315080096B09978914215D09A70F3E7032907D10A4B96
S315080096C090F83020D97891420BD0DA70E9E704296E
S315080096D007D1054B90F831201979914201D01A71BA
S315080096E0DFE70020704700BF8011002010B5012178
S315080096F00446FFF7CDFF02212046FFF7C9FF0321E5
S315080097002046FFF7C5FF20460421BDE81040FFF7B5
S31508009710BFBF000070B590F85C425CB1074D2B786E
S315080097200022012680F85C2280F8186123B9FFF729
S31508009730DDFF2E70204670BD1C46FBE77D1100201C
S3150800974010B50B4600205C1AA24204DD13F8014B43
S315080097502044C0B2F7E710BDF0B504460D468FB0F9
S3150800976000F25E213C2200F25D2037F035F894F8CD
S315080097705D3284F89952492B3CD194F85E32572BC6
S3150800978038D194F85F32412B34D194F86032502B9B
S3150800979030D194F86132492B2CD194F86202022810
S315080097A026D194F897323B2B20D194F89832212B66
S315080097B01CD13B2D1AD101AA04F2622304F2922786
S315080097C0164618685968154603C50833BB422A4623
S315080097D0F7D118682860342231462046FFF7B0FFD3
S315080097E094F89632834214BF032000200FB0F0BDD0
S315080097F00520FBE70120F9E710B50446FFF7ACFFA3
S3150800980020B92046BDE81040FFF7C3BE01280FD097
S31508009810052805D107490848BDE81040FFF740BCB0
S31508009820022801D10549F6E7032801D10449F2E7E0
S3150800983010BD00BFC8510408241E0020D6510408D4
S31508009840E151040810B5D0F84532C0F8193190F83E
S31508009850493280F81D3190F8443280F81E31B0F84C
S31508009860F431A0F81F310368C0F821314368C0F805
S3150800987025318368C0F82931C36CC0F82D31036DD2
S31508009880C0F8313190F8543080F8353190F86430AA
S3150800989080F83631B6B0044600F1550300F23712A7
S315080098A000F1610153F8040B42F8040B8B42F9D11D
S315080098B0198811809B78937004F1740104F1680388
S315080098C004F5A37253F8040B42F8040B8B42F9D142
S315080098D0198811809B789370A36FC4F85531E36F8C
S315080098E0C4F85931D4F88030C4F85D31B4F88430FE
S315080098F0A4F8613194F8773084F8633104F5B272CC
S3150800990004F1880304F1940153F8040B42F8040B9C
S315080099108B42F9D1198811809B789370D4F89830C6
S31508009920C4F87331D4F89C30C4F87731D4F8A03031
S31508009930C4F87B31B4F8A430A4F87F3194F8973092
S3150800994084F8813104F5C17204F1A80304F1B40165
S3150800995053F8040B42F8040B8B42F9D1198811808D
S315080099609B78937004F1C30104F1B70304F29112D2
S3150800997053F8040B42F8040B8B42F9D1198811806D
S315080099809B78937004F1D20104F1C60304F5D072F2
S3150800999053F8040B42F8040B8B42F9D1198811804D
S315080099A09B78937004F1E10104F1D50304F2AF1238
S315080099B053F8040B42F8040B8B42F9D1198811802D
S315080099C09B78937004F1F00104F1E40304F5DF7267
S315080099D053F8040B42F8040B8B42F9D1198811800D
S315080099E09B78937004F1FF0104F1F30304F2CD129E
S315080099F053F8040B42F8040B8B42F9D119881180ED
S31508009A009B789370D4F80431C4F8DC31D4F8083163
S31508009A10C4F8E031D4F80C31C4F8E431D4F8103184
S31508009A20C4F8E831D4F81431C4F8EC3104F58F7170
S31508009A30D22201A836F0C2FED22201A92046FFF79B
S31508009A407FFEB4F84A32A4F8F13194F84C3284F81F
S31508009A50F00184F8F33136B010BD002070470020BD
S31508009A60704770477047002070477047002070475E
S31508009A702DE9F0470446884600F0D6FBA36C94F817
S31508009A802010344F344EDFF8E89004F1080503BB84
S31508009A90204600F00DFCB8F1000F05D02F4B3A78A0
S31508009AA031882F4805F0C4FC29462D48B9F80040EE
S31508009AB005F01AFD31883A78201A00EBD07001EBD0
S31508009AC0600189B231802B46BDE8F047244805F08D
S31508009AD0AFBC0139C9B2204600F0EAFBB8F1000F65
S31508009AE005D01E4B3A7831881D4805F0A1FC2A4658
S31508009AF01C491D4837F050FC1B491948B9F8005055
S31508009B0005F0F2FC3188184B3A780D442D1AA9B2A3
S31508009B101348318005F08CFCA36B1B780C2505FBDC
S31508009B2003431B6C9BB194F8201001312046C9B23F
S31508009B3000F0BEFBA36B0D49187805FB00440A48E4
S31508009B40226C37F029FC084B3A783188BCE7BDE827
S31508009B50F08700BF991100209A110020EE510408E1
S31508009B60C0110020F05104088511002040A90408FE
S31508009B709C1100202C3037F07FBC000070B50546DC
S31508009B80084B45F8703B044600F14006B54204D040
S31508009B900C3D2846FFF7AEFAF8E7204600F014FB1E
S31508009BA0204670BD0052040810B50446FFF7E6FFCC
S31508009BB02046702135F0B1FC204610BD2DE9F3474B
S31508009BC01E460223044600930B9B0A9FDFF858A003
S31508009BD000F0D6FA2346134A43F82C2B04F1400525
S31508009BE00022E26204F170095A601A81A8462846E2
S31508009BF051460C35FFF7C3FA4D45F8D156B1002545
S31508009C00711908EB05000C35FFF7F3FA302DF7D17B
S31508009C100C9BA36307B1E76301232046E37102B0F7
S31508009C20BDE8F08700520408709B040810B5044686
S31508009C3000F0DCFAE06B10BD704700002DE9F04F2C
S31508009C40044685B00E4600F0EFFA94F82010DFF8C7
S31508009C507081534D204600F02BFB36B1514B98F8D6
S31508009C6000202988504805F0E3FB04F108024F4913
S31508009C704F4837F091FB4F4B4D494B481E8805F02E
S31508009C8033FC29884A4B98F800200E44361AB1B29C
S31508009C904548298005F0CCFB94F820102679023136
S31508009CA0C9B22046002E53D100F002FB42493E4875
S31508009CB03D4FDFF8109105F017FC2B8818442880D3
S31508009CC0636A9B68B34268D90321384605F052FD9A
S31508009CD094F83830B3422BD194F9493098F80020DB
S31508009CE0B5F800B0039204EB83033846D3F84CA0CA
S31508009CF0514605F0F9FB99F80010039A00910346BE
S31508009D005946384605F020FF0021384605F032FD51
S31508009D10298898F800205346384605F089FB5146AD
S31508009D20384605F0E1FB2B88184428800136C7E73A
S31508009D30D4F8E43029889B5798F8002004EB83036D
S31508009D403846DB6C039305F073FB039B1946E7E77C
S31508009D5000F0AEFAE26B1949154837F01DFB98F882
S31508009D600020134B2988104805F062FBE16B0E486A
S31508009D7005F0BAFB2B8811491844636A28801A68CB
S31508009D800B4837F009FB0A4B98F800202988064843
S31508009D9005B0BDE8F04F05F04BBB05B0BDE8F08F48
S31508009DA09A110020EE510408C0110020F051040851
S31508009DB0851100209C11002040D4040840A90408FD
S31508009DC0991100209E110020F8B50B78132B044634
S31508009DD00BD80A2B0BD90B3B082B08D8DFE803F066
S31508009DE00856076B070756076B002B2B46D0F8BD9E
S31508009DF090F83830D0F8E42090F94910D154416AE7
S31508009E0090F838308A68013A934215D2013390F8AF
S31508009E104820DBB280F83830002AE8D00968C95CE7
S31508009E209142E4D1D0F8E4202521D15490F8383075
S31508009E30013384F83830DAE7002500F12C0694F867
S31508009E402830AB4212DDD4F8E4305B57252B18BF17
S31508009E5004EB8303294630460CBFD4F8E070DF6C68
S31508009E60FFF730FA3B7803700135E8E7606A314658
S31508009E70FFF7BFF940F20113A380B8E790F838302E
S31508009E800BB1013BD5E743790371B0E790F8493048
S31508009E9090F8F02001335BB280F84930F2B9232BF1
S31508009EA0A5DD002384F84930A1E7022A9FD1232B98
S31508009EB09DDD1A23F6E790F8493090F8F020013B2B
S31508009EC05BB280F849301AB9002B90DA2323E9E708
S31508009ED0012A07D1002B8ADA1923E3E7012AE4D1FC
S31508009EE0192BDDE7022A82D1192BEFDD7FE7000067
S31508009EF00C4B10B504460360D0F8E40020B1D4F842
S31508009F00EC10091A35F009FB04F13C00FFF7F2F8EA
S31508009F1004F12C00FFF7EEF8204600F055F920462C
S31508009F2010BD00BF5C52040810B50446FFF7E0FFF9
S31508009F302046F42135F0F1FA204610BD2DE9F84FF8
S31508009F40D0E900896FF00043A9EB08049C42074654
S31508009F508A46934602D11E4835F0F5FA012C224668
S31508009F6038BF0122A418A1EB08052CD2002C2ADB45
S31508009F702BD0204635F0D3FA06469BF800307355A9
S31508009F80002D04DD2A464146304636F025FCA9EB6D
S31508009F900A090135B9F1000F354404DD4A46514630
S31508009FA0284636F00BFC4D44B8F1000F05D0B968C9
S31508009FB04046A1EB080135F0B0FA3444C7E900651C
S31508009FC0BC60BDE8F88F1C46D3E72646D5E700BF38
S31508009FD03852040810B50A46D0E90114A14206D041
S31508009FE092F900200A7042680132426010BDFFF7FC
S31508009FF0A5FFFBE72DE9FF4704461F46022300930A
S3150800A00026460C9B9DF8348000F0BAF8234B46F898
S3150800A0102C3B04F13C0A22493046FFF7B0F82049A8
S3150800A0205046FFF7ACF800251E49982204F14C006B
S3150800A03036F0C4FB67625046C4E939550F99C4F82F
S3150800A040EC5084F83850FFF7D4F8042304F1E409F7
S3150800A050E37124274FF0250A616A8B68AB420ED953
S3150800A0600B685B5D0DF10F01434548460CBF8DF843
S3150800A0700FA08DF80F700135FFF7ACFFECE784F8F9
S3150800A08028303046FFF7B5F89DF8383084F8F030B8
S3150800A090204684F8488004B0BDE8F0875C5204087E
S3150800A0A0709B0408B04E04082DE9FF4704461D4678
S3150800A0B09DF83030009326460D9B9DF8387000F0C9
S3150800A0C05FF8224B46F82C3B21493046FFF757F8F4
S3150800A0D01F4904F13C00FFF752F898221D4904F184
S3150800A0E04C0036F06BFB0022C4E939220423656272
S3150800A0F004F1E40AC4F8EC2084F83820E371154624
S3150800A1004FF024084FF02509616A8B68AB420ED9D7
S3150800A1100B685B5D0DF10F01BB4250460CBF8DF815
S3150800A1200F908DF80F800135FFF754FFECE784F8A0
S3150800A13028303046FFF75DF89DF83C3084F8F0305B
S3150800A140204684F8487004B0BDE8F0875C520408DD
S3150800A150709B0408B04E040810B5044600F046F893
S3150800A16094F8F030012B06D8002384F849300020F3
S3150800A17084F8380010BD022BF9D11A23F5E7000040
S3150800A18038B51D460E4B03600E4B4360082380F816
S3150800A1902130002380F822304B1E04460E2B94BF34
S3150800A1A00846002084F82000114604F1080037F01C
S3150800A1B063F99DF81030E5612371204638BD00BF6C
S3150800A1C0945204080202000510B5044B0446012106
S3150800A1D040F8083B35F0A1F9204610BD9452040812
S3150800A1E0037901718B4218BF437170478379012B3C
S3150800A1F010B508D00379032B05D0FFF7F1FFC36923
S3150800A2000BB108469847002010BD43790371704783
S3150800A2100079704780797047002383717047817190
S3150800A2207047C0797047000038B590F82130082B80
S3150800A230044623D11549164805F068F9144D2846F1
S3150800A24005F03BF9284605F049F995F82A2095F8CE
S3150800A25029309B1A0F4A137094F8223093B92B8829
S3150800A2600D4A1380A379012B02D02379032B0BD136
S3150800A2700121BDE83840064805F07CBA062BDDD139
S3150800A2800649D8E79BB2EBE70321F2E70462040824
S3150800A290C01100209E110020A0110020BA5A0408FF
S3150800A2A080F82210704708307047083037F0E4B855
S3150800A2B001390B2928D8DFE801F006101C282E34AE
S3150800A2C03A3F44494D51274B1A78274B1A70274B6A
S3150800A2D0274A1B885B08138007E0224B1A78224B13
S3150800A2E01A70224B1A88224B1A80224B00221A8097
S3150800A2F070471C4B1A781C4B1A701C4B1C4A1B883F
S3150800A3005B0813801B4A13807047164B1B785B004B
S3150800A310154A1370DBE7134B1B785B00124A137060
S3150800A320DFE7104B1B785B000F4A1370E5E70D4B10
S3150800A3301B7803EB4303EBE70A4B1B7803EB43035A
S3150800A340ECE7084B1B7803EB4303EDE7054B1B785B
S3150800A3509B00DDE7034B1B789B00DFE7014B1B786F
S3150800A3609B00E1E79E11002099110020A011002012
S3150800A3709C1100209A11002038B50B780E2B044644
S3150800A38011D004D80B2B07D00C2B2CD038BD2B2B77
S3150800A390FCD143790371F9E70368DB68984740F213
S3150800A3A00113A380F2E790F8313090F8305001336A
S3150800A3B080F8313000231A469D4294F9310008DCB2
S3150800A3C0002AF7D194F828308342DFDC84F831205C
S3150800A3D0DCE7E16AC95C814202BF013184F83110C9
S3150800A3E001220133E8E790F83130013B80F831303B
S3150800A3F090F8300000231946984294F931200ADC77
S3150800A4000029F7D1002ABEBF94F8283003F1FF339C
S3150800A41084F83130BAE7E56AED5CAA4202BF02F178
S3150800A420FF3284F8312001210133E5E7436B13B18C
S3150800A43090F831201A7000207047416280F8282071
S3150800A440704790F93120436A53F82200704790F814
S3150800A450380070472DE9F14F04460F46FFF7E4FE32
S3150800A46094F83830012B6AD194F820102046FFF76B
S3150800A4701FFF3FB1674A6849684B127809886848E0
S3150800A48004F0D6FF257904F1080815B16549424656
S3150800A49038E0DFF8A8A1DFF8A891614F2E4601350C
S3150800A4A005EB4501C9B22046FFF702FF94F93130A2
S3150800A4B0002B1A46B8BFDA1C921006EB8206B34286
S3150800A4C00ED149463846BAF800B005F00DF8514A9B
S3150800A4D0ABEB000081B212784B46384604F0A8FF71
S3150800A4E094F82830B34209DD636A4A4A4A4953F860
S3150800A4F0263012780988384604F09AFF042DCDD103
S3150800A50049494246494836F047FF94F82010204604
S3150800A510FFF7CEFE464B454941481C8804F0E4FF48
S3150800A5203D4B3C4A198812780C44241AA1B219806A
S3150800A5303E4B3B4801B0BDE8F04F04F079BFFBB98C
S3150800A54094F82010334E344D2046FFF7B1FE2FB154
S3150800A550324B32782988324804F06AFF94F8201082
S3150800A56023790231C9B22046002B47D1FFF7A0FE56
S3150800A57094F82830D3B92F492C4836F07DFF1EE0D1
S3150800A580022B44D194F82010224E234D2046FFF783
S3150800A5908FFE2FB1214B32782988214804F048FFD5
S3150800A5A094F8201023790231C9B2DCE794F93120F6
S3150800A5B0636A214953F822201C4836F0EDFE1B4BEE
S3150800A5C032782988164804F033FF04F10802164940
S3150800A5D0164836F0E1FE94F820102046FFF768FE8C
S3150800A5E0134B12490E481C8804F07EFF29880F4B2E
S3150800A5F032780C44241AA1B229809AE7FFF758FE4C
S3150800A60094F82830002BB6D0636B1A78D0E701B0DF
S3150800A610BDE8F08F991100209A110020EE51040828
S3150800A620C0110020C6520408F15104088511002003
S3150800A6309C110020CA52040840A90408A011002051
S3150800A640C452040838B5436A04466BB1002594F829
S3150800A6502830AB4208DD636A53F8250010B10121A2
S3150800A66034F05BFF0135F2E738BD000010B50C4B3E
S3150800A67003600446FFF7E6FF606B10B1012134F072
S3150800A6804CFFE06A10B1012134F047FF012104F1C3
S3150800A690080034F042FF2046FFF796FD204610BD1D
S3150800A6A0E052040810B50446FFF7E0FF20463C21B7
S3150800A6B034F033FF204610BD37B51D460223044645
S3150800A6C00093099BFFF75CFD0B4B2360002384F87E
S3150800A6D02830E36223869DF8203084F83830032337
S3150800A6E0E37125B19DF81830656284F82830079B18
S3150800A6F06363204603B030BDE052040837B504460C
S3150800A7000093069B089DFFF73BFD0C4B2360002337
S3150800A71084F82830E36223869DF8283084F8383098
S3150800A7200323E37125B19DF82430656284F8283047
S3150800A730079B6363204603B030BD00BFE0520408A0
S3150800A74010B50446FFF752FD94F83830022B13D1A2
S3150800A75094F8313094F8282001335BB29A4284F891
S3150800A7603130DCBF002384F8313023682046DB68AB
S3150800A770984740F20113A380002010BD704790F857
S3150800A7803600704710B5034B03600446FFF71CFDFF
S3150800A790204610BD2053040810B50446FFF7F2FF03
S3150800A7A020463C2134F0B9FE204610BD2DE9F04183
S3150800A7B004460D46FFF738FD94F82010224F234E25
S3150800A7C00139C9B22046FFF773FD2DB1204B3A78FF
S3150800A7D03188204804F02CFE04F108021E491F485F
S3150800A7E036F0DAFD1E4B1D491A481D8804F07CFE1A
S3150800A7F031881A4B3A780D442D1AA9B2154831807A
S3150800A80004F016FE2379022B13D1626A1549134800
S3150800A81036F0C2FD94F8201001312046C9B2FFF780
S3150800A82047FD3A7831880D4B0A48BDE8F04104F0F7
S3150800A830FFBD012BEED1A36A0B49084804F12C028F
S3150800A84036F0AAFDE6E700BF991100209A1100200C
S3150800A850EE510408C0110020F051040885110020AB
S3150800A8609C11002040A90408105304082C3036F027
S3150800A87003BE000037B51D46022304460093079B16
S3150800A880FFF77EFC22460A4B42F82C3B0023E36284
S3150800A8905360138184F836301DB16B68A3622B6848
S3150800A8A06362069BA36320460223E37103B030BDAF
S3150800A8B0205304084162704710B50446FFF796FC1A
S3150800A8C0A06B10BD2DE9F04105461E464FF4006306
S3150800A8D025F8043B04460F4628460C499046FEF7E1
S3150800A8E04EFC0A4904F11000FEF749FC0023638474
S3150800A8F084F8243041462846FEF79CFC9DF818301B
S3150800A9002777A67763772046BDE8F081709B040811
S3150800A91010B504461030FEF7EDFB201DFEF7EAFBE6
S3150800A920204610BD807F70471030FEF762BC0430A9
S3150800A930FEF75FBC0170704700787047407F70472C
S3150800A94038B54378082B054619D10F490F4804F046
S3150800A950DDFD0E4C204604F0B0FD204604F0BEFD99
S3150800A96094F8293094F82A209B1A85F825302388EC
S3150800A970EB8420460321BDE8384004F0FBBE062BD5
S3150800A980E7D10349E2E700BF04620408C0110020CA
S3150800A990BA5A040841707047037F0C2B18D8DFE8B1
S3150800A9A003F0070E181E2125292D32373C40440096
S3150800A9B0002380F82430C38C5B08038407E090F8F2
S3150800A9C0253080F82430C38C5B0803840023438435
S3150800A9D0704790F8253080F82430C38CF5E790F856
S3150800A9E02530E6E790F825305B00EAE790F8253051
S3150800A9F05B00F0E790F825305B00DAE790F8253041
S3150800AA0003EB4303DDE790F8253003EB4303E2E766
S3150800AA1090F8253003EB4303CBE790F825309B00ED
S3150800AA20CFE790F825309B00D5E790F825309B00B6
S3150800AA30BFE7000030B50378012B8FB004461FD05E
S3150800AA40FFF77EFF2046FFF7A7FF124923696268D2
S3150800AA5001A836F0A1FC237F258C0F4801A98BB1EC
S3150800AA6004F042FD281A658C00EBD07005EB6000F7
S3150800AA70608494F82420618C074801AB04F0D8FC64
S3150800AA800FB030BD04F030FD638C1D442D1A65846B
S3150800AA90EFE700BF11530408C01100207047806A11
S3150800AAA0704700207047000010B5034B036004464A
S3150800AAB0FFF78AFB204610BD5853040810B5044614
S3150800AAC0FFF7F2FF20462C2134F027FD204610BD63
S3150800AAD0F7B504460F46FFF7A7FB94F82010124E69
S3150800AAE0124D2046FFF7E4FB2FB1114B3278298827
S3150800AAF0104804F09DFC104B0E481F8804F108030B
S3150800AB001946019304F0F0FC2988019B3278381A1B
S3150800AB1000EBD07001EB6001064889B2298003B0CA
S3150800AB20BDE8F04004F084BC991100209A11002079
S3150800AB30EE510408C01100209C11002037B51D46AF
S3150800AB4002230093069B0446FFF71AFB044B236077
S3150800AB5020460023C4E90953E37103B030BD00BFA2
S3150800AB605853040810B50446FFF740FB606A10BD49
S3150800AB7070B5C0E90513059B9DF810409DF8246043
S3150800AB8043609DF818300372079B04774262C360DE
S3150800AB90B4FBF6F2012306FB124400250374E4B263
S3150800ABA09DF820304374C0E90D550570C577C56317
S3150800ABB080F82060D3B20CB9837770BD0133FBE708
S3150800ABC07047416170474163704781637047C1634D
S3150800ABD070470000F0B5844E84498BB0074630466E
S3150800ABE004F094FC304604F079FC0321304604F066
S3150800ABF0C1FD97F82030042B40F0D080FB7F5BB175
S3150800AC007B49304604F070FCC0F1F90081B2784BFC
S3150800AC100522304604F00CFCBB7FFA7F013B9A42C2
S3150800AC2005D0744B0522F9216F4804F001FC7249DE
S3150800AC306D4804F06BFC6C4804F03FFC6A4804F06D
S3150800AC404DFC6948032104F095FD796901A8FEF7D2
S3150800AC5096FA6A4904A8FEF792FA694901A8FEF726
S3150800AC601FFB0246002800F0BB800823002201A92A
S3150800AC7007A8FEF743FB07A904A8FEF7D3FA07A817
S3150800AC80FEF738FA00221146049B574804F0D0FB19
S3150800AC900499554804F028FC0C23082201A9C5B2DA
S3150800ACA007A8FEF72BFB07A904A8FEF7BBFA07A817
S3150800ACB0FEF720FAFB7F002B40F08D8003214A48DF
S3150800ACC004F058FD049B48480022294604F0B0FBCE
S3150800ACD00499454804F008FC03210544424804F059
S3150800ACE049FDFB7FEDB2002B77D10F230D2201A979
S3150800ACF007A8FEF703FB07A904A8FEF793FA07A817
S3150800AD00FEF7F8F9049B38480022294604F090FB20
S3150800AD100499354804F0E8FB0F2213232C1801A9DF
S3150800AD2007A8FEF7EBFA07A904A8FEF77BFA07A817
S3150800AD30FEF7E0F9FB7F2C48012B0CBF032101210C
S3150800AD40E4B204F017FD049B27480022214604F0CC
S3150800AD506FFB0499244804F0C7FB032104442248E6
S3150800AD6004F008FD039B132201A907A8FEF7C6FAFB
S3150800AD7007A904A8FEF756FA07A8FEF7BBF9E4B236
S3150800AD80049B00222146184804F052FB04A8FEF74B
S3150800AD90B1F901A8FEF7AEF90BB0F0BD194935783F
S3150800ADA0304604F0A1FBBB7FFA7F013B281A9A4282
S3150800ADB0C4B205D0134B03222146304604F038FBB3
S3150800ADC01149094804F090FB211AC9B201390E4B02
S3150800ADD0032289B228E7012171E70E230C2286E7B0
S3150800ADE07B690146CFE700BFC01100206C6A0408E2
S3150800ADF0BF9D040878A7040804620408709B040829
S3150800AE008853040818C3040849B70408007870472B
S3150800AE10C36810B504460BB19847207010BD0000F2
S3150800AE200378052B70B5044649D0FFF7D3FE94F88E
S3150800AE302030E57F267F15FB03F52B449E42A8BFED
S3150800AE401E46AE420DDDA36994F91D2053F8250070
S3150800AE500368AA421B690CBF0121002198470135E6
S3150800AE60EFE70025237AAB4217DD636853F8250020
S3150800AE70FFF758FD237883424FEA85060BD16368AE
S3150800AE8053F82500FFF75AFDE37F834203D1636831
S3150800AE909859FFF7CFFD0135E4E72178B1B9234A80
S3150800AEA013780133DBB2072B13700FD901232370F4
S3150800AEB0117023742046BDE87040FFF7A9BF1B4AEE
S3150800AEC013780133DBB2072B01D8137070BD012547
S3150800AED0002305741370FFF79BFF2046FFF798FFC2
S3150800AEE023784BB9206B2946FFF77AF9E16AE06BBC
S3150800AEF0BDE8704000F0C0BA042BE7D194F82050A2
S3150800AF00E37F15FB03F5237FAB42DFDDA36953F827
S3150800AF10250094F91D30AB4204D10021FFF760F9F2
S3150800AF200135F0E70121FFF77AF9F9E7A2110020C8
S3150800AF300378042B70B5044640F09380836990F932
S3150800AF401D20616A53F8220003685B699847636AA3
S3150800AF501B782B2B1AD194F91D20A36953F82200CC
S3150800AF60FFF756F9002800F08D802046FFF750FFBE
S3150800AF70032323700025237FAB4240F38380A36914
S3150800AF8053F82500FFF748F90135F4E70B2B79D17B
S3150800AF9094F91D20A36953F82200FFF739F9002810
S3150800AFA070D0E3681BB394F91D20A36953F82200F7
S3150800AFB0036801219B6898472046FFF729FF94F903
S3150800AFC01D20A36953F82200FFF72BF903281FD188
S3150800AFD094F82050E37F15FB03F5237FAB4217DD7A
S3150800AFE0A36953F82500FFF717F90135F5E7032399
S3150800AFF094F820502370E37F15FB03F5237FAB42BB
S3150800B00040DDA36953F82500FFF7FFF80135F5E79A
S3150800B0102378032B36D0052B0CD1A56AE06B0023C9
S3150800B0202B7000F058FAE36BEB63E862A16AE06BF9
S3150800B03000F022FA0123606AA569237403781DB912
S3150800B04003F0DF020B2A25D10F2B25D80A2B21D98D
S3150800B0500C3B032B34D8DFE813F010013901E90063
S3150800B0606301052B14D1C36A1B78052B0DD1022366
S3150800B0700370FFF7CDFEE06BE16A00F0FDF9E06BC7
S3150800B08000F006FA0123237470BDFFF7C1FED1E76D
S3150800B090032BCFD00023F6E72B2B00F0A7802C2B11
S3150800B0A0F8D1E36A002BEFD1D4E90D12E06B00F07A
S3150800B0B0D2F9002323702046BDE87040FFF7A8BEEA
S3150800B0C045BB042323702046FFF7A2FEA66AAEB945
S3150800B0D0022323702046FFF79BFE00230121206BE5
S3150800B0E02370FFF77DF8E16A002953D00B78E06BEF
S3150800B0F0052B4DD0BDE8704000F0BEB9E06B357049
S3150800B10000F0E9F9E36BF363F062A16AE06B00F023
S3150800B110B3F9B7E72378022BDCD094F91D3055F83C
S3150800B1202300FFF777F894F91D20A369054653F81D
S3150800B1302200FFF76DF8012DA6D00328A4D094F9B4
S3150800B1401D20A36953F82200FFF76BF8A36994F949
S3150800B1501D20064653F82200036800219B6898477D
S3150800B160054610B9002E40F01081E16A0B78052BD0
S3150800B17018BF00232370BEB9E06B002DBAD0A562B4
S3150800B1802E7000F0A8F9E36BA16AE862EB6302E0AF
S3150800B190A36A13B10021E06BACE700F06DF9E06B30
S3150800B1A0BDE8704000F074B9012E0CD1002D82D094
S3150800B1B00023A5622B7094F91D20A369E06B53F850
S3150800B1C022302B63DDE7022E40F0E580002DEFD11B
S3150800B1D05AE70121FFF723F80BE1042E7FF454AF59
S3150800B1E02378032B7FF450AF26704DE7E36A002BD4
S3150800B1F03FF457AF75B920462570FFF709FE206B57
S3150800B200FFF703F8E16A002900F08880E06B00F098
S3150800B21033F904E0206BFEF7F8FF00232370E16A98
S3150800B2200B78052B04BF00230B70B4E794F91D5067
S3150800B230227F6B1C5BB29A42637709DC531E627CE1
S3150800B2405BB26377002A3FF41FAF012303701BE745
S3150800B25094F8202093FBF2F102FB1133002B7FF4C4
S3150800B26013AFA17FE37F01398B42BFF60DAF042AE6
S3150800B27001D1013326E0657706E794F91D104B1EC8
S3150800B2805BB2002B63770CDA637C0BB96377FBE65A
S3150800B2900023D4E90D12E06B6377BDE8704000F037
S3150800B2A0DAB894F820200133B3FBF2F002FB10332E
S3150800B2B0002B7FF4E9AEE37F002B3FF4E5AE042ACA
S3150800B2C002D1013BE377DFE66177DDE694F82030CB
S3150800B2D0042B05D994F91D20042A01D10323D5E7A7
S3150800B2E0E67F7EB1042B3FF4CFAE627FD21A52B20C
S3150800B2F0013EF6B2002AE677B6BF13FB06F662777A
S3150800B3006677C1E6E36A002B3FF4CEAE002D3FF424
S3150800B31072AF206BFEF779FF267080E7294675E73E
S3150800B32094F82020042A19D994F91D30022B15DD2A
S3150800B330217F01335BB29942637701DC4B1E7EE7BE
S3150800B34093FBF2F102FB1133002B7FF49DAEA27F33
S3150800B350E37F013A9342BFF697AE8AE7A17FE37F80
S3150800B36001398B42BFF690AE042A3FF48DAE617F59
S3150800B370207F114449B20133DBB28842E377617713
S3150800B3803FF782AE12FB03F380E7012E3FF493AE3C
S3150800B390022E3FF479AE032E7FF41FAF2378032BDA
S3150800B3A07FF472AEA36994F91D2053F8220003684E
S3150800B3B0DB6A984702283FF467AE2046FFF728FD68
S3150800B3C0237894F82050042B1CBF04232370E37FB2
S3150800B3D015FB03F5237FAB427FF756AEA36953F8F7
S3150800B3E0250094F91D30AB427FF4F3AE0021FEF739
S3150800B3F0F7FE0135EEE70023037470470123037453
S3150800B4007047007C704710B590F82040816102773C
S3150800B410B2FBF4F104FB1122D2B2CBB20AB983779C
S3150800B42010BD0133FBE790F91D20836953F822000C
S3150800B4307047006B704781627047806A003818BF92
S3150800B440012070470023037001230374704741608D
S3150800B450704781607047002370B5C3600123037489
S3150800B460036804461B6815469847236829462046FC
S3150800B4705B68BDE87040184709B901230374C160C9
S3150800B4807047C36813B11846FFF7CABC4368184724
S3150800B490C36813B11846FFF74BBD8368184710B544
S3150800B4A00446C06818B1FFF7ACFF207410BD207CB5
S3150800B4B0FCE710B50446C06808B1FFF79CFF0023F7
S3150800B4C0237410BD10B50446C06808B1FFF796FF8F
S3150800B4D00123237410BDC0687047436810B504463D
S3150800B4E003B1984723682046DB69BDE81040184732
S3150800B4F0704780F8C630012380F8C41080F8C5204C
S3150800B50080F8C930704702EBC20202EB810202449E
S3150800B51092F8A43092F8A30003F00F0340EA032040
S3150800B520704702EBC20202EB8102024492F8A53090
S3150800B53092F8A4001B0143EA1010704702EBC202FE
S3150800B54002EB8102024492F8A20000F07F007047E5
S3150800B55002EBC20202EB8102024492F8A20080F0DA
S3150800B5608000C009704790F89D0000F00F007047F2
S3150800B5700023A0F8C230012380F8C930704720297B
S3150800B5804FF001030CBF4FF47F42FF22A0F8C22000
S3150800B59080F8C9307047012380F8C21080F8C320AC
S3150800B5A080F8C9307047012380F8C71080F8C82092
S3150800B5B080F8C9307047407E7047C3683BB10022A7
S3150800B5C01A72012283F84820062283F881207047E0
S3150800B5D0783002F04ABB043001F0A1BD30B54F23E4
S3150800B5E097B00C4605461A46002102A835F00EF912
S3150800B5F052228DF8082011228DF8092080228DF814
S3150800B6000A20FF228DF80C2062788DF80F20227808
S3150800B6108DF81020A2788DF81120E2788DF8122086
S3150800B62022798DF8132062798DF81420A2798DF885
S3150800B63015200022E271EA7D0192AA7D0092A9896D
S3150800B640A8684F2302AA01F0B9FA17B030BDA0F1D5
S3150800B6507800C3E7783002F09FBA7C3002F099BAD6
S3150800B6607C3002F085BA7C3002F03EBA7C3002F0BB
S3150800B6705BBA000008B5B0F99430012900EE903A9B
S3150800B6800CBFB0F99630B0F9923000EE103A2DEDB5
S3150800B690028BF8EEE00AB8EEC00A33F0FDFFDFEDE4
S3150800B6A0058A9FED058A30EE280A20EE080ABDECC9
S3150800B6B0028B08BDDB0F4940E12E65421FB50446E3
S3150800B6C0783002F0D2FAE27D01924323A27D8DF80A
S3150800B6D00C3000920223A189A0688DF80D3003AAC8
S3150800B6E001F06CFA63683BB9A4F8C030FF2384F80C
S3150800B6F0C230012384F8C53004B010BD13B50C4B15
S3150800B7000446002240F8043B0A4B01F07FFD0A4B31
S3150800B710E36704F17C00019002F0A7FA074B636027
S3150800B72030330198E36702F0A0FA204602B010BD54
S3150800B73008540408B0530408C0530408CC5304083A
S3150800B74080F8C530012380F8C31080F8C42080F83B
S3150800B750C630704700EB8101D1F8B000C0F30B206A
S3150800B760704700EB8101B1F8B200C0F30B107047C7
S3150800B77000EB810191F8B00000F07F00704700EB04
S3150800B780810191F8B00080F08000C00970470F2051
S3150800B79070470023A0F8BE30012380F8C6307047F2
S3150800B7A020294FF001030CBF4FF47F42FF22A0F877
S3150800B7B0BE2080F8C6307047012380F8BE1080F896
S3150800B7C0BF2080F8C63070477047407E7047C36810
S3150800B7D03BB100221A72012283F84820062283F818
S3150800B7E081207047783002F076BB043001F097BCB0
S3150800B7F0783002F0FDBA7C3002F0F7BA7C3002F0FD
S3150800B800E3BA7C3002F09CBA7C3002F0B9BA000088
S3150800B81008B5B0F9A7300129C3F1000300EE903A44
S3150800B8200ABFB0F9A930B0F9A5305B4200EE103A6C
S3150800B8302DED028BF8EEE00AB8EEC00A33F02CFFC5
S3150800B840DFED058A9FED058A30EE280A20EE080A04
S3150800B850BDEC028B08BD00BFDB0F4940E12E6542F7
S3150800B8601FB50446783002F036FB43238DF80C30BA
S3150800B87009238DF80D30E37D0193A37D0093A189FB
S3150800B880A068022303AA01F099F963683BB9FF226D
S3150800B890A4F8C030012384F8BF2084F8C23004B06D
S3150800B8A010BD0000F0B597B00D46044647220021AA
S3150800B8B004A834F0ABFFA2238DF8083031238DF8A5
S3150800B8C0093094F8C630354F1A010133DBB20F2B15
S3150800B8D008BF002384F8C63010238DF80B30FF23E9
S3150800B8E08DF80C30F7238DF80D306B788DF80E3007
S3150800B8F02B788DF80F300DF11601AB788DF80A20EC
S3150800B90004F184008DF8143002F008FB04F17C0081
S3150800B9100DF1210102F002FB03238DF83230EB789A
S3150800B920002B14BF012302238DF835302B798DF8AF
S3150800B93037306B798DF83830AB798DF8393002A805
S3150800B940EB798DF83A304B264FF0FF330246013E2D
S3150800B9500AD310F8011B5FFA83FC81EA0C0157F839
S3150800B960211081EA1323F2E7DB43190A8DF85330D5
S3150800B9708DF85410190C1B0E8DF8563000232B72B7
S3150800B980637E0193237E8DF855100093A189A068E4
S3150800B9904F2301F013F917B0F0BD00BF98540408FF
S3150800B9A0A0F178007EE700BF37B5114B04460022A8
S3150800B9B040F8043B0F4B01F029FC00250E4BE367CA
S3150800B9C004F17C00C4E92055C4E92255A4F8C850FE
S3150800B9D0019002F080FA094B636030330198E367FF
S3150800B9E084F8CA5002F077FA204603B030BD00BF8B
S3150800B9F0A0580408B05304085854040864540408AA
S3150800BA000D4B1A7810B44AB90C4B186803681146DE
S3150800BA101C68FF23A4465DF8044B6047012A07D13A
S3150800BA20074B186803681C680023FF221946F1E7CC
S3150800BA305DF8044B704700BFA8110020AC11002028
S3150800BA40B01100200F4B10B5187068B9CC2033F030
S3150800BA5066FD0D4B19680446FFF750FE0B4B1C603C
S3150800BA600B4BA360204610BD012809D1CC2033F02A
S3150800BA7056FD054B19680446FFF796FF054BEEE79A
S3150800BA800024EFE7A8110020A4110020AC11002023
S3150800BA9001BA0008B0110020024B00221A70024BAE
S3150800BAA019607047A8110020A4110020704770473C
S3150800BAB00120704790F85000704790F87A00704758
S3150800BAC0A1F1E00358425841704740F65C23994279
S3150800BAD018D142F2E8139A421DD043690BB9008B7C
S3150800BAE0D0B140F24C53994213D1B2F51A7F12D015
S3150800BAF040F22F439A420ED040F2D533D31A584219
S3150800BB005841704740F20D539942E6D140F25A63C4
S3150800BB10E1E70020704701207047019A43BB80F88F
S3150800BB205D10D37803F00303032B22D192F9023078
S3150800BB30002B1DDA90F85610012363F3870180F86D
S3150800BB405610917803EB4303034401F00F0183F881
S3150800BB505110918883F85210937990F878209A4278
S3150800BB6038BF80F8783090F85E30013380F85E3060
S3150800BB707047022BFCD192F902100029A8BF0323B3
S3150800BB80DFE7A0F10400FFF7C8BF10B5047934B1A8
S3150800BB90012C07D0C088B0FA80F0400910BDC380D8
S3150800BBA001230371C3885BB11488002CF2D0013BD2
S3150800BBB0C3800B6801330B601388013B1380F1E7E0
S3150800BBC00371E7E72DE9FF410446ADF80A10039231
S3150800BBD00426002500F12207BDF80A20002A00F0F5
S3150800BBE0AC8094F83030042BF8D8DFE803F0030E65
S3150800BBF02022340002232372D4F80930236140F24C
S3150800BC000223A382012384F830300DF10A0203A926
S3150800BC1004F1100003F058F8002800F08E80D4F8DC
S3150800BC2009301A7884F831205B7884F83230C4F801
S3150800BC30097094F83230D4F809202261042B94F85C
S3150800BC40313008BF84F83350023BDBB22372637588
S3150800BC50237584F8306094F83230042B17D0052BFE
S3150800BC603ED0022B5CD10DF10A0203A904F11000A3
S3150800BC7003F02AF8002860D094F8253084F8343088
S3150800BC8004F12003C4F8093084F83050A4E70DF114
S3150800BC900A0203A904F1100003F016F800284CD094
S3150800BCA094F82530E02BEBD194F82630012BE7D118
S3150800BCB094F8382094F827307AB1002BE0D0012286
S3150800BCC084F8332094F8222084F8362094F8232028
S3150800BCD084F8372084F83530D2E7012BD0D1EEE747
S3150800BCE00DF10A0203A904F1100002F0EDFF20B3DA
S3150800BCF094F83330002BC3D060680028C0D004F114
S3150800BD0020020368019294F835200092D3F8008047
S3150800BD1094F8362094F8373094F83410C047AFE7D3
S3150800BD2094F83130023B9BB20DF10A0203A904F1E3
S3150800BD301800FFF72AFF0028A2D104B0BDE8F08159
S3150800BD402DE9FF410446ADF80A10039204260025A2
S3150800BD5000F12207BDF80A20002A00F0AC8094F80A
S3150800BD603030042BF8D8DFE803F0030E2022340025
S3150800BD7002232372D4F80930236140F20223A382F6
S3150800BD80012384F830300DF10A0203A904F11000EA
S3150800BD9002F09AFF002800F08E80D4F809301A784D
S3150800BDA084F831205B7884F83230C4F8097094F846
S3150800BDB03230D4F809202261042B94F8313008BFB8
S3150800BDC084F83350023BDBB223726375237584F81B
S3150800BDD0306094F83230042B17D0052B3ED0022B56
S3150800BDE05CD10DF10A0203A904F1100002F06CFF00
S3150800BDF0002860D094F8253084F8343004F1200304
S3150800BE00C4F8093084F83050A4E70DF10A0203A9F2
S3150800BE1004F1100002F058FF00284CD094F82530A1
S3150800BE20FF2BEBD194F82630012BE7D194F8382074
S3150800BE3094F827307AB1002BE0D0012284F8332019
S3150800BE4094F8222084F8362094F8232084F83720A2
S3150800BE5084F83530D2E7012BD0D1EEE70DF10A028E
S3150800BE6003A904F1100002F02FFF20B394F8333031
S3150800BE70002BC3D060680028C0D004F120020368F4
S3150800BE80019294F835200092D3F8008094F8362071
S3150800BE9094F8373094F83410C047AFE794F8313047
S3150800BEA0023B9BB20DF10A0203A904F11800FFF741
S3150800BEB06CFE0028A2D104B0BDE8F081002370B55D
S3150800BEC080F8513043F60843A0F852304FF48022E8
S3150800BED04FF48063C0E915230423044680F85C30D8
S3150800BEE000F1640500F1740655F8040B10B10368F7
S3150800BEF09B689847AE42F7D10023012284F8413067
S3150800BF0084F84230A4F8463084F87D3084F85030FE
S3150800BF1084F85E202366A4F8783084F87A3070BDF9
S3150800BF2038B5174B036034330025044643600123B4
S3150800BF3080F85E30C0E91955C0E91B5580F84150B4
S3150800BF4080F8435080F84650A0F84850C16480F8FD
S3150800BF5050500566A0F8785080F87A50FFF7AEFF83
S3150800BF60E36C3BB103F1780252F8041B21B91E3584
S3150800BF7043F82540204638BD0135102DF4D1F9E7A0
S3150800BF80685904082DE9F04704468AB09146884660
S3150800BF901D46FFF793FF94F85020E76C002A56D108
S3150800BFA03B6803921B6811463846984706460028A0
S3150800BFB04FD0D0F800A0BAF1000F4CD0039A857183
S3150800BFC004F15103036005AB0093E06C122311469C
S3150800BFD002F0D4FBC6F800A0054660B123680D2818
S3150800BFE008BF05469B68204618BFE125984728469E
S3150800BFF00AB0BDE8F0873B6802465E6841464B4694
S3150800C0003846B047014684F8500030B39DF81830DA
S3150800C010092B0AD12B462A46E06C02F0FCFB236862
S3150800C02020469B689847D125E1E79DF81B3084F8A0
S3150800C03052309DF8253084F85430BDF81C30A4F8E9
S3150800C0407630BDF81E30A4F87430E025CFE7D92540
S3150800C050CDE7D625CBE7D725C9E7D425C7E710B559
S3150800C0600446FFF72BFFE06C94F8501003689B68B2
S3150800C0709847002010BDF0B585B04023ADF80E30C6
S3150800C08090F8783000F1C907CDE90073044690F8B6
S3150800C090572090F85010C06C0DF10E0302F0E3FB28
S3150800C0A004F16405743460B9BDF80E304BB12E4600
S3150800C0B056F8040B18B1036839461B689847A64218
S3150800C0C0F6D155F8040B10B103685B689847AC4283
S3150800C0D0F7D105B0F0BD00B5B0F8863023F00103FE
S3150800C0E089B0A0F886300023CDE90613CDE90233DE
S3150800C0F0CDE90033CDE90422202390F8512090F8A9
S3150800C1005010C06C02F07EFA09B05DF804FB0023FB
S3150800C1100146A0F8863003220C2380F88920A0F86F
S3150800C1208A308931FFF7D7BFB0F8863023F010037D
S3150800C130A0F886301A2380F889304FF48673A0F861
S3150800C1408A30C368002B014614BF0323022380F8F4
S3150800C1508C3004228931FFF7BEBFB0F8863023F051
S3150800C1602003A0F886300923014680F88930102379
S3150800C170A0F88A3003228931FFF7ADBFB0F88630C0
S3150800C18023F04003A0F886300123014680F8893061
S3150800C1901023A0F88A3003228931FFF79CBFB0F834
S3150800C1A0862080F88C1022F4007210B4A0F886203D
S3150800C1B04FF488740422A0F88A4080F889205DF834
S3150800C1C0044B00F18901FFF786BFB0F8863023F0EB
S3150800C1D00203A0F88630092380F8893040F20473F8
S3150800C1E0A0F88A30C369C0F88C30038CA0F8903068
S3150800C1F00146002380F892300A228931FFF76BBF87
S3150800C200B0F8863023F00803A0F88630192380F8A2
S3150800C210893040F60423A0F88A30C369C0F88C3008
S3150800C220038CA0F8903001230146A0F89230002331
S3150800C230A0F894300D228931FFF74DBFF8B51323C6
S3150800C24080F889300C23044680F88A3008460D4663
S3150800C250FBF7E8FF013084F88B0000272846FBF738
S3150800C260E1FFFEB2F31CB04207F10107234403D9EC
S3150800C270AA5D83F88920F1E7002283F889202846F9
S3150800C280FBF7D0FF043082B204F189012046BDE8ED
S3150800C290F840FFF720BF0000012380F8893040F6F8
S3150800C2A00C03A0F88A30054B4FF0FF320146C0E96F
S3150800C2B0232389310B22FFF70EBF00BFFF1FFF00A4
S3150800C2C0562280F889204FF48672A0F88A2080F8D2
S3150800C2D08C10042200F18901FFF7FDBEB0F8863004
S3150800C2E023F08003A0F88630012380F8893040F2D5
S3150800C2F00453A0F88A30054BC0F88C3001460A234F
S3150800C30080F8903008228931FFF7E5BE338B9E30DE
S3150800C3100223014680F889300423A0F88A300322D4
S3150800C3208931FFF7D8BEB0F8862022F48172A0F8CA
S3150800C3308620052280F8892040F60452A0F88A2033
S3150800C3400A7880F88C204A7880F88D208A7880F8D8
S3150800C3508E20CA7880F88F200A7980F890204A794A
S3150800C36080F891204CF61842A0F892200122C0F8D5
S3150800C3709420002280F8982000F189011022FFF706
S3150800C380AABE00F11C01FFF7CEBFF8B50D2380F851
S3150800C390893041F20473A0F88A3090F84360C36983
S3150800C3A0C0F88C30038CA0F89030044606B390F899
S3150800C3B07B20062380F8923000F193039AB14269F4
S3150800C3C0C0F89320028B9A800022C4F89920C4F8FA
S3150800C3D09D20A4F8A12004F1890120461A22BDE86F
S3150800C3E0F840FFF778BEC269C0F89320028CEAE7E6
S3150800C3F007693846FBF716FF84F892003846FBF7BC
S3150800C40011FFF5B2A84206F1010610D805F10A0097
S3150800C410C0B2C5F11002102D00F18900D2B24FF05A
S3150800C420000188BF0022204434F0F0F9D3E77B5D91
S3150800C430254485F89330E1E70E2380F8893040F2E9
S3150800C4400463A0F88A30C369C0F88C300146038CAF
S3150800C450A0F8903009228931FFF73DBE0C2380F8F9
S3150800C460893040F20463A0F88A30C369C0F88C307A
S3150800C4700146038CA0F8903009228931FFF72BBEBC
S3150800C4802B2380F8893040F60413A0F88A30C36954
S3150800C490C0F88C30038CA0F8903003230146A0F82E
S3150800C4A09230002380F894300C228931FFF713BEAE
S3150800C4B02C2380F8893040F20463A0F88A30C369D7
S3150800C4C0C0F88C300146038CA0F8903009228931D7
S3150800C4D0FFF701BE112380F889304FF40173A0F8E5
S3150800C4E08A30438B80F88C300146C3F3032380F8E7
S3150800C4F08D3005228931FFF7EEBDB0F8862080F829
S3150800C5008C1022F00402C1F3032110B4A0F886208F
S3150800C5104FF44174062280F88D101321A0F88A4042
S3150800C52080F88E105DF8044B80F8892000F18901A7
S3150800C530FFF7D1BDF0B585B04023ADF80E3090F8C1
S3150800C5407830019300F18903009390F8542090F80D
S3150800C550501004460DF10E03C06C02F084F910F079
S3150800C560FB0F26D194F88930172B1CD80BB3013B47
S3150800C570162B1ED8DFE813F05B007900C80004010B
S3150800C580E3003601EF001D001D001D001D001D0003
S3150800C5901D001F001D001D001D001D001D001D00A3
S3150800C5A01D0025013201312B00F03D81332B00F0AF
S3150800C5B03E8105B0F0BD94F88E30002BF9D1B4F861
S3150800C5C0863043F00102A4F88620B4F88C2041F2A4
S3150800C5D001018A4208D194F88F2084F8402043F05C
S3150800C5E04103A4F88630E4E741F204018A4211D1F6
S3150800C5F09A050AD494F88F203AB994F8972012F03D
S3150800C600080218BF012284F8792043F4007343F026
S3150800C6100103E6E741F209018A42CAD1D4F88F201C
S3150800C6206261B4F89320228343F02103D9E794F892
S3150800C6308830042B13D994F8433013B994F848304A
S3150800C6406BB1002384F8883084F8413084F843308D
S3150800C65084F8463084F848300A2384F8813094F800
S3150800C6608830013384F88830A3E794F88B50002D7E
S3150800C6709FD0EE0094F843C0F6B2002101EB4103C7
S3150800C680334454FA83F393F88D0093F88E2093F885
S3150800C6908F30BCF1000F1BD0D3B9052A18D110F082
S3150800C6A00C0F15D084F88030012384F87E0084F8B6
S3150800C6B07F2084F87C30062202FB01418C3104F18C
S3150800C6C01C0034F089F8B4F8863043F0800388E714
S3150800C6D094F848706FB102F00F07052F09D110F0D2
S3150800C6E0C80F06D084F87E0084F87F2084F880304E
S3150800C6F0E1E70131CFB2BD42C0D884F87E0084F8A4
S3150800C7007F2084F8803054E7B4F8862042F480739A
S3150800C710A4F8863094F88B306BB994F88D3094F879
S3150800C7208C101B0203F470630B4342F4817263831B
S3150800C730A4F886203DE7062384F8813039E794F883
S3150800C7408B30002B7FF435AFB4F8863023F0020324
S3150800C75043F0040345E794F88B30002B7FF429AFA8
S3150800C76004F1220304F1400193F8702003F8012B29
S3150800C7700AB18B42F8D1B4F8863043F0080330E7A3
S3150800C780D4F88B30E361B4F88F30238494F8923070
S3150800C79084F87F3003F00F0394F8912094F89310EF
S3150800C7A084F87E20052B84F8801005D112F0C80F76
S3150800C7B01CBF012384F84730B4F8863043F01003D1
S3150800C7C00FE794F84330204613B1FFF7DEFDF0E695
S3150800C7D02369002BF9D1FFF72FFEEAE62046FFF77B
S3150800C7E03DFEE6E694F88B30BBB994F8433033B196
S3150800C7F094F841301BB9012384F84130D9E694F8FE
S3150800C8004830002B3FF4D5AE94F84630002B7FF421
S3150800C810D0AE012384F84630CBE6618B2046FFF77D
S3150800C8206CFE102388E72046FFF72AFEC1E620465D
S3150800C830FFF73EFEBDE6242380F889304FF44373A4
S3150800C840A0F88A3040F604030146A0F88C3000238D
S3150800C85080F88E3006228931FFF73DBC70B590F816
S3150800C86081300446132B27D8DFE813F0140027007D
S3150800C8704E00590064006E009500A000B100BD008E
S3150800C880CC00E600F20046012600580164017B0050
S3150800C89087008F00B0F88230B0F8842001339BB24D
S3150800C8A09A42A0F8823007D2FFF731FC012384F8B8
S3150800C8B081300023A4F8823070BDB0F88220B0F829
S3150800C8C08630013292B2DE07A0F8822009D500230D
S3150800C8D0A0F88230022380F88130BDE87040FFF767
S3150800C8E0AABFB0F884309A42E6D903EB83035B000B
S3150800C8F09BB2B3F5FA6F88BF4FF4FA63A0F8843099
S3150800C900002380F88130D5E7B0F88630DD07D3D527
S3150800C910032380F88130BDE87040FFF71EBCB0F8ED
S3150800C92086309806C8D52046FFF728FC042384F8E5
S3150800C9308130C1E7B0F886305906BDD5C16839B12E
S3150800C940FFF77CFC0523F2E7B0F88630DA07B3D5A3
S3150800C95094F84930EBB100212046FFF720FC11235B
S3150800C960E5E7B0F886309B05A6D590F8793083B10F
S3150800C9700121FFF7A5FC1223D9E7B0F88630DE07B8
S3150800C9809AD5FFF789FC1323D1E7B0F88630DD077F
S3150800C99092D50623CBE790F8483013B990F8433080
S3150800C9A053B32046FFF79AFC0723C0E7B0F8863052
S3150800C9B0180681D52046FFF7ABFC94F87C3023B1E6
S3150800C9C02046FFF71DFC0C23B1E70823AFE7B0F8B4
S3150800C9D08630D9077FF570AF002380F87C30FFF7E3
S3150800C9E0D0FC0923A3E7B0F88630DA057FF564AFF3
S3150800C9F09E0703D5FFF76EFD0A2398E7BDE870404A
S3150800CA00FFF7BFBC90F84130002B7FF455AF90F884
S3150800CA104330002B7FF450AF90F84630002B7FF45C
S3150800CA204BAF90F84830002B7FF446AFFFF77CFBFE
S3150800CA30012323720B237AE7B0F88630DD0602D588
S3150800CA4000230372BCE758077FF536AF10236EE75D
S3150800CA50B0F8863019077FF52FAF00F12205444953
S3150800CA600822284634F010FD70B90126A4F84400BF
S3150800CA7084F87B003F4984F842601622284634F041
S3150800CA8003FD10BB84F8446094F8803073B9B4F899
S3150800CA907E2042F208539A4208D137491322284683
S3150800CAA034F0F2FC10B9012384F87D3094F8433051
S3150800CAB013B994F848301BB194F87C30002B84D114
S3150800CAC02046FFF782FB0D2331E72C49162228461C
S3150800CAD034F0DAFC30B940F2011384F87B60A4F82C
S3150800CAE04430D1E726491322284634F0CDFC0028E5
S3150800CAF0CAD184F87B60C7E7B0F886309A077FF515
S3150800CB00DBAE90F87D3013B1012380F84630002360
S3150800CB1063726381A4F886300F2308E7B0F8823081
S3150800CB2001339BB2B3F57A7F7FF6C4AE0023A0F833
S3150800CB30823061E7B0F886305B077FF5BDAE002529
S3150800CB40A0F8865040222946893033F05FFE4022FD
S3150800CB50294604F1C90033F059FE84F84150A4F877
S3150800CB604250A4F8465084F84850A4F87C5043E74D
S3150800CB70E8580408F1580408335904080859040801
S3150800CB801F59040890F87A3010B50446A3B129F065
S3150800CB90C1FD236EC01A00280EDB29F0BBFD94F8F0
S3150800CBA07830184420662046FFF7C4FC2046FFF775
S3150800CBB055FE2046FFF75FFA002010BD2DE9F0412B
S3150800CBC01E460F3382B003F4FC7302AFADEB030DC0
S3150800CBD0331D8DF80A301B120D468DF80B300023D5
S3150800CBE080468DF808508DF80D30C5F303253B7E39
S3150800CBF08DF80E3011463B7F8DF80F30324602AC69
S3150800CC0045F0200504A88DF809508DF80C6033F01E
S3150800CC10D5FD98F85A2098F85010D8F84C0000948A
S3150800CC2006F1080301F03CFE10B1642029F078FDF6
S3150800CC30BD46BDE8F08173B5BDF8185080F80A21E5
S3150800CC40042280F80B2180F80D51002202262D0AB5
S3150800CC5080F80C2180F8096180F80E511D7880F85B
S3150800CC600F515B7880F8103101230192009300F28E
S3150800CC7009120823FFF7A2FF02B070BDF0B480F8CE
S3150800CC800A21082280F80B210327002280F80C21AC
S3150800CC9080F809711F7880F80D715B78049D80F81B
S3150800CCA00E312B7880F80F316B789DF8146080F878
S3150800CCB0103101230592049380F81161A0F812211E
S3150800CCC080F81421F0BC0C2300F20912FFF776BF96
S3150800CCD037B580F80A21082280F80B21042500229E
S3150800CCE080F80C2180F809511D7880F80D515B7881
S3150800CCF080F80E31084BC0F81031FF2380F8143144
S3150800CD00012380F80F210192009300F209120C23E7
S3150800CD10FFF754FF03B030BD000102FF37B580F8B6
S3150800CD200A210A2280F80B210525002280F80C2109
S3150800CD3080F809511D7880F80D515B7880F80E311E
S3150800CD404FF08073C0F810314AF20203A0F814318C
S3150800CD50022380F81631012380F80F2101920093EF
S3150800CD6000F209120E23FFF729FF03B030BD73B591
S3150800CD7080F80A21042280F80B210626002280F872
S3150800CD800C2180F809611E7880F80D615B78069D94
S3150800CD9080F80E312B7880F80F316B7880F81031D7
S3150800CDA001230192009300F209120823FFF706FFF8
S3150800CDB002B070BD73B580F80A21042280F80B21F1
S3150800CDC00726002280F80C2180F809611E7880F871
S3150800CDD00D615B78069D80F80E312B7880F80F314F
S3150800CDE06B7880F8103101230192009300F2091242
S3150800CDF00823FFF7E3FE02B070BD37B580F80A21B5
S3150800CE0080F80D3108229DF8183080F80B2180F83B
S3150800CE100E3100220B25012380F80C2180F80F2102
S3150800CE20C0F8102180F814210192009380F8095166
S3150800CE300C2300F20912FFF7C1FE03B030BD10B58E
S3150800CE408AB001238DF8203000238DF821300DF1AA
S3150800CE5022028B1D13F8014D02F8014B8B42F9D1C2
S3150800CE6008AA069200230822CDE904220793039311
S3150800CE700322F523CDE901320923009390F85120C6
S3150800CE8090F85010C06C212301F0BCFB0AB010BD0D
S3150800CE9000B58DB010228DF82B2001228DF82C209C
S3150800CEA002228DF82D2012228DF82E200A68CDF840
S3150800CEB025208A88ADF8292009A90022079206911B
S3150800CEC0039205230B210322CDE90132CDE9041192
S3150800CED08DF824300923009390F8512090F85010CB
S3150800CEE0C06C212301F08EFB0DB05DF804FB000039
S3150800CEF02DE9F04FD0F84C9090F8548090F85010E7
S3150800CF004FF0000A80F854A01F46D9F8003093B0B5
S3150800CF101B68044648469847064620B9D62528463B
S3150800CF2013B0BDE8F08F4FF4967029F0F9FB94F82A
S3150800CF305030E06C5246514601F06DFC054630B162
S3150800CF4086F806A0236820469B689847E7E7D9F83D
S3150800CF500030B0711B6894F850104846984700286E
S3150800CF60DCD0877104F1510794F85010E06C3B4609
S3150800CF70012201F0F9FA05460028E3D1B4F8762033
S3150800CF8040F24C539A4244D1B4F87430B3F51A7F40
S3150800CF9007D040F22F42934203D040F2D532934253
S3150800CFA037D1642029F0BCFB94F8512094F850102E
S3150800CFB0E06C012301F046FC05460028C2D16369EE
S3150800CFC00BB9238B6BB1B4F87430B3F51A7F04F13F
S3150800CFD01401204603D040F22F42934216D1FFF7A0
S3150800CFE02EFF94F8512094F85010E06C002301F0BD
S3150800CFF029FC00231A4694F85010E06C01F00BFC4B
S3150800D000236820469B689847D12588E7FFF740FFA5
S3150800D010E7E7DFF8D890DFF8D8A0DFF8D8B02E46D3
S3150800D020F3B29845E06C94F850102CD9D4F874E013
S3150800D030CE4504F1040203AD0DF12C0C01D0DE45FA
S3150800D0402ED1CDF80CA00492009500228DF814205C
S3150800D050ADF820200A92ADF83C208DF83E208DF8D8
S3150800D0604420CDF815C0CDF81CC0CDF824C001F079
S3150800D070ADFB054600287FF465AF94F85E30032BB8
S3150800D08006F10106CCD994F85E20E06C94F85010AD
S3150800D090032A0AD800231A4601F0BDFBD12551E719
S3150800D0A0DFF854E0CDF80CE0CDE73B4601F05CFA3A
S3150800D0B0054600287FF446AF94F85D3094F8512071
S3150800D0C094F85010E06C01F0BDFB054600287FF48B
S3150800D0D039AF6423A4F884300123A4F8820084F8C5
S3150800D0E08100207284F87A3019E700BFE8215C0ACB
S3150800D0F0505904085A060D055C59040870477047CC
S3150800D10070470022036880F871200A2181761B6A1D
S3150800D110427580F8692080F86A200261184790F8FD
S3150800D1206A3013B5044663B1027D013200F16F031C
S3150800D130D2B202750093818900F11B038068FFF75C
S3150800D14016FE227DA189A0680132D2B204F16D03D0
S3150800D1502275009304F11803FFF709FE2368204699
S3150800D1609B6898470E23A376092384F8713002B08A
S3150800D17010BD7FB590F871300446DBB9806890F829
S3150800D1804630CBB1437ABBB9637DABB994F8692015
S3150800D19092B901234372418B84F8693011230093B5
S3150800D1A0A18104F16B0322612275FFF744FD022376
S3150800D1B084F8713004B070BD2369DB07FAD50126FF
S3150800D1C004F1160504F16B03227DA1890393CDE9C9
S3150800D1D00056FFF753FD304629F0A2FA0022A1892E
S3150800D1E0039BA068CDE90052227DFFF747FD237D0A
S3150800D1F033442375304629F093FA2B46227DA189BC
S3150800D200A068FFF765FD0423D2E7000070B5044661
S3150800D210816041B101F16405002055F8046BC6B977
S3150800D22001EB800044660B610C48206070230020E7
S3150800D23084F86B300A4B84F86800C4E9080084F85F
S3150800D240700081F848202046E366FFF75AFF20461B
S3150800D25070BD01300428E0D1E5E700BFA8590408ED
S3150800D260007100507FB5837E0B2B044645D00E2BEC
S3150800D2704ED00A2B3FD1036913F480722AD000F1ED
S3150800D2801B05012623F480730361CDE9005600F1DE
S3150800D2906F03027D818980680393FFF7EFFC3046B0
S3150800D2A029F03EFA0022A189039BA068CDE9005225
S3150800D2B0227DFFF7E3FC237D33442375304629F0AE
S3150800D2C02FFA2B46227DA189A068FFF701FD0B23C3
S3150800D2D0A37610E059050ED523F48063036100F1A7
S3150800D2E01B0380F86A200093027D818900F16F0391
S3150800D2F08068FFF75FFD04B070BD03699A05FAD52B
S3150800D30023F400730361012380F86A300A23DFE7F8
S3150800D31003695B04EFD581898068FFF7EEF84FF65D
S3150800D320FF73A38123689B68204604B0BDE870405C
S3150800D330184707B51346027F0192C27E00920A4635
S3150800D34081898068FFF73AFC03B05DF804FB0000AA
S3150800D35010B480F829100724084980F82A200022EA
S3150800D36080F8284080F82B20C16202865DF8044BBD
S3150800D3700A2200F12801FFF7DCBF00BF05000235CD
S3150800D3801FB590F86830012B84BF002380F86830F9
S3150800D39090F8683043F070038DF80F30C37D019321
S3150800D3A0837D00938189806801230DF10F02FFF7C1
S3150800D3B005FC05B05DF804FB7FB590F87130023BBB
S3150800D3C00446072B77D8DFE803F03746048A0D5C56
S3150800D3D0667803699A076ED5FFF7D2FF062384F8A5
S3150800D3E0713068E00369DB0665D500F1180501268A
S3150800D3F0CDE9005600F16D03027D818980680393AB
S3150800D400FFF73CFC304629F08BF90022CDE90052A3
S3150800D410039B227DA189A068FFF730FC237D334456
S3150800D4202375304629F07CF9227D2B46A189A06810
S3150800D430FFF74EFC0823D2E703695E073BD5027D5A
S3150800D44081890132D2B200F1160302758068FFF7AE
S3150800D4503FFC0323C3E703699D072CD5FFF790FF1D
S3150800D460012029F05DF9227DA189A0680132D2B296
S3150800D47013230093227504F16D03FFF7DCFB0723E2
S3150800D480ADE70369580616D5227D0132D2B2227558
S3150800D49004F11803CAE7036999060CD583680022C4
S3150800D4A083F8462083F84820036801251B694575DB
S3150800D4B0984784F8715004B070BD03691A06FAD506
S3150800D4C0027D013200F16B03D2B2027500938189A5
S3150800D4D000F116038068FFF74AFC05237FE7036916
S3150800D4E01B07E8D581898068FFF707F84FF6FF73B1
S3150800D4F0A3810023236172E773B504460D46637D55
S3150800D500806863B90B7A022B09D18B89012B06D166
S3150800D510827A22B98372438BA3810A23A376437A3C
S3150800D520BBB990F84730A3B1637D93B994F86930D5
S3150800D5307BB92A7A022A0CD1AA89112A09D1012291
S3150800D540427280F8473084F86920428BA28184F8B9
S3150800D55071302A78237BA1899A4240F0D8816A786B
S3150800D5600B0A43F020039A4240F0D181EB88012B45
S3150800D57040F04A812B7A012B1CD0032B4AD12B8AE7
S3150800D580C3B96B8AB3B9AB7B94F86F209A421AD1A8
S3150800D590EE7B94F87020964215D16A7A22752B7B19
S3150800D5A0E37601326B7B2377D2B2227504F11B0333
S3150800D5B0FFF78EFB2046FFF755FE204602B0BDE872
S3150800D5C07040FFF7F9BE94F86B209A420FD1E97BB9
S3150800D5D094F86C2091420AD16B7A23752B7BA3753C
S3150800D5E06B7BE375236943F004032361E2E794F850
S3150800D5F06D209A42DED1EA7B94F86E309A42D9D1F0
S3150800D6006B7A23752B7B23766B7B6376236943F0D2
S3150800D6104003EAE7022B24D1AB89012B09D16B7AA7
S3150800D6202375AB7BE376EB7B2377236943F480731F
S3150800D630DBE7112B09D16B7A2375AB7BA375EB7BE3
S3150800D640E375236943F00103CFE7132BB2D16B7A55
S3150800D6502375AB7B2376EB7B6376236943F0100354
S3150800D660C3E7052B31D12B8A002BA3D12B7B94F84A
S3150800D6706F209A420AD1697B94F87020914205D1AD
S3150800D6806B7A2375236943F40073AEE794F86B202D
S3150800D6909A420AD1697B94F86C20914205D16B7A3B
S3150800D6A02375236943F002039FE794F86D209A4295
S3150800D6B080D16A7B94F86E309A427FF47BAF6B7A9E
S3150800D6C02375236943F020038FE7042B29D12B7B8D
S3150800D6D094F86F209A420AD16E7B94F8702096428D
S3150800D6E005D104F11B036A7AFFF718FB62E794F881
S3150800D6F06B209A4207D16E7B94F86C20964202D131
S3150800D70004F11603EFE794F86D209A427FF452AFBE
S3150800D7106A7B94F86E309A427FF44CAF04F1180392
S3150800D720E1E7062B39D12B7B94F86F209A420AD170
S3150800D7306E7B94F87020964205D16B7A237523691F
S3150800D74043F4806351E794F86B209A4212D16E7BBA
S3150800D75094F86C2096420DD16A7A227504F1160364
S3150800D760009304F16B03FFF725FB236820469B68AB
S3150800D77098471FE794F86D209A427FF41BAF6A7B9F
S3150800D78094F86E309A427FF415AF6A7A227504F1DE
S3150800D7901803009304F16D03E5E7072B29D12B7BCA
S3150800D7A0E27E9A4209D1697B227F914205D16B7A42
S3150800D7B02375236943F4804317E7A27D9A4209D16A
S3150800D7C0697BE27D914205D16B7A2375236943F023
S3150800D7D008030AE7227E9A427FF4ECAE6A7B637EF0
S3150800D7E09A427FF4E7AE6B7A2375236943F0800388
S3150800D7F0FBE60A2B7FF4DEAE6A7A22756B7B009312
S3150800D8002B7BFFF7FAFAD5E6AA7994F86F10EB792D
S3150800D810914235D194F87010994231D12B7A022B66
S3150800D82015D1032384F828306B7A84F82930AB7A2B
S3150800D83084F82A30002384F82B300522E2622386F6
S3150800D8400A2204F128012046FFF773FDB2E6042BED
S3150800D8500DD1052384F828306B7A84F82930AB7A01
S3150800D86084F82A3000232B4A84F82B30E6E7062B67
S3150800D8707FF4A0AEAA7A697A2046FFF769FD99E691
S3150800D88094F86D1091422AD194F86E10994226D1D7
S3150800D8902B7AA12B7FF48EAE28F03CFF6067AE880A
S3150800D8A02368F6B2711E5B6905F10902C9B2204602
S3150800D8B098476B7A012B04D0022B7FF47BAE606A03
S3150800D8C000E0206A00283FF475AE02680A35B31EE8
S3150800D8D000951568DBB200222146A8476AE694F847
S3150800D8E06B1091427FF466AE94F86C209A427FF4EE
S3150800D8F061AE2B7AA32B7FF45DAEA9882368013924
S3150800D9009B6905F10902C9B22046984752E602B05A
S3150800D91070BD00BF05000235002800F0A780132857
S3150800D92000F08780012800F0A180142800F0838089
S3150800D930022800F09B8015287FD0032800F09680E7
S3150800D94016287CD0A0F10803DBB21E2B03D9332896
S3150800D95006D104207047464A22FA03F3DA07F8D4B8
S3150800D96000F0EF03092B6CD0A0F12703012B68D92F
S3150800D9700A2868D0292866D00B2866D02A2864D0B9
S3150800D980A0F10E03DBB21D2B04D83A4A22FA03F3A0
S3150800D990DB075CD4A0F10F03DBB21D2B03D90C28DF
S3150800D9A008D10A207047334A22FA03F3D90709D562
S3150800D9B0092070472D28F4D00D284AD02E2848D0A3
S3150800D9C0042848D01E2846D0052846D01D2844D00D
S3150800D9D0062844D01F2842D0072842D0202840D005
S3150800D9E0A0F11003DBB21F2B04D8234A22FA03F353
S3150800D9F0DA0738D4A0F11103DBB21F2B04D81F4A6B
S3150800DA0022FA03F3DB0730D4A0F11203DBB21F2B93
S3150800DA1005D932280CBF13204FF0FF307047184A3B
S3150800DA2022FA03F313F0010F0CBF4FF0FF30122058
S3150800DA307047002070470120704702207047032076
S3150800DA407047052070470620704707207047082052
S3150800DA5070470B2070470C2070470D2070470E202A
S3150800DA6070470F207047102070471120704700BF7D
S3150800DA70018009420100402001000480010204805F
S3150800DA800104008008B5FFF747FFC3B2122B28BF71
S3150800DA904FF0FF3008BD032921D8DFE801F0020D59
S3150800DAA0161B037A03F00F02072A1AD013F00E0F7B
S3150800DAB00CBF012000207047007A00F00F000138E3
S3150800DAC002288CBF002001207047007A00F00F0062
S3150800DAD00338F5E7007A00F00F000538F0E7002074
S3150800DAE0704701207047000013B5044608460191A7
S3150800DAF0FFF7C8FF031E12DB032B06DC019920463D
S3150800DB0002B0BDE81040FFF7C6BF064AA068D35C5E
S3150800DB10C0F31700D84000F0010002B010BD002085
S3150800DB20FBE700BFCC59040810B504460846FFF7C2
S3150800DB30A9FF002817DB0D4BB4F844101A5C012323
S3150800DB4003FA02F294F8433043EA0123134223EA24
S3150800DB50020384F843304FEA132314BF0120002040
S3150800DB60A4F8443010BD0020FCE700BFCC590408D7
S3150800DB7010B504460846FFF785FF031E07DB082B8A
S3150800DB8001D1E07A10BD092B01D1207BFAE70020EC
S3150800DB90F8E7014408797047012910B5044610468C
S3150800DBA04CD9002A4AD01378012B52D14B1EDAB22F
S3150800DBB03C2A28BF3C22411C201D32F0FFFDA268EA
S3150800DBC0236CC2F31702C3F317039A4236D022EA2C
S3150800DBD0030384F843301B0AA4F84430236C62F329
S3150800DBE01703236400212046FFF755FF237A03F025
S3150800DBF00F035A1E022A98BF40F00200A3F103023F
S3150800DC0098BFC0B2022A98BF40F00400A3F10503EA
S3150800DC1098BFC0B2022B98BF40F0080094F84E3067
S3150800DC2098BFC0B2834209D094F8432084F84E00C6
S3150800DC3020EA030363F3030284F8432094F84D3083
S3150800DC4093B12146204651F8463BBDE810401B6873
S3150800DC501847112B08D1032906D9CB1EDAB23C2A5C
S3150800DC6028BF3C22C11CA7E710BD90F8263043F018
S3150800DC70800380F8263090F82A3043F0800380F835
S3150800DC802A3090F82F3043F0800380F82F3090F830
S3150800DC90333043F080034FF07F3280F83330082367
S3150800DCA0C0E9012390F8382042F0800280F8382035
S3150800DCB090F83C2042F0800280F83C20026C02F08A
S3150800DCC07042002342F0080203730264A0F846304B
S3150800DCD08364A0F84C3080F84E30704708B5FFF7DB
S3150800DCE01BFEC3B2132B28BF4FF0FF3008BD032914
S3150800DCF021D8DFE801F0020D161BC37E03F00F02E0
S3150800DD00072A1AD013F00E0F0CBF01200020704707
S3150800DD10C07E00F00F00013802288CBF00200120C9
S3150800DD207047C07E00F00F000338F5E7C07E00F0AC
S3150800DD300F000538F0E70020704701207047000003
S3150800DD4013B5044608460191FFF7C8FF021E13DB08
S3150800DD50032A06DC0199204602B0BDE81040FFF709
S3150800DD60C6BFE37EA08B43EA0020044B9B5CD840E9
S3150800DD7000F0010002B010BD0020FBE7DE590408E0
S3150800DD8010B504460846FFF7A9FF002817DB0D4B18
S3150800DD90B4F840101A5C012303FA02F294F83F30F3
S3150800DDA043EA0123134223EA020384F83F304FEA89
S3150800DDB0132314BF01200020A4F8403010BD002012
S3150800DDC0FCE700BFDE59040810B504460846FFF70D
S3150800DDD085FF031E07DB082B01D1207E10BD092B0A
S3150800DDE001D1607EFAE70020F8E70144087D704714
S3150800DDF0012970B50446104652D9002A50D0137826
S3150800DE00012B5CD14B1EDAB2282A28BF2822411CD6
S3150800DE1004F1140032F0D2FCE57EA28BE36B45EAEE
S3150800DE200222C3F317039A4235D022EA030384F881
S3150800DE303F301B0AA4F84030E36B62F31703E36331
S3150800DE4000212046FFF753FF05F00F035A1E022A4A
S3150800DE5098BF40F00200A3F1030298BFC0B2022A9D
S3150800DE6098BF40F00400A3F1050398BFC0B2022B87
S3150800DE7098BF40F0080094F84B3098BFC0B2834270
S3150800DE8009D094F83F2084F84B0020EA030363F393
S3150800DE90030284F83F20B4F84C300133A4F84C3020
S3150800DEA094F84A301BB9E37A0BB9E37C93B121465F
S3150800DEB0204651F8423BBDE870401B681847312B95
S3150800DEC008D1022906D08B1EDAB2282A28BF2822B2
S3150800DED0811C9DE770BD0822C2764FF07F324261F1
S3150800DEE090F8342042F0800280F8342090F83820E8
S3150800DEF042F0800280F83820C26B02F0704200239C
S3150800DF0042F00802C0E9113383830371C3720373B5
S3150800DF10C3740383C263A0F8423070470378262B84
S3150800DF2012D007D8012B09D0022B07D000230B707B
S3150800DF304B7007E0FC2BF9D10B7018E00B70437897
S3150800DF404B7083788B7012E00B704378DB434B7011
S3150800DF5083780BB102238B70C3780B7103794B71ED
S3150800DF6043798B7183795B0808BF01234B720023C1
S3150800DF70C371704702480122102129F0B5BA00BFC3
S3150800DF800010024002480022102129F0ADBA00BF55
S3150800DF90001002401FB50F4C8DF80700FFF7F2FF7F
S3150800DFA00DF107014FF0FF33012220462BF09AFFAF
S3150800DFB000238DF80F3001224FF0FF330DF10F01CA
S3150800DFC020462CF031F9FFF7D5FF9DF80F0004B075
S3150800DFD010BD00BF2091012037B504460D4644F018
S3150800DFE00204FFF7CFFF4FF0FF33022201A90548CD
S3150800DFF08DF804408DF805502BF074FFFFF7BAFF33
S3150800E00003B030BD209101202DE9F04F1D4687B0A1
S3150800E0104B780293013B3F2B0C46039200F2BA80E1
S3150800E02028F078FB00F59C5308330193A378DFF8B2
S3150800E0306CB113F0010F14BF80214021E820FFF7CF
S3150800E040CBFF4FF00008002D00F09480029BAB42F6
S3150800E05028BF2B4699465FFA83FAFFF793FF1223E8
S3150800E0608DF8173001224FF0FF330DF1170158468E
S3150800E0702BF038FF10994FF0FF334A4658462BF0DD
S3150800E08031FFFFF777FF51463820FFF7A5FF2178C4
S3150800E090F02041F02001FFF79FFFC820FFF77AFF25
S3150800E0A00206FAD58021C820FFF796FFF820FFF769
S3150800E0B071FF002600F00F083746B8F1000F19D097
S3150800E0C028F028FB019BC01A002813DAB8F1060FBE
S3150800E0D01BD0B8F10E0F14D0B8F1040F05D1039B6D
S3150800E0E00136B6B223B39E4222D100213820FFF76B
S3150800E0F073FF42E0109BA5EB09054B44ADB21093A4
S3150800E100A1E70137FFB2032FEEE7F820FFF742FF3A
S3150800E110A37880F02000C0F3401060F3000313F0EA
S3150800E120010FA37014BF80214021E820FFF754FF98
S3150800E13000213820FFF750FF109B10201978FFF7B1
S3150800E1404BFF51463820FFF747FF2178F02041F072
S3150800E1502001FFF741FFC820FFF71CFF0306FAD589
S3150800E1608021C820FFF738FFF820FFF713FF00F0DB
S3150800E1700F08A2E7B8F1000FB7D1F820FFF70AFF9A
S3150800E180A378C0F3401060F30003A370404607B0BD
S3150800E190BDE8F08F4FF0DA08F8E700BF20910120BC
S3150800E1A02DE9F04788469246994628F0B3FA0024A6
S3150800E1B000F59C5608362746254648EA0A0828F0F8
S3150800E1C0A9FA801B00281ADA4146F020FFF704FF57
S3150800E1D028F0A0FA801B002808DAC820FFF7DAFE24
S3150800E1E00306F5D58021C820FFF7F6FEF820FFF7CD
S3150800E1F0D1FE00F00F05042D04D00E2D0AD02846B6
S3150800E200BDE8F0870134A4B2B9F1000FD7D04C4568
S3150800E210D5D1F4E70137FFB2032FF9E72DE9F04F1F
S3150800E2202DED028B85B01E469DF8443000934B7841
S3150800E23001930023B6F8009033808B78DDF840A070
S3150800E240DFF810B113F0020F0D4608EE100A14BFDE
S3150800E25020211021E82008EE902AFFF7BDFE18EECF
S3150800E260903A2A7818EE100A0021FFF799FF062837
S3150800E270804613D1F820FFF78DFEAB7880F01000AA
S3150800E280C0F3001060F3410313F0020FAB7014BF24
S3150800E29020211021E820FFF79FFEE0E7002848D15B
S3150800E2A0C820FFF777FE430750D53020FFF772FEE8
S3150800E2B03488A9EB0404484524B2074624EAE474E2
S3150800E2C0C8BF5FFA89F7BC424FF00803A8BF3C46AF
S3150800E2D08DF80F30FFF756FE4FF0FF3301220DF190
S3150800E2E00F0158462BF0FEFD22460021504632F01B
S3150800E2F08DFA4FF0FF33A2B2514658462BF094FFE1
S3150800E300FFF738FE0421C820FFF766FE3388019A16
S3150800E3103B449BB29742A244338001D34B450ED36C
S3150800E320F820FFF737FEAB78C0F3001060F341031F
S3150800E330AB70404605B0BDEC028BBDE8F08F009B84
S3150800E340002B8CD0184628F0EBF988E74FF0F00838
S3150800E350EFE700BF209101202DE9F84F9DF828A08E
S3150800E360074615461E464FF0000900EB810802F1E4
S3150800E3701E0BD8F87800036832465C68294653466F
S3150800E380A047E028044626D1F5B9E8200121FFF781
S3150800E39023FE662028F0C4F9D8F8780003683246C8
S3150800E3A01C6829465346A0470D28044624D15FFA1F
S3150800E3B089F3022B15D915BB0121E820FFF70CFEBE
S3150800E3C0662028F0ADF914E057F82B0003683146AB
S3150800E3D05B699847E0E70D2809D15FFA89F3022BB4
S3150800E3E007D8642028F09CF909F10109C1E700283B
S3150800E3F0D2D02046BDE8F88F0028FAD0DBE71E35D4
S3150800E400314657F8250003685B699847F1E7012309
S3150800E41070B5024600211E46051DC3EBC30404441D
S3150800E4200133102BD17416755175A56002F10702D8
S3150800E430F3D1C17170BD000038B50A4B03604FF4C3
S3150800E44080738381031D00258360074B85734360B2
S3150800E4500446FFF7DCFF054B84F8B85011221A7002
S3150800E460204638BDFC59040800083C00B5110020B8
S3150800E47010B5012300F10C02C3EBC304D8B2145D36
S3150800E4808C4203D00133102BF6D1002010BD2DE9A4
S3150800E490F84399460B0605460F4690463DD4B9F112
S3150800E4A0070F3AD812B1C379072B36D00021284670
S3150800E4B0FFF7DEFF044670B1C60097B9331A2B443E
S3150800E4C0B8F1000F0AD041221A73EB790133EB71C8
S3150800E4D0361A35442C7B2046BDE8F88301221A7388
S3150800E4E0F6E74FF00004C7F3020767F3C504B8F16F
S3150800E4F0000F0FD0EB790133DBB2EB7103F00703A2
S3150800E50043F0400324F047041C43361A35442C7361
S3150800E510E4B2E0E769F30204F7E70024DBE710B5A5
S3150800E520044609B9083010BDFFF7A2FF0028FAD043
S3150800E53000B20834C0EBC0002044F4E710B5144616
S3150800E540FFF7EDFF034668B1006860B15A7900230A
S3150800E550D9B28A4206D90178A14203F1010302D051
S3150800E5600330F5E7002010BD70B50E4615461C466B
S3150800E5703BB1FFF7D4FF30B1067104604571002046
S3150800E58070BDD820FCE7D620FAE7F7B505460E4653
S3150800E59001921F46FFF7C3FF044660B3036863B3DF
S3150800E5A0019A31462846FFF7C9FF386038B38378A1
S3150800E5B09B080F2B28BF0F231A4601239340089A5E
S3150800E5C0013B13803146E020FFF706FDD820FFF710
S3150800E5D0E1FCA37901465BB195F8B800014341F027
S3150800E5E00201C9B2D820FFF7F7FC002003B0F0BD3E
S3150800E5F000F0F901F6E7D620F8E7D720F6E7DB20A2
S3150800E600F4E700002DE9F04F2DED028B89B01E4688
S3150800E61000230593ADF80E300DF10E03009305ABFC
S3150800E620DDE91ABA08EE102ABDF86090BDF86480D4
S3150800E6300546FFF7AAFF0446002840F090809DF89B
S3150800E64050308DF819309DF854308DF81A309DF8F1
S3150800E65058308DF81B30BDF85C30ADF81C308DF89D
S3150800E6601860ADF81E90FFF78DFC22238DF8123046
S3150800E67001224FF0FF330DF112013F482BF032FC17
S3150800E6804FF0FF33082206A93B482BF02BFCFFF777
S3150800E69071FCBDF80E3018EE102A10212846FFF737
S3150800E6A07FFD044600285AD176B2BBF1000F5CD034
S3150800E6B00599002E8B783CDA43F002038B704E46A0
S3150800E6C0002E55D00023CDE900B3BDF80E200599DC
S3150800E6D0ADF8108004AB2846FFF7A0FD06280446CF
S3150800E6E00CD1F820FFF756FC059B80F020009A789D
S3150800E6F0C0F3401060F341029A70E1E778BBBAF1C3
S3150800E700000F0ED0DAF80030BDF810101B681F464F
S3150800E710A9EB0603ADF812305A460DF1120350461E
S3150800E720B847BDF81030F61A4345B6B2C8D2A0218C
S3150800E7300DE043F001038B70BDF80E20CDF800B054
S3150800E74043462846FFF760FC044640B98021BDF8D9
S3150800E7500E3018EE102A2846FFF722FD04462046FA
S3150800E76009B0BDEC028BBDE8F08F002EEEDADEE7CD
S3150800E770002CDCD0F3E700BF2091012030B589B02A
S3150800E78000240C9D0794CDE90535CDE90343012303
S3150800E790CDE90143062300938023FFF733FF09B031
S3150800E7A030BD30B589B000240D9D0794CDE90535F7
S3150800E7B0CDE90343022302939DF8303001930623E3
S3150800E7C000938023FFF71EFF09B030BD2DE9F04105
S3150800E7D098B008ADCDE900351C46092306460F4614
S3150800E7E09046FFF7DEFF98B91E9BCDE906534023F6
S3150800E7F00593BDF82230CDE903030223CDE9014391
S3150800E800062300934246802339463046FFF7FAFE30
S3150800E81018B0BDE8F08110B588B00024019305232F
S3150800E820CDE90644CDE90444CDE9024400932346E4
S3150800E830FFF7E8FE04464FF4967027F071FF20466E
S3150800E84008B010BD10B588B00024019309230093C1
S3150800E850CDE90644CDE90444CDE902442346FFF751
S3150800E860D1FE08B010BD30B585B01D460023039310
S3150800E870ADF80A300DF10A03009303AB0446FFF71F
S3150800E88084FE58B99DF824300193089B0093BDF87F
S3150800E8900A2003992B462046FFF7C0FC05B030BD79
S3150800E8A030B585B01D4600230393ADF80A300DF147
S3150800E8B00A03009303AB0446FFF767FE40B9089BBB
S3150800E8C00093BDF80A2003992B462046FFF79CFBC8
S3150800E8D005B030BD2DE9F04106460C4679B3C1EBCB
S3150800E8E0C10303444FEAC1081B7B5B061DD50723FA
S3150800E8F003FB010301271D7B05F007057B1E0E2B75
S3150800E90094BF3B460123C3EBC3023244DFB2127BFA
S3150800E910C2F3C202AA4214D00133DAB20F2AF2D9DC
S3150800E920F379AB4201D1013DF571A8EB04043444F7
S3150800E93000230122043623736273A373A660BDE81D
S3150800E940F08139463046FFF7C5FFD7E7412910B5AC
S3150800E950044602D1FFF75BFD10BDFFF789FD0146AE
S3150800E9602046FFF7B7FFF7E770B51C4683680546EC
S3150800E970D3B1134684730022FFF789FD0646A8B172
S3150800E98001462846FFF7CBFD90B100228471334635
S3150800E99011462846FFF73FFF044618B13146284678
S3150800E9A0FFF7D4FF204670BDD724FBE7D424F9E748
S3150800E9B0D624F7E72DE9F04F2DED048B89B01E46D6
S3150800E9C008238DF809303C238DF80A3002AB846899
S3150800E9D08360924603AB00228673894600931146EC
S3150800E9E0122305468DF80820FFF7C8FEAC600446DA
S3150800E9F000284DD1BDF8143008EE103ABDF816308F
S3150800EA0008EE903A9DF8103009EE103A9DF811304C
S3150800EA1005F1780709EE903ABB4680465BF8040B89
S3150800EA20A8B908F101085FFA88F8B8F1100FF5D10E
S3150800EA3057F8040B00283AD10134E4B2102CF7D168
S3150800EA403346524649462846FFF78EFF20E00368BC
S3150800EA501B6998470028E4D15BF8040C036819EE93
S3150800EA60901A1B6A98470028DBD05BF8040C0368E9
S3150800EA7018EE902A9B6918EE101A984768B1009606
S3150800EA8053464A4641462846FFF766FCD128C8D071
S3150800EA9009B0BDEC048BBDE8F08F5BF8040C036885
S3150800EAA019EE101ADB6998470028E8D1B9E7036818
S3150800EAB01B6998470028BFD157F8040C036819EE5C
S3150800EAC0901A1B6A984758B9534600964A462146F3
S3150800EAD02846FFF741FC00F0F703D12BD8D1ABE766
S3150800EAE057F8040C036818EE902A9B6918EE101A5A
S3150800EAF098470028A0D157F8040C036819EE101A95
S3150800EB00DB6998470028DFD096E700002DE9F04139
S3150800EB104FF4005105466848684E28F0DFFCA0B956
S3150800EB20C820FFF737FA10F020010BD0F820FFF7BE
S3150800EB3031FA00F0C004802C12D00DD83CB3402C1A
S3150800EB401AD02021C820FFF747FA3378032B27D895
S3150800EB50DFE803F028235931C02CF2D1012309E05C
S3150800EB60D820FFF717FA80070BD4C921D820FFF75A
S3150800EB7033FA02233370E4E7D820FFF70BFA81074C
S3150800EB80F3D4CB21D820FFF727FA0323F2E7D121C4
S3150800EB90D820FFF721FA3470D3E7494B13221A70AD
S3150800EBA0002616E0464A137803F0F003102BF7D038
S3150800EBB011231370F4E70126414C237803F0F00380
S3150800EBC0102B06D127F0A6FD3E4BC830186020232F
S3150800EBD0237005F1780705F1B8083C4654F8040B8C
S3150800EBE010B10368DB6898474445F7D1344C22785E
S3150800EBF0402A3AD009D8202A28D0302A2FD0112ADC
S3150800EC0016D0BDE8F0810026D6E7512A3DD0802AE5
S3150800EC1044D0502AF5D1C820FFF7BCF94306F0D5F1
S3150800EC205123237027F076FD264B14301860E8E749
S3150800EC30002385F8B83057F8040B10B103689B68B1
S3150800EC4098474745F7D112232370DAE727F062FD84
S3150800EC501C4B1B68C01A0028D3DB30232370012104
S3150800EC60E820FFF7B9F94023EEE7E820FFF792F925
S3150800EC70C207C6D4D820FFF78DF940F00800C1B204
S3150800EC80D820FFF7A9F95023DEE727F043FD0D4BFF
S3150800EC901B68C01A0028B4DB802323700022334681
S3150800ECA011462846FFF786FE18B1D228A9D0A02318
S3150800ECB0CAE79023C8E700BF00080240B411002045
S3150800ECC0B5110020B8110020036830B59BB104794E
S3150800ECD09CB113887BB10B681D7843791B1B0468AC
S3150800ECE0E5540379013B03711388013B13800B68D4
S3150800ECF001330B60EBE7002030BD43790371012037
S3150800ED00FAE7000007B508461946431EADF806207F
S3150800ED10072B1ED8DFE803F004162329353F3F44A6
S3150800ED2000221021234828F0DFFB022027F0F8FCF8
S3150800ED3020480122102128F0D7FB01221E484FF453
S3150800ED40004104E0BDF806203AB91A48202128F007
S3150800ED50CBFB012003B05DF804FB0122F5E7BDF803
S3150800ED600630002BE9D00022E8E7BDF8062032B9C4
S3150800ED701021104828F0B8FB29F0E8FDE9E7012240
S3150800ED80F6E74FF47A7301220DF106010B48006885
S3150800ED902BF0A8F8DDE7BDF806204FF47A73F5E7FF
S3150800EDA0064BBDF8062018682BF0E2FA012027F07A
S3150800EDB0B7FCCEE70004024000000240BC11002068
S3150800EDC027F0AEBC08B5094B012218604FF4004184
S3150800EDD0074828F089FB0A2027F0A2FCBDE808406E
S3150800EDE0044A0549054800F067BC00BFBC1100206D
S3150800EDF00000024005ED000800000020C0110020B8
S3150800EE002DE9F04F89B00746BDF848600096DDF851
S3150800EE104C90884614461D4600F055F8A8B1EB1DDF
S3150800EE20C3F3CC03264404934FEAD50AB3B2059339
S3150800EE30CAEB4A3305EBC3039BB2039325F00703DA
S3150800EE4043440693059B9C4202D109B0BDE8F08F66
S3150800EE5008F1070189B2CB462E46072E1CD8039B1C
S3150800EE60ABB119F80AB0BDF818101E461BF0010F11
S3150800EE7005D022463846079100F067FC0799013EFF
S3150800EE800131B6B289B24FEA5B0B002EEED1049B74
S3150800EE9001349944A4B2D5E71BF8013B00932246F6
S3150800EEA002233846079100F055FC0799083E0831B9
S3150800EEB0B6B289B2D1E710B4BDF8044001945DF842
S3150800EEC0044BFFF79DBF70B50546BDF81040B5F871
S3150800EED04260C08F013C14449642A4B212D3A042A9
S3150800EEE001D9A24210D9B5F84000AA8F013B0B44BC
S3150800EEF088429BB20AD39A420BD9994294BF002002
S3150800EF00012070BDA042ECD90020FAE79A42F4D954
S3150800EF10FAE70120F5E710B48C680023A44601211E
S3150800EF205DF8044B604710B48C680023A44603219F
S3150800EF305DF8044B604710B48C680023A4461A4653
S3150800EF405DF8044B0421604710B48C680023A4467E
S3150800EF5001225DF8044B0421604710B48C68002335
S3150800EF60A44602215DF8044B604710B48C68002360
S3150800EF70A44605215DF8044B6047F8B505460E46DC
S3150800EF80571E002017F8014F50B9FF2C38D02246DB
S3150800EF9031462846FFF7E9FF0028F2D10020F8BDE0
S3150800EFA0FF2CF4D0FE2CFAD0EF2CEAD8DF2C06D9A9
S3150800EFB004F00F0231462846FFF7CFFFE1E7CF2CD2
S3150800EFC006D904F00F0231462846FFF7ACFFD8E70A
S3150800EFD0BF2C12D9240102343146284604F0FE0417
S3150800EFE0FFF7A9FF2046FFF7EBFE31462846FFF755
S3150800EFF0ABFF2046FFF7E4FEC3E72306C1D4F8E7D4
S3150800F0000120BFE7F8B5DFF844C00F4F002413F816
S3150800F010015B05F00F0E661C2D091CF80EE007F8BB
S3150800F02004E0B6B2013A1CF80550BD55023492B256
S3150800F030A4B2002AEBD18C68034B4FF480620821F6
S3150800F040A0470120F8BD00BF84120020085A040812
S3150800F050F8B5DFF840C00E4F002413F8015B05F041
S3150800F0600F0E661C2D091CF80EE007F804E0F6B230
S3150800F070013A1CF80550BD55023412F0FF02E4B2FD
S3150800F080EBD18C68024B80220621A0470120F8BDEF
S3150800F09004120020085A040801207047F8B54B6886
S3150800F0A01D881F7A07FB052206460C4602F0FF0557
S3150800F0B00F4AFFF762FF2A4621463046FFF755FFFB
S3150800F0C06A1C2146D2B23046FFF74FFF214630462A
S3150800F0D00022FFF742FF21465C223046FFF745FF34
S3150800F0E0214630460122BDE8F840FFF736BF00BF8B
S3150800F0F0965A04082DE9F74F9946A2F10A030446E1
S3150800F10090460C2B22D8DFE803F007212121217F26
S3150800F1109FA7212121123B0002220191FFF7FBFE46
S3150800F1204E4A01992046FFF728FF01990EE04E68DE
S3150800F1307589D6F80CB04FEA950A0027C5F38705F6
S3150800F1403388FAB2934207F1010707D84B4642467D
S3150800F150204603B0BDE8F04F00F0FBBB2046019106
S3150800F160FFF79CFF5B4601992A462046FFF770FF8A
S3150800F170019900222046FFF7D6FED3440199DFE71E
S3150800F180D1F804A0BAF80A70DAF80CB07F00BFB25A
S3150800F1900026BAF80020B242D8D948680191027A06
S3150800F1A0058802FB056505F0FF052D4A2046FFF791
S3150800F1B0E4FE01992A462046FFF7D7FE05F1080224
S3150800F1C00199D2B22046FFF7D0FE019900222046C7
S3150800F1D0FFF7C3FE01995C222046FFF7C6FE019998
S3150800F1E001222046FFF7B9FE5B4601993A462046BA
S3150800F1F0FFF708FF0836019900222046FFF793FE1D
S3150800F200BB440199F6B2C4E701220191FFF78BFED0
S3150800F210019920460022FFF7A0FE0199C122204647
S3150800F220FFF7A3FE019920460122FFF796FE99F8FB
S3150800F2300020019952082046FFF797FE01990022FF
S3150800F2402046FFF770FE70E7064A2046FFF795FE50
S3150800F250012003B0BDE8F08F034AF6E7185A040800
S3150800F260965A0408B15A0408A65A04084218435C78
S3150800F270507800EB032080B270470020704790F961
S3150800F2802900013080B27047704708B5FFF7FCFFC8
S3150800F29010F0FD0F14BF0320062008BD0621FFF756
S3150800F2A0E5BF0821FFF7E2BF807A7047C07A70474A
S3150800F2B02DE9F84F8468237805461846FFF7E4FFDA
S3150800F2C080461846FFF7E1FFB8F1010F8146204650
S3150800F2D014BF4FF0FF0A4FF00F0AFFF7E7FF0F467C
S3150800F2E083462046FFF7DDFF602F0AD948B1204440
S3150800F2F06126BB4515D20020E86185F82000BDE8E7
S3150800F300F88F2046FFF7D0FF06462046FFF7C6FFD0
S3150800F310402F03D910B120444126EAE704F1110031
S3150800F320E7E75E45E7D80278FF2A05D101305E4552
S3150800F330E1D00136F6B2F6E7BE421ED118F0FD0F4F
S3150800F3400AD1EA77427885F82020C2782A770279A6
S3150800F3506A774279AA77D2E702F00F0102391209D1
S3150800F360A9776A77427802F00F01120985F820100A
S3150800F370EA77827812092A77C1E782780AEA0202CE
S3150800F3804A441044D3E72DE9F04F0F4687B0194693
S3150800F39005469046FFF78CFF0446D8B1AB6895F949
S3150800F3A01E2093F8009095F8203095F91D100393C8
S3150800F3B01A440F44A8EB0208BFB21FFA88F8009354
S3150800F3C04246EB7FEE7F39462846FFF77CFD20B99B
S3150800F3D095F91C0007B0BDE8F08F48460736FFF7D9
S3150800F3E054FFC6F3C40B06F0F8063E440444B6B20E
S3150800F3F04FF0000903995FFA89F308EB090299426D
S3150800F40092B2E5D93946A2460CE01AF8013B0093B8
S3150800F41028460023CDE9041200F09CF90499059AC0
S3150800F420083189B2B142F0D15C4409F10109E1E73A
S3150800F4302DE9F0411D46436A174680460C46984713
S3150800F440384487B2013D002615F8013F13B9304606
S3150800F450BDE8F08121463A464046FFF794FF14FA84
S3150800F46080F416FA80F6A4B2B6B2EDE78368BBB1AB
S3150800F47090F82820AAB95A7980F829201B7B80F8A9
S3150800F4802A3090F92A2090F929309B1A90F82B20D7
S3150800F4909BB2402A1EBFDBB253439B0980F82C302F
S3150800F4A07047012A0BBFDA7B5A7B80F8292080F83F
S3150800F4B029200CBF1B7C9B7BE1E7002280F82820D3
S3150800F4C0FFF7D4BF012380F82830FFF7CFBF00002D
S3150800F4D0014B4362704700BF7BF20008014B436251
S3150800F4E0704700BF7FF2000870B505464E1E00241F
S3150800F4F016F8011F39B12846FFF7DAFE95F91C30D0
S3150800F5001C44A4B2F4E7204670BD000083688B4211
S3150800F51010B504D08160FFF7A9FF014B436210BD07
S3150800F5207BF2000810B40C68A4465DF8044B6047EB
S3150800F53037B5836B019104460220984701990A2240
S3150800F54000232046FFF7EEFFA36B054603209847E6
S3150800F550A36B00209847284603B030BD13B5044670
S3150800F560836B019102209847A36B01209847019964
S3150800F570002314222046FFF7D5FF04F13C03019926
S3150800F58017222046FFF7CEFFA36B002002B0BDE886
S3150800F5901040184737B50446836B019102209847F7
S3150800F5A0A36B012098470199002315222046FFF7EF
S3150800F5B0B9FF0199054628B104F13C0317222046F4
S3150800F5C0FFF7B0FFA36B00209847284603B030BD6D
S3150800F5D037B50446836B019102209847A36B012037
S3150800F5E098470199002316222046FFF79BFF0199A9
S3150800F5F0054628B104F13C0317222046FFF792FF7F
S3150800F600A36B00209847284603B030BD07B58DF890
S3150800F61007200DF107030F22FFF784FF03B05DF8FB
S3150800F62004FB10B45DF8044BC2850386322200F150
S3150800F6302E03FFF777BF07B546220DF10603FFF73E
S3150800F64071FFBDF8060003B05DF804FB07B5472255
S3150800F6500DF10603FFF766FFBDF8060003B05DF877
S3150800F66004FB08B548220023FFF75CFF80B208BDFB
S3150800F67010B541680446FFF7DEFF61682080204622
S3150800F680FFF7E4FF616860802046FFF7EAFF6168DC
S3150800F690E07404F13C0320461722BDE81040FFF74A
S3150800F6A041BF10B541680446FFF742FF18B120462E
S3150800F6B0FFF7DEFF012010BDF8B500260123174627
S3150800F6C022220446C0E902660382866180F8343045
S3150800F6D082740D46FFF7FCFE064BA362064B84F8C0
S3150800F6E02C60A36365602046AF60BDE8F840FFF76D
S3150800F6F0D8BF00BF01000040BDFC00084168FFF705
S3150800F7002DBF836910B5044603B198476168204642
S3150800F710BDE81040FFF73EBF836910B5044603B144
S3150800F720984761682046BDE81040FFF751BF0A4672
S3150800F7304168FFF76BBF416800231022FFF7F2BE4E
S3150800F740416800231122FFF7EDBE13460A464168B9
S3150800F750FFF767BF30B49DF8085080F8333080F85B
S3150800F7603250C185028630BC416800F12E033B2227
S3150800F770FFF7D8BE80F834107047C37C282B04D016
S3150800F780022B14BF012003207047FF20704708B5DD
S3150800F790C37C302B024603D14FF6FF73838608BD20
S3150800F7A0FFF7EBFF82F83400F9E703880022013BF4
S3150800F7B08280C380027270478288038841881A440F
S3150800F7C092B28A4282800DD2027A01320272C288CD
S3150800F7D013449BB299429CBF01F1FF339BB2C3808D
S3150800F7E00120704700207047C38810B58B4234BF8C
S3150800F7F000230123914294BF00210121848843EA12
S3150800F800010094428CBF002000F001001940084313
S3150800F81010BD00230B8083884B804389013B8B8076
S3150800F820C388CB8070470B4649885B79012B04D087
S3150800F830032B06D00A46FFF7D7BF01F1080292B29A
S3150800F840F9E7A1F108030A4699B2F4E770B54589C4
S3150800F850C46880889DF81060121AAD08D2B288086C
S3150800F86012FB05F2490010FA82F201F0060136B9D8
S3150800F8700320A55C8840C0B225EA0000A05403F026
S3150800F880030303FA01F1A35C1943A15470BD42892D
S3150800F890C0685200002130F0B9BF37B585881446D4
S3150800F8A04A8895420BD8C588954208D30D8843895E
S3150800F8B0AB4204D900948B792946FFF7C7FF03B0FA
S3150800F8C030BD70B50D7906460C462B0604D50022C8
S3150800F8D021463046FFF7E1FF6379032B06D8DFE8B8
S3150800F8E003F0020A0E112388013323806D0015F0F8
S3150800F8F0FF05EAD170BD638801336380F6E7238884
S3150800F900013BF2E76388013BF7E770B50D790646D8
S3150800F9100C46AB09A371012221463046FFF7BDFF0D
S3150800F9206379032B06D8DFE803F0020A0E11238851
S3150800F93001332380AD0015F0FF05EAD170BD638859
S3150800F94001336380F6E72388013BF2E76388013BCE
S3150800F950F7E713B508462D2A446819462FD00FD85D
S3150800F960172A09D8132A09D9153A2046022A2CD863
S3150800F970DFE802F0313137002C2A24D0012017E0C5
S3150800F980462A31D00ED8322A14D03B2AF6D1204640
S3150800F9900193FFF748FF01990028EFD02046FFF7AB
S3150800F9A090FFEBE7472A22D0482A14BF01200220FD
S3150800F9B002B010BD00222046FFF76FFFDEE72046A3
S3150800F9C0FFF7A3FFDAE70122F5E7FFF7EEFE204689
S3150800F9D0FFF75DFFD2E7FFF7EFFE0028F7D100201B
S3150800F9E0E6E7FFF716FFC9E763890B80C6E7638872
S3150800F9F0FBE72DE9FF410D461C461E46CF184FF082
S3150800FA00FF08B91B072E89B21AD8E308C3EB43339C
S3150800FA1024F0070104EBC3042944A4B289B264B1F3
S3150800FA2084F007040134FF2304F0070403FA04F4FE
S3150800FA30E4B200940023FFF78DFE04B0BDE8F08120
S3150800FA40CDF800800023083ECDE90202B6B2FFF7E2
S3150800FA5081FEDDE90202D4E72DE9FF4115461C4681
S3150800FA601E46D7184FF0FF08BA1B072E92B21AD8AF
S3150800FA70E308C3EB433324F0070204EBC3042A4428
S3150800FA80A4B292B264B184F007040134FF2304F0EF
S3150800FA90070403FA04F4E4B200940123FFF75AFEBC
S3150800FAA004B0BDE8F081CDF800800123083ECDE919
S3150800FAB00201B6B2FFF74EFEDDE90201D4E72DE9F1
S3150800FAC0F341BDF82070009705460E461446984641
S3150800FAD0FFF7F9F9F8B14346224631462846FFF7BB
S3150800FAE088FF3B46224631462846FFF7B5FF08F110
S3150800FAF0FF3131443B462246284689B2FFF7ACFF20
S3150800FB007A1E2244434692B23146284602B0BDE8E0
S3150800FB10F041FFF76EBF02B0BDE8F0812DE9F04174
S3150800FB20BDF81850154406460F4698461446ADB219
S3150800FB3022460134434639463046A4B2FFF759FFF8
S3150800FB40AC42F5D1BDE8F0812DE9F341BDF820803E
S3150800FB50CDF8008004460D4616461F46FFF7B3F952
S3150800FB6050B13B46324629462046CDF8208002B0A1
S3150800FB70BDE8F041FFF7D2BF02B0BDE8F081002032
S3150800FB807047322A2DE9F3414968054616461C4650
S3150800FB9060D00DD82C2A5DD02D2A0FD0172A24D054
S3150800FBA023463246284602B0BDE8F041FFF7BABC04
S3150800FBB0462A48D0472A4AD03B2AF1D128460191FD
S3150800FBC0FFF744FD67880199FF43384487B2284602
S3150800FBD0FFF731FD23886780DB431844637920806B
S3150800FBE0023303F00303637145E00191FFF79AFCC2
S3150800FBF001992846FFF71FFDB4F8048001996FEABA
S3150800FC00080840441FFA80F82846FFF714FD26889E
S3150800FC100199F643304486B22846FFF717FDE78870
S3150800FC200199FF43384487B22846FFF70FFD6388DA
S3150800FC30A4F80080DB4318446780A680E080012092
S3150800FC4002B0BDE8F081FFF7F6FC2080F7E7FFF782
S3150800FC50FDFCFAE728460191FFF7F8FC6788019949
S3150800FC60FF43384487B22846FFF7E5FC23886780B8
S3150800FC70DB43184420800199234632462846FFF77D
S3150800FC8051FCDCE7426804498A4203D15268426063
S3150800FC90FFF7EEBC704700BF1C0000204268054B0A
S3150800FCA09A4218BF5A60044A18BF43601A60FFF7A1
S3150800FCB0DFBC00BF1C00002083FB00087047000063
S3150800FCC0F8B5084E084F0223054633700A24012268
S3150800FCD0294638462EF0CCFC013C307001D000286D
S3150800FCE0F5D1F8BD841800208818002070B5084E94
S3150800FCF00223054633700A240122294600202EF0E5
S3150800FD00B7FC013C307001D00028F5D170BD00BFAA
S3150800FD1084180020024B312283F87820704700BFF0
S3150800FD20BC1A00202DE9F0411446DFF838800B4F45
S3150800FD3005460E46384638F81410002227F0D4FB3C
S3150800FD40B2B229460648C8232AF0CCF838F8141067
S3150800FD5038460122BDE8F04127F0C6BB000C024038
S3150800FD60D8910120CE080020042A01D8FFF7DABF6F
S3150800FD7070470000DFF844C001700E490022C0E950
S3150800FD800322C0E905C1C0E90722C0E909220A49D8
S3150800FD90427042804260C26240F6B832028641F240
S3150800FDA08832C0E90D120222C2630822A0F8402058
S3150800FDB0704700BF00943577801A0600006CCA8821
S3150800FDC037B504788DF802309DF818308DF8033071
S3150800FDD061F07F019DF81C308DF80010032C8DF81A
S3150800FDE001208DF8043013DC0A4D0B4835F8141041
S3150800FDF0002227F079FB0522694608484FF47A73F2
S3150800FE002AF070F835F814100348012227F06CFB25
S3150800FE1003B030BDCE080020000C0240D891012066
S3150800FE20F0B5224B224F234E234D87B0044618685F
S3150800FE301B7900908DF804306946C82305221F48AF
S3150800FE402AF050F821781E4B1E4833F8111001226B
S3150800FE5027F04AFB2378012237F81310304627F09B
S3150800FE6043FB0A2026F05CFC28682B79227802904E
S3150800FE70052102A88DF80C30FFF776FF0A2026F038
S3150800FE804FFCD5F805006B7A22780490052104A862
S3150800FE908DF81430FFF768FF2378002237F813101F
S3150800FEA0304627F021FB07B0F0BD00BF699A040869
S3150800FEB0D608002000080240484F0408D8910120BF
S3150800FEC0CE080020000C024010B5344B0478D3F855
S3150800FED01E0093F8222090B005210090D3F82D003B
S3150800FEE08DF80420029093F83120D3F832008DF86B
S3150800FEF00C20049093F83620D3F823008DF81420AC
S3150800FF00069093F82720D3F837008DF81C20089020
S3150800FF1093F83B20D86B8DF824200A9093F840205C
S3150800FF20D3F841008DF82C200C9093F84520D3F88F
S3150800FF3046008DF834200E90224693F84A308DF804
S3150800FF403C306846FFF710FF224668460521FFF752
S3150800FF500BFF224602A80521FFF706FF224604A842
S3150800FF600521FFF701FF224606A80521FFF7FCFE3B
S3150800FF70224608A80521FFF7F7FE22460AA805210A
S3150800FF80FFF7F2FE22460CA80521FFF7EDFE2246F2
S3150800FF9005210EA8FFF7E8FE10B010BD484F04086B
S3150800FFA000B5214B0278D3F80A00997B8DB00290F0
S3150800FFB0D3F80F008DF80C100490D97CD3F84B00B9
S3150800FFC08DF81410069093F84F10D3F819008DF891
S3150800FFD01C100890597F186D8DF8241093F854302A
S3150800FFE00A90052102A88DF82C300192FFF7BCFE75
S3150800FFF0019A02A80521FFF7B7FE019A04A8052170
S31508010000FFF7B2FE019A06A80521FFF7ADFE019A90
S3150801001008A80521FFF7A8FE019A05210AA8FFF7F6
S31508010020A3FE0DB05DF804FB484F040800B5154B57
S315080100300278D3F80A00997B89B00290D3F80500B3
S315080100408DF80C100490597A18688DF814101B79DC
S315080100500690052102A88DF81C300192FFF784FE4F
S31508010060019A02A80521FFF77FFE019A04A8052136
S31508010070FFF77AFE019A052106A8FFF775FE09B072
S315080100805DF804FB484F040807B5002201F3060191
S31508010090CBB2CDE900226D21FFF792FE03B05DF8E0
S315080100A004FB07B500230422CDE9002334211A46AF
S315080100B0FFF786FE03B05DF804FB000007EE901A11
S315080100C0DFED106AB8EEE77A13B5C6EE877AFCEE6D
S315080100D0E77A17EE901A0B0C14BF012300230A0EB8
S315080100E014BF012200220C1E18BF0124090A14BFDD
S315080100F001210021009101941421FFF761FE02B04C
S3150801010010BD00BF0000804B07B5CBB20193C1F308
S31508010110072300930A0EC1F307432D21FFF750FE6B
S3150801012003B05DF804FB000007B5094A8A42A8BF77
S315080101300A46D3B20193C2F3072300932721C2F3D8
S315080101400743120EFFF73CFE03B05DF804FB00BF40
S3150801015000FE7F0007B50129B8BF01214FF6FF73DD
S315080101609942A8BF1946CBB20193C1F307210023CF
S3150801017000911A462821FFF723FE03B05DF804FB18
S3150801018037B501290B464FF6FF72B8BF01239342D3
S31508010190A8BF1346DAB2C3F30723009300230C461C
S315080101A0019226211A460546FFF70AFE21462846E8
S315080101B003B0BDE83040FFF7CDBFF0B5042385B0E5
S315080101C000250C46CDE900532A462B462021064632
S315080101D0C4F30727FFF7F4FD220EC4F30743E4B27D
S315080101E03046CDE900742121CDE90223FFF7E8FD68
S315080101F0DDE902233046CDE900742D21FFF7E0FD44
S31508010200CDE900552B462A4620213046FFF7D8FD71
S3150801021005B0F0BD10B5374B0478D3F8550093F8FF
S31508010220592092B005210090D3F85A008DF8042080
S31508010230029093F85E20D3F85F008DF80C200490A5
S3150801024093F86320586E8DF81420069093F8682069
S31508010250D3F869008DF81C20089093F86D20D3F81F
S315080102606E008DF824200A9093F87220D3F8730053
S315080102708DF82C200C9093F87720986F0E908DF8B6
S31508010280342093F87C20D3F87D008DF83C2093F830
S3150801029081301090224668468DF84430FFF764FD98
S315080102A0224602A80521FFF75FFD224604A805217B
S315080102B0FFF75AFD224606A80521FFF755FD2246F6
S315080102C008A80521FFF750FD22460AA80521FFF7D0
S315080102D04BFD22460CA80521FFF746FD22460EA82E
S315080102E00521FFF741FD2246052110A8FFF73CFD30
S315080102F012B010BD484F040807B5CDE90012002217
S315080103001021FFF75DFD03B05DF804FB2DE9F04709
S3150801031001299DF820909DF824A09DF8288004467F
S315080103200D4617461E461ED1FFF73AFE2046FFF731
S3150801033071FF394620466763FFF7F6FE31462046C8
S315080103402686FFF71DFF84F8409084F841A04346AE
S31508010350524649462046FFF7CFFF84F8448084F881
S315080103604350BDE8F0870229E0D1FFF7ADFDDDE78F
S3150801037030B58DB00024244B01941A6B234842F002
S3150801038001021A631A6B02F001020192019A0294A0
S315080103905A6C42F480725A645B6C099403F4807354
S315080103A002930222029B07A90323CDE9072326F01C
S315080103B033FF2146102203A830F028FA14481549BC
S315080103C084604FF480330125C0E90013124B0461A0
S315080103D0047680F82040C4628362C460C56180F8EF
S315080103E03040456126F0B0F908B124F038FB002306
S315080103F00748059303A9CDE9035526F025FB08B15E
S3150801040024F02DFB0DB030BD00380240000002403B
S31508010410381B0020002001400100000F10B50446DA
S3150801042088B01422002103A830F0F0F92268124B93
S315080104309A421ED103F58C33002101915A6C0F485B
S3150801044042F480725A645A6C02F480720192019ADB
S3150801045002911A6B42F001021A631B6B03F0010346
S315080104600293029B0622032303A9CDE9032326F05F
S31508010470D3FE08B010BD00BF0020014000000240B5
S315080104800A480B4A08B51023C0E9002300238361F3
S315080104908383C0E90233C0E9043326F071FB18B13E
S315080104A0BDE8084024F0DBBA08BD00BF801B002068
S315080104B00064004010B5044688B01422002103A840
S315080104C030F0A4F92268134B9A4221D103F5EA3395
S315080104D0002101911A6C104842F000721A641A6CD4
S315080104E002F000720192019A02911A6B42F0080217
S315080104F01A631B6B03F008030293029B0222032370
S31508010500CDE90332069303A90923079326F084FE4E
S3150801051008B010BD00640040000C024013B5104835
S31508010520104B03600024CDE9004426F02FFC08B1E6
S3150801053024F095FA3C230A4800226946CDE900349D
S3150801054026F037FC08B124F08AFA054810226946D4
S3150801055026F02FFC08B124F082FA02B010BD00BFC4
S31508010560A81B00200074004010B5044688B0142268
S31508010570002103A830F04AF92268124B9A421ED18B
S3150801058003F5E233002101911A6C0F4842F000523B
S315080105901A641A6C02F000520192019A02911A6BBE
S315080105A042F001021A631B6B03F001030293029BDB
S315080105B03022032303A9CDE9032326F02DFE08B033
S315080105C010BD00BF007400400000024007B5284B6B
S315080105D000220092196B41F480011963196B01F429
S315080105E08001009100990192196B41F40011196378
S315080105F01B6B03F40013019309211020019B26F0BC
S315080106004DFB102026F07CFB00220A21112026F042
S3150801061045FB112026F074FB002211462F2026F0F7
S315080106203DFB2F2026F06CFB002205213A2026F0FF
S3150801063035FB3A2026F064FB002203213B2026F0F5
S315080106402DFB3B2026F05CFB00220421452026F0E9
S3150801065025FB452026F054FB00220621462026F0DC
S315080106601DFB462003B05DF804EB26F049BB00BF2D
S31508010670003802402DE9F0478CB01422002107A862
S3150801068030F0C4F800245F4B01941A6B5E4FDFF813
S3150801069080A15E4EDFF87C81DFF87C9142F0100282
S315080106A01A631A6B02F010020192019A02941A6BEC
S315080106B042F004021A631A6B02F004020292029AC9
S315080106C003941A6B42F080021A631A6B02F08002D5
S315080106D00392039A04941A6B42F001021A631A6B85
S315080106E002F001020492049A05941A6B42F002027E
S315080106F01A631A6B02F002020592059A06941A6B9E
S3150801070042F008021A631B6B03F008030693384686
S3150801071001221021069B26F0E7FE2246504642F2A8
S31508010720D32126F0E1FE224630464FF6107126F017
S31508010730DBFE224640464FF4004126F0D5FE304600
S315080107400122802126F0D0FE224648464FF44C71FC
S3150801075026F0CAFE22463846032126F0C5FE0125A3
S31508010760132307A93846CDE90735CDE9094426F00B
S3150801077053FD42F2D32307A95046CDE90735CDE902
S31508010780094426F049FD4FF6807307A93846CDE995
S315080107900734099526F040FD4FF6907307A93046B0
S315080107A0CDE90735CDE9094426F036FD4FF48072C7
S315080107B0022307A94046CDE90723CDE909440B944D
S315080107C026F02AFD4FF4004307A94046CDE907352F
S315080107D0CDE9094426F020FD082307A93046CDE9CD
S315080107E00734099426F018FD4FF44C7307A94846B7
S315080107F0CDE90735CDE9094426F00EFD0CB0BDE873
S31508010800F08700BF0038024000100240000C024089
S3150801081000080240000002400004024008B50B48E7
S315080108200B4A0C4BC0E9002300234FF48042C0E970
S315080108300233C0E90423C0E90633036227F042F80C
S3150801084018B1BDE8084024F00AB908BDBC1B002050
S3150801085000540040801A060030B5044689B01422B7
S31508010860002103A82FF0D2FF2268144B9A4223D104
S31508010870134C144800250195236B43F002032363A7
S31508010880236B03F002030193019BC0221223CDE9D6
S31508010890032301210323CDE90513042303A90793A0
S315080108A026F0BAFC0295236C43F400132364236CE7
S315080108B003F400130293029B09B030BD00540040B3
S315080108C00038024000040240BFF34F8F0549064B2A
S315080108D0CA6802F4E0621343CB60BFF34F8F00BFCF
S315080108E0FDE700BF00ED00E00400FA0570470000CF
S315080108F02DE9F0418A4B93F90030002B40F028810D
S31508010900DFF848C2874E9CF80010874D8748884C07
S31508010910002900F0CD80012916D1864FB6F90010BD
S315080109203F78B5F9002003680B3F082F0CD8DFE89C
S3150801093007F00544AB6F970B5A0B820000238CF81E
S3150801094000307D4B01221A70B6F90030052BDCBF49
S31508010950062333800368132B00F3D780142303601F
S31508010960B6F90030B5F900200068D91E9142DCBFFE
S31508010970043B2B80B5F90030012BDCBF02232B8009
S315080109802368002BDCBF01232360F7F7FBFD62A375
S31508010990D3E90023F7F760FE06460F462068F7F706
S315080109A0F1FD32463B46F8F7E7F820B130463946BD
S315080109B0F8F702F92060BDE8F081604F97F90070F9
S315080109C03FB901313180032F2368BAD1023323603D
S315080109D0B7E7012F04D0022FF5D101330360B0E741
S315080109E001322A80ADE7554F97F9007027B9544B64
S315080109F01B7819443180A4E7012F05D0022FA0D115
S31508010A004F4A12781344E9E74D4B1B781A44E8E735
S31508010A104A4F97F9007037B901393180032F236896
S31508010A208FD1023BD3E7012F03D0022FF6D1013B29
S31508010A30D4E7013AD5E7414F97F900701FB9404B02
S31508010A401B78C91AD6E7012F06D0022F7FF479AF92
S31508010A503B4A12789B1AC1E7394B1B78D21AC0E771
S31508010A60364F97F900703FB914313180032F236847
S31508010A707FF467AF1433AAE7012F03D0022FF5D10C
S31508010A801433ABE71432ACE72C4F97F900703FB932
S31508010A9014393180032F23687FF453AF143B96E74B
S31508010AA0012F03D0022FF5D1143B97E7143A98E7A3
S31508010AB0204A13780C2B19D00E2B08D00B2B7FF458
S31508010AC043AF1D4A01238CF8003013703CE71B4FD6
S31508010AD03B7801335BB2032BC3BF04233B70194B2D
S31508010AE03B70C2BF1970292313702AE7134B93F978
S31508010AF0001031B901211970134902270F702A21F3
S31508010B0011701A78013A1A701BE7B3F5616F7FF70E
S31508010B1027AF4FF4616322E7CDCCCCCCCCCCDC3FFC
S31508010B20A0080020520700209C0C0020E0080020A5
S31508010B30400A002069890120CC080020CD3C00200C
S31508010B408E030020CF3C0020CC3C0020681F0020EB
S31508010B50012B7FF430AFDFF8ECE2AF499EF80020B5
S31508010B60AE4EAF4FAF4C002A00F08A81012A21D13F
S31508010B70DFF8D4C20A689CF800C0B6F90050B7F984
S31508010B800000B4F90030ACF10B0CBCF1090F11D817
S31508010B90DFE81CF00A0072003201C1000F011000E3
S31508010BA092006C01DF00280100238EF800309E4B6D
S31508010BB001221A700B680E2BDCBF0F230B609B4BAF
S31508010BC0D3ED007AB2EE067A67EE877A91ED007A6E
S31508010BD0B8EEC77AB4EEE77AF1EE10FA48BFFDEE41
S31508010BE0E77A9FED937A48BFC1ED007AD1ED007A95
S31508010BF0F8EEE77AF4EEC77AF1EE10FAC4BF8D4B38
S31508010C000B600B68B3F5167F07DB0A2093FBF0F23E
S31508010C1000FB12320AB19B1A0B60B6F90030002BA1
S31508010C2080F2598100233380B7F90030002B80F216
S31508010C30578100233B8008687F4DF7F7A3FC74A30F
S31508010C40D3E90023F7F708FD06460F462868F7F7A4
S31508010C5099FC32463B46F7F771FF20B130463946D3
S31508010C60F7F7AAFF2860B4F9003040F2E24293424E
S31508010C7040F33B8122809EE6DFF8C4C19CF900C09F
S31508010C80BCF1000F06D1B2F5167FACBF0A320132AC
S31508010C900A608CE7BCF1010F08D0BCF1020F08D03D
S31508010CA0BCF1030F83D10133238080E705353580F5
S31508010CB07DE7053038807AE7DFF884C19CF900C002
S31508010CC0BCF1000F11D15D4B44F24F6082421B7893
S31508010CD004DD282010FB03230B6068E7B2F5167FB5
S31508010CE001DB0A20F6E71344F6E7BCF1010F0AD047
S31508010CF0BCF1020F0BD0BCF1030F7FF458AFB3F56B
S31508010D007A7FD0D153E74D4B1B781D44CFE74B4B28
S31508010D101B781844CEE7DFF828C19CF900C0BCF15E
S31508010D20000F06D1B2F5167FACBF053A02F1FF32C4
S31508010D30AEE7BCF1010F08D0BCF1020F07D0BCF138
S31508010D40030F7FF434AF013BAEE7053DAFE7053846
S31508010D50B0E7DFF8ECC09CF900C0BCF1000F12D176
S31508010D60364B44F24F6082421B7804DD6FF0270050
S31508010D7000FB0323B0E7B2F5167F02DB6FF009002B
S31508010D80F6E7D31AA8E7BCF1010F0AD0BCF1020FA6
S31508010D900BD0BCF1030F7FF40AAFB3F57A7FD2D13A
S31508010DA005E7264B1B78ED1A81E7244B1B78C01AF9
S31508010DB080E7DFF88CC09CF900C0BCF1000F01D1B7
S31508010DC0143265E7BCF1010F08D0BCF1020F07D058
S31508010DD0BCF1030F7FF4EBAE323365E70A3566E7FC
S31508010DE00A3067E7164A92F90020032A7FF4DFAE34
S31508010DF0B3F57A7FF0D1DAE6DFF844C09CF900C092
S31508010E00BCF1000F22D1143A42E700BFAFF30080CC
S31508010E10BA490C022B87863FDC0D0020548F01202E
S31508010E20528F01207C090020CC0800203441002083
S31508010E3000BA5B49A0BB0D00E40D00208E0300201B
S31508010E40CE3C0020681F002069890120BCF1010FF2
S31508010E5008D0BCF1020F07D0BCF1030F7FF4A7AE8F
S31508010E60323B21E70A3D22E70A3823E7224A92F96B
S31508010E700020032A7FF49BAEB3F57A7FF0D196E67C
S31508010E801E4805780C2D18D00E2D07D00B2D7FF492
S31508010E9091AE1B4A8EF8003013708BE6164D2B78EF
S31508010EA001335BB2032BC3BF04232B70154B2B7085
S31508010EB0C2BF1A702923037079E60F4A92F90050C6
S31508010EC02DB91370104B02251D702A230370137850
S31508010ED0013B13706BE6C82B7FF7A6AEC823A2E6C3
S31508010EE0C82B7FF7A8AEC823A4E6092B3FF763AD45
S31508010EF00A2323805FE500BFCE3C002069890120D3
S31508010F00CC080020D03C0020CC3C0020024B1A889B
S31508010F1002B91880704700BFDC2C00209FED097AC2
S31508010F200949C7EE007A0A68B7EE007A77EEC77AFA
S31508010F30FCEEE77AC2ED0B7AD36AC1ED037A013B7F
S31508010F405362704750A9AB4C8C92012008B5F9F74A
S31508010F505DFF00F0FD03012B03D0042818BF002014
S31508010F6008BD0320FCE7FFF7F1BF0000F8B52149EA
S31508010F702148224C224D234F234EFEF7C7FA1E481D
S31508010F80FEF79BFA1C48FEF7A9FA1B480321FEF750
S31508010F90F1FB1E4B18481B6B00221146FEF748FA57
S31508010FA094F900201A491B4830F0F6F994F9002003
S31508010FB019491A4830F0F0F900243B7855F8040B22
S31508010FC0ABB196F90030A34211D00121F9F727F9FF
S31508010FD055F8040C96F900200368A2420CBF0121BA
S31508010FE000211B6901349847032CE6D1F8BD00217D
S31508010FF0ECE700BF04620408C0110020900D002030
S315080110002C000020681F0020D83C00206C08002016
S31508011010E1A7040865040020F3A704085304002087
S315080110202DE9F04F60496148614E624D91B0FEF776
S315080110306DFA5E48FEF741FA5C48FEF74FFA5B48DF
S3150801104090F82A3090F829400321E41AFEF792FB1A
S31508011050594B56489B6A00221146FEF7E9F996F95B
S315080110600030E4B2002B6FD1296803A830F004FAE6
S31508011070A4B203AB4D4822466921FEF7D9F996F980
S315080110800130002B6AD1296803A830F0F5F9670009
S3150801109003AB46483A466921FEF7CAF996F9023082
S315080110A0002B65D1296803A830F0E6F903AB3F4860
S315080110B0E2196921FEF7BCF996F90330002B61D1D3
S315080110C0296803A830F0D8F93848DFF8FC90374E7C
S315080110D0DFF8F8A0DFF8F8B003ABA2006921FEF744
S315080110E0A7F925464FF0000859F8041B3046FEF7C4
S315080110F0FBF9C0F1640087B203213046FEF73AFBDB
S315080111009AF9003043450ED19BF80010002943D0C7
S315080111100021304600943C232A46FEF715FD00219E
S315080111203046FEF727FB2A4659F8043C394630462D
S3150801113008F10108FEF77CF92544B8F1040FADB2B0
S31508011140D2D111B0BDE8F08F1C4A55F8233092F977
S3150801115000201B4903A830F01FF989E7174A55F8FB
S31508011160233092F90020164903A830F015F98EE7C5
S31508011170124A55F8233092F90020114903A830F094
S315080111800BF993E70D4A55F8233092F900200C49DB
S3150801119003A830F001F997E70A4B2A461B6830463F
S315080111A0FEF746F9BFE700BF04620408C011002034
S315080111B002040020A40800206C080020900D0020DD
S315080111C05DC004086C0C0020040C0020D53C0020EE
S315080111D0681F00202DE9F04F2DED028BDFF8A8934B
S315080111E099F9006095B0002E00F0028199F9003056
S315080111F0012B40F0F880D24ED249DFF89093DFF800
S3150801120090A33046FEF782F93046FEF756F9304686
S31508011210FEF764F996F82A3096F8297003213046C4
S31508011220FF1AFEF7A7FAC84B002211469B683046FB
S31508011230FEF7FEF8C54BC649B3F90040D9F80030A8
S3150801124002930A25BAF9003094FBF5F2FFB203932B
S3150801125005FB12434FEA470B1BB207A830F09CF86F
S3150801126007AB5A466E213046FEF7E2F8BAF9003066
S3150801127093FBF5F205FB12331FFA87F8B449DFF839
S3150801128014A3B44F1BB207A830F086F807AB08EBD6
S315080112900B026E213046FEF7CBF89AED007AAE4B7B
S315080112A0B7EE008AC8EE077AB3F9001091FBF5F29A
S315080112B005FB12131BB212B20593049207EE101A1C
S315080112C0B8EEC77A01EB410167EE877A9FEDA37AFB
S315080112D0C900C7EE876A07EE901AF8EEE77AC7EDF6
S315080112E0006AC7EE877A17EE900AF7F75DF9DDE926
S315080112F00423CDE900019A4907A830F04DF86E217B
S3150801130007AB4FEA88023046FEF792F8D9F8001083
S31508011310B1F5167F80F2468191FBF5F407EE901A36
S31508011320F8EEE77AF2EE046A87EEA67A05FB14135D
S315080113300293DAED006AC8EE267A67EE277A97ED08
S31508011340007AC7EE877A17EE900AF7F72DF9029B0E
S31508011350CDE900012246834907A830F01DF807ABFD
S3150801136042466E217648804F754CDFF82C92DFF89D
S3150801137014A2FEF75DF873497148FEF7C7F870487D
S315080113800321FEF7F7F9C346002657F8041B204642
S31508011390FEF7AAF8C0F1690085B203212046FEF7D7
S315080113A0E9F999F900309E4210D19AF800100029FE
S315080113B000F0128100212046CDF8008069235A46A3
S315080113C0FEF7C2FB00212046FEF7D4F95A4657F824
S315080113D0043C294620460136FEF72AF8C344042E62
S315080113E01FFA8BFBD1D115B0BDEC028BBDE8F08F8E
S315080113F0534C5449DFF850A1DFF8A0812046FEF787
S3150801140085F82046FEF759F82046FEF767F894F85E
S315080114102A3094F8295003212046ED1AFEF7AAF935
S31508011420DAF80830324631462046FEF701F8B8F9AF
S31508011430003047490A27EDB293FBF7F207FB12334F
S31508011440ADB21BB207A82FF0A7FF07AB2A467D212D
S315080114502046FDF7EDFF454BB8F90010B3F900300A
S3150801146091FBF7F007FB101193FBF7F209B207FBA3
S315080114701233CDE900011BB23D49DFF824816F0023
S3150801148007A82FF089FF07AB3A467D212046FDF7CD
S31508011490CFFF384B38491A6807A82FF07DFF07ABED
S315080114A0EA197D212046FDF7C3FF344B32491A68F4
S315080114B007A82FF071FF07ABAA007D212046FDF78B
S315080114C0B7FF20492046FEF721F803212046FEF7FB
S315080114D051F9AB4658F8041B2046FEF705F8C0F14A
S315080114E0780087B203212046FEF744F9244B93F985
S315080114F00030B3420DD1234B1978C9B100212046DA
S31508011500009578235A46FEF71FFB00212046FEF771
S3150801151031F95A4658F8043C394620460136FDF752
S3150801152087FF05EB0B02042E1FFA82FBD2D15DE67B
S31508011530DAF800305A462046FDF77AFFE9E700BF98
S31508011540C0110020046204086C080020548F012091
S31508011550E3BB0408984600207C09002000007A4471
S3150801156021A8040835A80408180800209C0C0020A6
S3150801157005A80408E008002016A80408400A002067
S31508011580CD3C0020681F0020A0080020DC0D0020AB
S31508011590528F012078090020CE3C002052070020F6
S315080115A008080020029B1C44039B4FF416711C4437
S315080115B048F6A043B4FBF1F0B4FBF3F203FB124384
S315080115C001FB1044B3FBF1F3B4FBF5F506490095AD
S315080115D007A82FF0E1FEC2E6044B5A461B682046CF
S315080115E0FDF726FFF2E600BF4CB204086C0800209E
S315080115F02DE9F04F2DED028BB24EB349DFF814A356
S3150801160091B03046FDF782FF3046FDF756FF30466A
S31508011610FDF764FF96F8294096F82A309AF90050A2
S31508011620E41AE4B2002D00F09B809AF90030012BF0
S3150801163040F09180A348DFF8E092A44D0321FEF71C
S3150801164099F800221146D9F80C309E48FDF7F0FEAC
S315080116509F4B2D681B680A20642193FBF0F25943BE
S31508011660A4B200FB123391FBF5F103A80091994945
S315080116702FF092FE03AB224669219248FDF7D8FE68
S31508011680954B93F90020954B03A853F82210650052
S315080116902FF082FE03AB8B482A466921FDF7C8FE67
S315080116A08F4B93F90030022B40F0F4808D4903A843
S315080116B02FF0E2FE03AB834862196921FDF7B8FEF4
S315080116C0894B93F90030002B40F0EA80874B03A839
S315080116D019682FF061FE7B480121FEF74BF879481E
S315080116E0DFF83882774DDFF81CB203ABA200692117
S315080116F0FDF79EFEA246002758F8041B2846FDF76B
S31508011700F3FEC0F1640086B203212846FEF732F8DB
S31508011710774B93F900309F420FD19BF800100029AF
S3150801172000F0C88000212846009464235246FEF73B
S315080117300BFA00212846FEF71DF8524658F8043CD4
S31508011740314628460137FDF773FE04EB0A02042FDA
S315080117501FFA82FAD0D111B0BDEC028BBDE8F08F29
S31508011760DFF8B4B103213046FEF704F82A462946C4
S31508011770DBF80C303046FDF75BFE5E4B5E49B3F98C
S315080117800020A5B203A82FF007FE03AB2A4669215C
S315080117903046FDF74DFE594B5749B3F9002003A8CA
S315080117A06F002FF0F9FD03AB3A4669213046FDF784
S315080117B03FFE4B4B93F90030022B54D1494903A8FC
S315080117C02FF05AFE03AB3F48EA196921FDF730FEAF
S315080117D0454B93F90030002B4BD1444B03A81968AC
S315080117E02FF0DAFD37480121FDF7C4FF3548DFF848
S315080117F03091344E03ABAA006921FDF719FE2F4635
S315080118004FF0000859F8041B3046FDF76DFEC0F18C
S31508011810640083B20321304608EE103AFDF7AAFFA9
S31508011820374B93F9003043450DD1364B197851B3EF
S3150801183000213046009564233A46FEF785F90021D2
S315080118403046FDF797FF3A4659F8043C18EE101A48
S31508011850304608F10108FDF7EBFDEA19B8F1040F66
S3150801186097B2CFD1E1E628499A1E03A82FF094FD35
S31508011870A8E7264B93F90020254B03A853F8221015
S315080118802FF08AFDB2E7DBF800303A463046FDF71D
S31508011890CFFDD8E71C499A1E03A82FF07DFD09E75D
S315080118A01A4B93F900201A4B03A853F822102FF06C
S315080118B073FD14E7D9F8003052462846FDF7B8FDFE
S315080118C03BE700BFC011002004620408DC0D0020BC
S315080118D0E40D00205CA80408D43C0020540800202C
S315080118E0900D00204AA80408302D00203800002059
S315080118F0D03C0020DA3C00209BB90408DC3C0020DF
S31508011900CF3C0020681F00204FA80408D13C0020C6
S3150801191048080020A00800206C080020380800208C
S31508011920280800202DE9F04F7A4B7B4C93F90030BB
S315080119307A497B4E93B0032B05AD204600F3A2806E
S31508011940FDF7E4FD2046FDF7C9FD03212046FDF715
S3150801195011FF0522734BDFF80092DFF800A2F92187
S315080119602046FDF765FD70492046FDF7CFFD204667
S31508011970FDF7A3FD2046FDF7B1FD94F82A3094F84A
S31508011980297003212046FF1AFDF7F4FE726867499C
S3150801199028462FF001FD002211462B462046FDF769
S315080119A047FD634B93F90020624BFFB2BFB253F870
S315080119B0221028462FF060FD2B463A468A212046FA
S315080119C0FDF736FD5C4B5D491A784FEA470828460C
S315080119D02FF0E2FC42462B468A212046FDF728FDD8
S315080119E0574B56491A7828462FF0D6FC07EB0802BA
S315080119F02B468A212046FDF71BFD524B93F9002001
S31508011A00514B284653F822102FF036FD2B46BA00C3
S31508011A108A212046FDF70CFDBB464FF0000859F810
S31508011A20041B2046FDF760FDC0F1870085B203213E
S31508011A302046FDF79FFE374B93F9003043450FD1FA
S31508011A409AF80010002900F00F840021204600971B
S31508011A5087235A46FEF778F800212046FDF78AFEC5
S31508011A605A4659F8043C2946204608F10108FDF76B
S31508011A70DFFCBB44B8F1040F1FFA8BFBCFD113B0BF
S31508011A80BDE8F08F072B40F349830B2B40F3E58222
S31508011A900F2B40F3DF81132B40F34181172B5FDDB9
S31508011AA0FDF734FD2046FDF719FD03212046FDF714
S31508011AB061FE0522254BF3212046FDF7B9FC1A499B
S31508011AC02046FDF723FD2046FDF7F7FC2046FDF7E6
S31508011AD005FD94F82A3094F8297003212046FF1A47
S31508011AE0FDF748FE72681A4928462FF055FC002270
S31508011AF011462B462046FDF79BFC164BFFB219688B
S31508011B0028462FF0B9FC2B46BA0028212046FDF7B6
S31508011B108FFCB4E7E84D0020C01100206C6A040868
S31508011B206C0C002078A70408046204086DA8040850
S31508011B3077040020700B00201404002071A8040803
S31508011B4015040020D8520020300C0020BF9D04083F
S31508011B5077A80408D80D0020A40B0020681F0020D0
S31508011B60FDF7D4FC2046FDF7B9FC03212046FDF715
S31508011B7001FEA64B0522F3212046FDF759FC052255
S31508011B80A34BF9212046FDF753FCA2492046FDF750
S31508011B90BDFC2046FDF791FC2046FDF79FFC94F815
S31508011BA02A3094F82970B4F8009003212046FF1AC8
S31508011BB0FDF7E0FD7268984928462FF0EDFB0022F3
S31508011BC02B4611462046FDF733FC944B93F900202A
S31508011BD0934B284653F82210FFB22FF04DFC4FEADB
S31508011BE059082B46BFB28F4D3A4608F10A012046DD
S31508011BF0FDF71EFC296D2046FDF776FCA8EB0000D3
S31508011C001FFA80FA03212046FDF7B4FD864B93F9A6
S31508011C100030142B0FD1854B1978002900F0F68472
S31508011C2000212046009743463A46FDF78DFF0021DD
S31508011C302046FDF79FFD2B6D7D483A465146FDF737
S31508011C40F7FB696D7A48FDF74FFCA9EB000000EB3D
S31508011C50D070C0F34F0803217548FDF78BFD724B11
S31508011C6093F900307C00152B224610D16F4B197859
S31508011C70002900F0D2846E48009700214B46029451
S31508011C80FDF762FF6A480021FDF774FD029A6B6D44
S31508011C906748DFF8BCA1664D4146FDF7C9FB3C44E0
S31508011CA04FF0160B03212846FDF764FD5E4B93F9A9
S31508011CB000309B4540F0CC845C4BDAF8002093F861
S31508011CC00080B8F1000F00F0AF845A4905A82FF03B
S31508011CD063FB05A92846FDF707FC4B4680462246C5
S31508011CE0002128460097FDF72FFFA9EB08080021D8
S31508011CF02846FDF73FFD08EBD87805AB2246C8F321
S31508011D004F012846FDF794FB3C44BBF1170FA4B2DB
S31508011D100AF1040A3FF4B3AE4FF0170BC2E7FDF719
S31508011D20F5FB2046FDF7DAFB03212046FDF722FDE8
S31508011D30364B0522F3212046FDF77AFB0522344B63
S31508011D40F9212046FDF774FB32492046FDF7DEFBF3
S31508011D502046FDF7B2FB2046FDF7C0FB94F82A3072
S31508011D6094F829A00321AAEB030A204623880293A3
S31508011D70FDF700FD7268304928462FF00DFB002259
S31508011D8011462B462046FDF753FB2C4B93F90020B1
S31508011D902B4B284653F822102FF06EFB029B4FEA75
S31508011DA0530B5FFA8AFAABF10F094FEA4A081FFA91
S31508011DB089F942462B4649462046FDF739FB214B10
S31508011DC093F90020204B1FFA8AF753F82210284668
S31508011DD02FF052FB07EB08022B4649462046FDF732
S31508011DE027FB104B2046196CFDF77EFB174BABF111
S31508011DF0140B1FFA8BFB1B78ABEB0000C2461FFACC
S31508011E0080F8002B40F0F4820321F2E2BF9D04081A
S31508011E1078A70408046204087BA80408704800200F
S31508011E20140C0020A40B0020E84D0020681F002098
S31508011E30C0110020F2A804087FA80408E18901203E
S31508011E403C0C0020302D00207C0B0020B4430020E0
S31508011E50FC0B0020FDF75AFB2046FDF73FFB03214B
S31508011E602046FDF787FC9F4BDFF8AC820522F3215C
S31508011E702046FDF7DDFA05229B4BF9212046FDF7A1
S31508011E80D7FA9A492046FDF741FB2046FDF715FB8F
S31508011E902046FDF723FB94F82A3094F82970B4F804
S31508011EA0009003212046FF1AFDF764FC72689049E9
S31508011EB028462FF071FA002211462B462046FDF7D7
S31508011EC0B7FA8C4B93F900208B4BFFB253F82210CB
S31508011ED04FEA590B2846BFB22FF0CEFA2B463A469F
S31508011EE00BF10A012046FDF7A3FAD8F8301020466F
S31508011EF0FDF7FAFAABEB00001FFA80FA0321204638
S31508011F00FDF738FC7D4B93F900300C2B0FD17C4B38
S31508011F101978002900F02B820021204600975B469C
S31508011F203A46FDF711FE00212046FDF723FCD8F8B5
S31508011F30303074483A465146FDF77AFAD8F83410E3
S31508011F407048FDF7D1FAA9EB000000EBD070C0F399
S31508011F504F0A03216B48FDF70DFC684B93F90030D6
S31508011F607C000D2B224610D1654B1978002900F00B
S31508011F7004826448009700214B460294FDF7E4FD6C
S31508011F8060480021FDF7F6FB029AD8F834305D481F
S31508011F905146FDF74DFAD8F838105A48FDF7A4FA14
S31508011FA0A9EB000000EBD070C0F34F0A0321554896
S31508011FB0FDF7E0FB514B93F900300E2B07EB0402BA
S31508011FC010D14F4B1978002900F0DD814D48009753
S31508011FD000214B460292FDF7B7FD4A480021FDF75D
S31508011FE0C9FB029AD8F8383046485146FDF720FA17
S31508011FF0D8F83C104348FDF777FAA9EB000000EB47
S31508012000D070C0F34F0401213E48FDF7B3FB3B4BAB
S3150801201093F900300F2B4FEA870240F0C281384B03
S315080120201978002900F0B581364802920321FDF797
S31508012030A1FB4B46029A334800970021FDF784FD20
S3150801204030480021FDF796FB2F4928462FF014FA50
S315080120502B46029A21462B4859E5FDF757FA2046A1
S31508012060FDF73CFA03212046FDF784FB1D4B0522AB
S31508012070F3212046FDF7DCF905221B4BF921204601
S31508012080FDF7D6F919492046FDF740FA2046FDF72E
S3150801209014FA2046FDF722FA94F82A3094F8298092
S315080120A0278803212046A8EB0308FDF763FB72681E
S315080120B0164928462FF070F900222B46114620466C
S315080120C0FDF7B6F9124B1A785FFA88F8002A00F07C
S315080120D0D88002EB82020F49C2EB021228462FF082
S315080120E05BF9D2E0BF9D040878A7040804620408D6
S315080120F083A804085E1D0020580B0020E84D002027
S31508012100681F0020C0110020A5A8040887A8040894
S31508012110FC8801209FA80408A40B0020FDF7F6F906
S315080121202046FDF7DBF903212046FDF723FB9E4BED
S31508012130DFF8AC92DFF8AC820522F3212046FDF7E1
S3150801214077F90522994BF9212046FDF771F9984946
S315080121502046FDF7DBF92046FDF7AFF92046FDF7E6
S31508012160BDF994F82A3094F8297003212046FF1AFC
S31508012170FDF700FB72688F4928462FF00DF90022FA
S3150801218011462B462046FDF753F999F90030FFB25F
S31508012190BFB258F8231028462FF06EF93A462B4657
S315080121A041212046FDF744F999F901304FEA470ADA
S315080121B058F8231028462FF05FF952462B4641213D
S315080121C02046FDF735F999F90230284658F82310C3
S315080121D02FF052F907EB0A022B4641212046FDF75B
S315080121E027F999F90330DFF8F4A158F82310DFF835
S315080121F0F89128462FF040F92B46BA00412120468E
S31508012200FDF716F9BB464FF0040859F8041B20469A
S31508012210FDF76AF9C0F13C0085B203212046FDF7B6
S31508012220A9FA654B93F9003043450DD19AF8001088
S3150801223009B30021204600973C235A46FDF784FC42
S3150801224000212046FDF796FA5A4659F8043C2946D4
S31508012250204608F10108FDF7EBF8BB44B8F1080F71
S315080122601FFA8BFBD1D10AE433685A462046FDF79B
S31508012270DFF8FFF7F5BB33685A462046FDF7D8F86D
S31508012280E2E74E4928462FF0F7F81FFA88F42B465D
S3150801229022468A214A48DFF85491DFF840A1FDF722
S315080122A0C7F8484B93F90020474B4FEA440853F8BF
S315080122B0221028462FF0E0F82B4642468A2140484C
S315080122C0FDF7B6F8414B93F90020414B284653F8E0
S315080122D022102FF0D1F82B4604EB08028A21384840
S315080122E0374DFDF7A5F83B4B35481A783A4B79082F
S315080122F053F822300A31A200FDF79AF8A3464FF0A7
S31508012300080859F8041B2846FDF7EEF8C0F18700BE
S3150801231087B203212846FDF72DFA274B93F900309A
S3150801232043450DD19AF80010D9B1002128460094E9
S3150801233087235A46FDF708FC00212846FDF71AFAB5
S315080123405A4659F8043C3946284608F10108FDF76A
S315080123506FF8A344B8F10C0F1FFA8BFBD1D1FFF725
S315080123608EBB33685A462846FDF762F8E8E73368B4
S315080123703A462046FDF75CF8D9E5336810480294D9
S31508012380FDF756F800E633680D480292FDF750F856
S3150801239027E633680A480292FDF74AF8D8F83C302E
S315080123A057E6D8F83C3055E6BF9D040878A70408D7
S315080123B0046204088BA80408E84D00208FA80408C5
S315080123C0C011002028250020680B0020204D002080
S315080123D0280C0020500B00201C0C0020681F002030
S315080123E0FE030020480C0020B40B0020C40B00207B
S315080123F001212046FDF7BEF99D4B93F90030102BBC
S3150801240040F0DE809B4B1978002900F0A1809A4B99
S315080124101C78002C00F0B580984928462FF02CF836
S3150801242029469748FDF760F8022104469448FDF7C6
S31508012430A1F9029B924800973A460021FDF784FBD1
S3150801244000218F48FDF796F9029B191B01EBD17103
S315080124502B463A46C1F34F018948DFF83892884C32
S31508012460FCF7E6FF1123039359F8041B2046FDF7F1
S315080124703BF8ABEB00001FFA80F803212046FDF775
S3150801248079F97B4B039A93F9003093420FD1794B33
S315080124901978002900F0A7800021204600975B469D
S315080124A05246FDF751FB00212046FDF763F959F81D
S315080124B0043C524641462046FCF7BAFF07EB0A039D
S315080124C01FFA83FA039B122B40F08A806D4C6C48E5
S315080124D0E16CFDF709F8029B181A674B1B7800EBAC
S315080124E0D070C0F34F08002B00F0838001216448A7
S315080124F0FDF740F95E4B93F90030132B4FEA87023B
S3150801250040F082805B4B1978002974D05E490392AA
S3150801251028462EF0B1FF29465948FCF7E5FF022166
S3150801252004465748FDF726F9DDE902325448009773
S315080125300021FDF709FB00215148FDF71BF9029B14
S31508012540039A191B01EBD1712B46C1F34F0182E5A1
S3150801255033684B483A46FCF76BFF4A4B48481B6CB5
S315080125603A464146FCF764FF484B93F90020484B2D
S31508012570284653F822102EF07FFF2B463A46494645
S315080125806AE7424B93F90020414B284653F822103B
S315080125902EF072FF2B463A4649463948FCF748FF62
S315080125A03748009721465B463A46FDF7CDFA344847
S315080125B02146FDF7DFF8334B3A461B6C41464BE79C
S315080125C0324B93F90020324B284653F822102EF04D
S315080125D053FF2B463A4649462948FCF729FFEAE7BD
S315080125E01223039340E7336852462046FCF720FF3F
S315080125F05DE703217BE7336821480292FCF718FF60
S31508012600E36C029A414626E5E36CFBE733683A46F2
S315080126102046FCF70DFFFFF70EBB336818480294F6
S31508012620FCF706FFFFF732BB11462846FCF75CFFAD
S3150801263033680290414622462846FCF7F9FE029B7A
S31508012640A9EB030808EBD878DAF80030FFF756BB90
S31508012650DAF800102846FCF747FFA9EB000000EB63
S31508012660D070DAF800302246C0F34F01FFF749BBB4
S31508012670E84D0020681F0020B4430020B7A80408CD
S31508012680C0110020A40B0020D3A80408783B002021
S31508012690840B0020E80B00202DE9F04F61496248C0
S315080126A0624F93B0FCF732FF5F48FCF717FF5E48AD
S315080126B00321FDF75FF83B78BBB95D4B5A482D22DC
S315080126C00521FCF7B5FE5B4B57482D220F21FCF778
S315080126D0AFFE594B544839220521FCF7A9FE574B41
S315080126E0514839226421FCF7A3FE55494E48FCF7A7
S315080126F00DFF4D48FCF7E1FE4B48FCF7EFFE4A4853
S315080127000321FDF737F84F4B4748DB6A002211468C
S31508012710FCF78EFE3B788BB94B4B43482822182190
S31508012720FCF786FE494B404834220F21FCF780FE10
S31508012730474B3D4834227021FCF77AFE3B78012B42
S3150801274005D1444B384828221821FCF771FEDFF8D9
S315080127500C91354D99F90020DFF804B14FF6FB735A
S31508012760F62113FB0213013A93FBF2F39BB203938F
S315080127704FF0000899F900305FFA88F69E424EDA62
S3150801278003212846FCF7F6FF039B16FB03F4324B9D
S3150801279093F900309E42A4B20FD13B78012B1BD18D
S315080127A00E23611D00930F220A2389B22846FDF7DD
S315080127B0CBF900212846FCF7DDFF721C594605A80E
S315080127C02EF0EAFDA11D05AB102289B22846FCF7B9
S315080127D02FFE08F10108CDE7022B14D14FF00E0A9E
S315080127E0611D2846CDF800A00A230F2289B2FDF7FC
S315080127F0ABF9211D1023009352460C2389B22846B2
S31508012800FDF75DF9D5E7002BD7D1611D0E2300939E
S315080128100F220A2389B22846FDF751F9CDE713B0ED
S31508012820BDE8F08F6C6A0408C0110020681F0020FB
S3150801283049B7040818C30408BF9D040878A7040803
S31508012840046204086C080020FEA804081BA90408F1
S315080128500DB9040823A90408D63C0020900D0020D0
S31508012860EDB304082DE9F04F2DED028BBA4DBB49A6
S31508012870DFF838A3BA4E93B02846FCF747FE284638
S31508012880FCF71BFE2846FCF729FE95F82A3095F831
S31508012890294028460321E41AFCF76CFF0022114659
S315080128A0DAF804302846FCF7C3FD28460321FCF76D
S315080128B061FFAC4B93F90020AB4BE4B253F82210FD
S315080128C005A82EF069FDA4B22846A84D05AB2246F7
S315080128D06E21FCF7ADFD2B781BB196F90030012B63
S315080128E00BD0A34BA34AA44905A82EF055FD9A4837
S315080128F005AB62006E21FCF79BFD2B78012B33D1CA
S3150801290096F90030012B38D19C4B18680368DB6BAC
S31508012910984767008146002800F05181944B954AF3
S31508012920954905A82EF038FD05A98B48FCF7DCFD6D
S31508012930032180468848FCF71DFF5FFA88F30133B7
S315080129403A46854800946D21FDF7FEF88248002134
S31508012950FCF710FF6E21804805AB3A46FCF768FD87
S315080129607D480321FCF706FF2B78022B40F0868170
S3150801297096F90030012B00F04F8196F90030022BB1
S3150801298040F080812B78012B34D196F90030022B47
S315080129906AD17A4B18680368DB6B984704EB4407DE
S315080129A08146002800F07C81714B724A724905A85C
S315080129B02EF0F2FC05A96848FCF796FD032180462E
S315080129C06548FCF7D7FE5FFA88F301333A46624851
S315080129D000946D21FDF7B8F85F480021FCF7CAFE9F
S315080129E06E215D4805AB3A46FCF722FD5A4803219C
S315080129F0FCF7C0FE2B78022B36D196F90030022B54
S31508012A0032D15C4A5E4905A82EF0C6FC04EB4402A5
S31508012A1005AB6E2150480392FCF70AFD05A94E48FD
S31508012A20FCF762FD524907464B48FCF75DFDFFB2CC
S31508012A30C3B2039A48480094013307F16D01FDF7C3
S31508012A4083F845480021FCF795FE494905A82EF06B
S31508012A5013FD07F16E01039A3F4805ABFCF7E8FC45
S31508012A603D480321FCF786FE3B480121FCF782FE1F
S31508012A702B78444A9FED447A002B00F0438196F95E
S31508012A800030012B40F039815368126A9FED3F8A65
S31508012A909B1A002BB8BF5B4207EE903AF8EEE77A2D
S31508012AA0A70087EE870A0237FDEEC07ACDED037AD5
S31508012AB0F8EEE77A30EE670A20EE080A2CF062FD96
S31508012AC0FDEEC07A039A17EE903A092BCCBF30492E
S31508012AD0304905A82EF060FC05AB3A461E48002190
S31508012AE0FCF7A6FC2B782C4A9FED2C7A002B00F0DC
S31508012AF0108196F90030012B40F006815368126A5D
S31508012B009B1A002BB8BF5B4207EE903AF8EEE77ABC
S31508012B1087EE870AFDEEC07ACDED037AF8EEE77AFD
S31508012B2030EE670A20EE080A2CF02CFDFDEEC07A7D
S31508012B30039A17EE903A092BCCBF1949194905A8EA
S31508012B402EF02AFC05AB3A4603484B21FCF770FCEC
S31508012B50154B93F900202BE0C011002004620408EC
S31508012B60CC3C0020A008002000080020681F002097
S31508012B70779A04086E9A04083DA90408AC1F002038
S31508012B8044A90408883E0020BCB64C450000C8424A
S31508012B9049A9040852A90408D03E0020E0A3074623
S31508012BA05CA9040865A90408D85200206C0800200D
S31508012BB09D4B002A40F0AF809C4A1A60AFE09C49C1
S31508012BC09C48FCF791FC5FFA80F808F101033A4644
S31508012BD0984800946D21FCF7B7FF49469548FCF7DC
S31508012BE0C9FD934905A82EF047FC05AB3A466E2167
S31508012BF09048FCF71DFC8F480321FCF7BBFD8E4A64
S31508012C008E4905A82EF0C8FB05AB3A4608F16E01B8
S31508012C108848FCF70DFCA7E6854A894905A82EF0E0
S31508012C20BBFB620005AB6E2182480392FCF700FCF0
S31508012C3005A98048FCF758FC7F4907467D48FCF7FB
S31508012C4053FCFFB2C3B2039A7A480094013307F1E1
S31508012C506D01FCF779FF77480021FCF78BFD764972
S31508012C6005A82EF009FC07F16E01039A714805AB18
S31508012C70FCF7DEFB6F480321FCF77CFD2B78002B64
S31508012C807FF47BAE6C4B6A4A6E4905A82EF084FB2D
S31508012C9005AB04EB44026E216648FCF7C9FB71E6F5
S31508012CA063496448FCF720FC5FFA80F808F10103E0
S31508012CB03A46604800946D21FCF746FF49465D484F
S31508012CC0FCF758FD5A4905A82EF0D6FB05AB3A463E
S31508012CD06E215848FCF7ACFB56480321FCF74AFD20
S31508012CE0554A564905A82EF057FB05AB3A4608F151
S31508012CF06E015048FCF79CFB7CE6022B02D1536817
S31508012D00D269C3E6136AFBE7022B02D15368D2697B
S31508012D10F6E6136AFBE7022A74D0012A74D093ED0A
S31508012D20007A2B78484A002B75D096F90030012B8A
S31508012D306CD15368126ADFF824B19B1A002BB8BF0D
S31508012D405B4207EE903AF8EEE77AA04687EE870AE5
S31508012D504FF00009FDEEC07ACDED037AF8EEE77A79
S31508012D6030EE670A20EE080A2CF00CFCFDEEC07A5C
S31508012D70039A17EE903A092BCCBF3449344905A872
S31508012D802EF00AFB3A4605AB96212A48294FFCF74D
S31508012D904FFB28480321FCF7EDFC5BF8041B38467A
S31508012DA0FCF7A2FBC0F16400C3B20321384608EE62
S31508012DB0103AFCF7DFFC96F900304B450CD129781F
S31508012DC059B300213846009464234246FCF7BCFEF9
S31508012DD000213846FCF7CEFC42465BF8043C18EE67
S31508012DE0101A384609F10109FCF722FB04EB08021F
S31508012DF0B9F1030F1FFA82F8CFD113B0BDEC028BDC
S31508012E00BDE8F08F134AD8E6134AD6E6022B02D15B
S31508012E105368D2698FE7136AFBE7DAF8003042464E
S31508012E203846FCF705FBD7E73425002074D135462B
S31508012E306E9A0408C0110020779A04083FA904086D
S31508012E4044A904083DA90408641D00206FA90408C3
S31508012E507AA90408DBAC2D47E4385E46F40700205E
S31508012E601FB55B4B93F90030A3B923F063FB594BAC
S31508012E7093F90030012B40F0A98057484368B3F510
S31508012E80E13F00F0A3804FF4E13104B0BDE8104002
S31508012E9023F082BB012B05D14FF461414F4823F042
S31508012EA07BFBE4E7022B02D14FF46131F6E7032BF2
S31508012EB004D14FF4E13023F079FBD8E7042B02D192
S31508012EC023F004FBD3E7082B02D14FF4E131E5E700
S31508012ED0072B68D14FF4E120414C23F067FB414BA6
S31508012EE004F14C0019682EF0C7FA3F4B04F155005E
S31508012EF019682EF0C1FA32233C4984F8643004F18A
S31508012F00F3002EF0B9FA3A4B04F1A80019682EF02D
S31508012F10B3FA384B04F1B70019682EF0ADFA364BFF
S31508012F2004F1C60019682EF0A7FA344B04F1D5004E
S31508012F3019682EF0A1FA324B04F1680019682EF0CF
S31508012F409BFA3049B1F906300093B1F90220B1F97B
S31508012F500430B1F9001004F16800F6F7F5FA2A4BC6
S31508012F6004F1880019682EF087FA2849B1F9063064
S31508012F700093B1F90220B1F90430B1F9001004F156
S31508012F808800F6F7E1FA0023C4F808312046204BF9
S31508012F90C4F80C31F6F756FCDB2204F219110F4876
S31508012FA027F038FF63E70B2B02D14FF4966175E7DB
S31508012FB0052B7FF45CAF174B1878174B03A953F809
S31508012FC020000A222FF080F9014667E704B010BDF8
S31508012FD0783B0020302D0020E09401209C940120AC
S31508012FE0CC380020E0070020E407002086A9040861
S31508012FF0540700207407002090070020AC07002022
S31508013000B4070020C0070020D0070020D4070020FD
S3150801301066662E41F0080020A4C9040860B9074B6A
S3150801302093F86030012B9EBF054B01221A70054AA1
S3150801303000231370044A1370704700BFBC1A00209E
S3150801304069890120042A00205C0A002008B5F7F7DF
S31508013050DDFE01280AD1084B1B7B2BB9014607481F
S31508013060F7F7DDF8032008BD0021F8E70328FAD0B1
S31508013070042818BF0020F6E7BC1A0020444F002098
S3150801308070B5F7F7C3FE0128044626D12A4B2B4D06
S315080130901E7826BB01462A48F7F7C1F8A9682848C9
S315080130A0F7F708FC274B28481E702146F7F7B7F8AB
S315080130B026482146F7F7B3F82148F7F7A9F8012872
S315080130C02AD023480121F7F7AAF822480121F7F760
S315080130D0A6F821480121F7F7A2F8032070BD184880
S315080130E0F7F79AF829681648F7F7E4FB1B4B1B789C
S315080130F01BB9144A1370214602E0012B07D100219E
S315080131001148F7F78CF81148F7F786F8D4E7022B38
S31508013110F9D10C4B1C70EEE70948F7F779F8012845
S31508013120DBD10B48F7F778F80A48F7F775F80A4834
S31508013130F7F772F8D1E700BF211E0020B00800207A
S31508013140E03C0020042A0020E44C0020E046002050
S31508013150FC2A002060460020A82C0020500B0020E5
S31508013160012808B50BD1064B064819682EF084F9D3
S31508013170BDE80840034903225620F6F749B908BDB8
S31508013180D44700202134012003461046CA1A02D02A
S3150801319019462DF021BB704737B50D460446002266
S315080131A00A48102124F0A0F944F002044FF0FF3335
S315080131B0022201A906488DF804408DF8055026F02B
S315080131C091FEFAF7D7FE03B030BD00BF00100240EA
S315080131D0209101201FB5104C8DF8070000220F48D9
S315080131E0102124F081F90DF107014FF0FF33012277
S315080131F0204626F077FE00238DF80F3001224FF086
S31508013200FF330DF10F01204627F00EF8FAF7B2FE4B
S315080132109DF80F0004B010BD209101200010024056
S3150801322013B50190F4F7FEFF01302DF0B7FA044605
S3150801323010B101992EF020F9204602B010BD000008
S3150801324010B5FFF7EDFF0446F4F7ECFF2318C0B1FC
S3150801325013F8012D2F2A00F1FF30F8D188B1002289
S315080132601A7020462BF087FD052805D12046FFF761
S31508013270E7FF20462BF07FFD18B9044821462EF0BA
S3150801328017F82046BDE810402DF090BA92A9040817
S31508013290194B30B51A68194C194DF4EE007AF9B97B
S315080132A0297800EB820306EE901A54F82330F8EEDB
S315080132B0666A013200EB820054F82020D21A07EE22
S315080132C0102AB8EEC77A27EE277A07EE903AF8EE73
S315080132D0E77AE6EE877AFDEEE77A17EE900A30BDD1
S315080132E02978531E06EE901A00EB8303F8EE666AF8
S315080132F054F82330023ADDE7242C0020DC52002062
S31508013300292C00202DE9F04F8F4ADFED907A002312
S315080133102DED088B13608E4A13608E4A13608E4A10
S3150801332013608E4BD3ED008A68EEA78ADFED8C7A9F
S31508013330B0EEE87AB4EEE77AF1EE10FA41BF894BBE
S31508013340DFED898A01221A60884B1B6887B0B3F5BD
S31508013350616F019300F3F380854B9FED868A5B6B62
S315080133600293854B854C5B6B0393854B5B6B04938F
S31508013370844B00255B6B0593AB46B0EE489AAA468B
S31508013380F0EE489A2F46B0EE48AA0126019BB342B1
S3150801339040F3C180226823699B1A002BB8BF5B42A0
S315080133A007EE903A62686369F8EEE77A9B1A002B92
S315080133B0B8BF5B4287EEA87AA26807EE903AA3697E
S315080133C09B1A002BF8EEE77AB8BF5B42C7EEA8AAAC
S315080133D0E26807EE903AE3699B1AF8EEE77A002B62
S315080133E0B8BF5B42C7EEA8BA07EE903AF8EEE77A9D
S315080133F0BDEEC77A87EEA8BADDED027AB8EEC76ADE
S31508013400F8EE676AFDEEEAAAC6EE267AFDEEEBBA93
S31508013410F4EECA7AF1EE10FABDEECBBA13DD17EE69
S31508013420100AF5F7AFF8804602988946F5F79AF833
S3150801343002460B4640464946F5F738FAF5F704FCC5
S315080134400AEE100A01279DED037AF8EEEA7AF8EEFC
S31508013450476A87EEA67AB4EEE97AF1EE10FA14DD38
S315080134601AEE900AF5F78EF8804603988946F5F71D
S3150801347079F802460B4640464946F5F717FAF5F735
S31508013480E3FB09EE900A4FF0010A9DED047AF8EE86
S31508013490EB7AF8EE476A87EEA67AB4EEC97AF1EEC8
S315080134A010FA14DD1BEE900AF5F76CF880460498BD
S315080134B08946F5F757F802460B4640464946F5F759
S315080134C0F5F9F5F7C1FB09EE100A4FF0010B9DED71
S315080134D0057AF8EECB7AF8EE476A87EEA67AB4EE65
S315080134E0C87AF1EE10FA13DD1BEE100AF5F74AF861
S315080134F0804605988946F5F735F802460B46404653
S315080135004946F5F7D3F9F5F79FFB08EE100A0125A9
S31508013510013610343AE717B10B4B83ED00AABAF11D
S31508013520000F02D00A4BC3ED009ABBF1000F02D07F
S31508013530084B83ED009A15B1074B83ED008A07B056
S31508013540BDEC088BBDE8F08F4C4600200024743F83
S31508013550504600205446002058460020780900208D
S315080135600AD7233C90460020FFFF7F7FE888012089
S31508013570883E002000000000D03E0020DC520020DA
S31508013580641D0020AC1D002070B55D4B93F9003019
S3150801359083B95C4B1B683BB95B4A136801331360FB
S315080135A05A4B01221A7070BD012BF9D1564A13687C
S315080135B0013BF4E7012BF6D1524C2368002B3BD192
S315080135C0534B51481D6803686A1E9A4240F082802F
S315080135D0504B06221A70504B0A26B3F900204F4B5E
S315080135E092FBF6F107EE901AD3ED006AB8EEE77A88
S315080135F006FB1122C7EE267A12B24949B6EE007ABF
S3150801360077EE877AFDEEE77A17EE903A1BB2002A33
S3150801361051D10B80434B1B7813B90B88DB000B8008
S31508013620414A056000231380404A13700123236031
S3150801363023F070F83E4B18602368012BB0D132484D
S315080136400368002B5AD1334B04221A70394B0A25C9
S31508013650B3F90020314B92FBF5F107EE901AD3ED41
S31508013660006AB8EEE77A05FB1122C7EE267A12B28E
S315080136702B49B6EE007A77EE877AFDEEE77A17EEF2
S31508013680903A1BB25ABB0B80264B1B7813B90B8891
S31508013690DB000B80244A00231380244A236013701D
S315080136A00123036023F036F8214B234A1860138857
S315080136B00133138074E7C7EE267A37EE877A07EE69
S315080136C0903AF8EEE77A77EE277AFDEEE77A17EE83
S315080136D0903A9EE77FF664AF0133036060E7C7EE71
S315080136E0267A37EE877A07EE903AF8EEE77A77EE9A
S315080136F0277AFDEEE77A17EE903AC4E7013BECE745
S31508013700D43C00208C460020242C0020CC08002024
S31508013710580A002095460020528F0120780900207A
S31508013720A02C00209C460020D42C0020FD29002036
S31508013730F8470020548F0120568F012008B52D4BDC
S3150801374093F90030002B39D12B4B1B68002B36D14E
S315080137502A4B1B68002B31D0294A126893422DD374
S31508013760284B06221A70284BB3F90020274B0A204A
S3150801377092FBF0F107EE901AD3ED006AB8EEE77AFC
S3150801378000FB1122C7EE267A12B22149B6EE007A5B
S3150801379077EE877AFDEEE77A17EE903A1BB2CAB949
S315080137A00B801C4B1B7813B90B88DB000B801A4B5B
S315080137B000221A8022F0AEFF184B186008BD012BB3
S315080137C0FCD10E4B1B68002BF8D10E4B04221A7044
S315080137D0134BC9E7C7EE267A37EE877A07EE903A92
S315080137E0F8EEE77A77EE277AFDEEE77A17EE903A62
S315080137F0D6E700BFD43C00208C460020242C0020AC
S31508013800580A002095460020528F01207809002089
S31508013810A02C00209C460020D42C0020F84700202C
S31508013820548F012010B50446ADF5667D2E48FCF788
S3150801383047FA122221465AA82AF044FF052807D139
S315080138402046FFF7FDFC0A2221465AA82AF03AFF2C
S3150801385030B12548FCF74AFA00200DF5667D10BD02
S31508013860224922461AA82DF097FD1AA8F4F7DAFC80
S315080138706B4602461AA95AA82BF0DBF81C4A1D49C1
S3150801388001A82DF089FD01A8F4F7CCFC6B46024688
S3150801389001A95AA82BF0CDF817496B464FF40062D7
S315080138A05AA82BF0C6F815496B464FF480725AA8E8
S315080138B02BF0BFF812496B464FF480725AA82BF0C9
S315080138C0B8F810496B46C0225AA82BF0B2F800285E
S315080138D0BFD15AA82BF0BDF90028BAD10248FCF786
S315080138E005FA0120B9E700BFA5A9040897AA0408A3
S315080138F0D1A90408E1A90408702F002012060020A6
S31508013900120500207037002010B5ADF5507D0190E5
S315080139102248FCF7D5F90199012244A82AF0D2FEDA
S315080139200446002832D144AA4FF4807104A82BF02A
S31508013930D5FA44AA4FF4807104A82BF0CFFA184996
S3150801394003AB4FF4006244A82AF0C0FF154903AB44
S315080139504FF4807244A82AF0B9FF134903AB4FF418
S31508013960807244A82AF0B2FF104903ABC02244A8CA
S315080139702AF0ACFF30B10948FCF7B8F920460DF535
S31508013980507D10BD44A82BF064F904460348FCF7A2
S31508013990ADF9B4FA84F04009F1E700BFA5A9040816
S315080139A0702F002012060020120500207037002013
S315080139B010B50446ADF5667D2848FCF781F9122253
S315080139C021465AA82AF07EFE052807D12046FFF788
S315080139D037FC0A2221465AA82AF074FE30B11F483C
S315080139E0FCF784F900200DF5667D10BD1C492246B9
S315080139F01AA82DF0D1FC1AA8F4F714FC6B46024656
S31508013A001AA95AA82BF015F8164A174901A82DF034
S31508013A10C3FC01A8F4F706FC6B46024601A95AA89D
S31508013A202BF007F811496B464FF461425AA82BF05F
S31508013A3000F80028D3D10E496B4645F260425AA8D0
S31508013A402AF0F7FF0028CAD15AA82BF002F9002854
S31508013A50C5D10248FCF74AF90120C4E7A5A904081B
S31508013A6097AA040847AA0408E1A90408DC52002019
S31508013A708034012070B50546ADF5667D3948FCF7F9
S31508013A801FF9122229465AA82AF01CFE05280446BF
S31508013A9008D12846FFF7D4FB0A2229465AA82AF054
S31508013AA011FE044634B12F48FCF720F900200DF524
S31508013AB0667D70BD2C492D4E2A461AA82DF06CFC40
S31508013AC01AA8F4F7AFFB6B4602461AA95AA82AF0B8
S31508013AD0B0FF274A274901A82DF05EFC01A8F4F793
S31508013AE0A1FB6B46024601A95AA82AF0A2FF56F87D
S31508013AF0045B6B46012205F143015AA82AF099FF96
S31508013B006B46042205F134015AA82AF092FF6B4646
S31508013B10022205F130015AA82AF08BFF6B460122D1
S31508013B2005F140015AA82AF084FF6B46012205F1E6
S31508013B3041015AA82AF07DFF01346B46012205F19D
S31508013B4044015AA82AF075FF042CD0D10028AAD11D
S31508013B505AA82BF07EF80028A5D10248FCF7C6F82A
S31508013B600120A4E7A5A9040897AA0408D0C904084E
S31508013B7056AA0408E1A9040870B5ADF5547D059067
S31508013B803748FCF79DF80599012248A82AF09AFDBD
S31508013B900446002845D148AA4FF4807108A82BF09D
S31508013BA09DF948AA4FF4807108A82BF097F92D4E74
S31508013BB056F8045B07AB012205F1430148A82AF030
S31508013BC085FE07AB042205F1340148A82AF07EFEDA
S31508013BD007AB022205F1300148A82AF077FE07ABA8
S31508013BE0012205F1400148A82AF070FE07AB01221F
S31508013BF005F1410148A82AF069FE013407AB012203
S31508013C0005F1440148A82AF061FE042CD0D120B15F
S31508013C101348FCF76BF800201EE048A82BF019F8AA
S31508013C2004460F48FCF762F8002CF4D10D4D55F8FF
S31508013C30040B90F84420038E90F84310029290F8F2
S31508013C404120019290F840200092426B0134FCF722
S31508013C505DFB042CEBD101200DF5547D70BD00BF31
S31508013C60A5A90408D0C9040810B5504B504C1A88A8
S31508013C70504920462DF090FB4F4B214618462DF012
S31508013C80FBFB4E4A127882724D4A1278C2724D4A2D
S31508013C90127802734C4A127842734C4A127882732C
S31508013CA04B4A1278C2734B4A127802744A4A1278FE
S31508013CB042744A4A12788274494A1278C274494A45
S31508013CC0D169126A8261484A4161D169126A0262FE
S31508013CD0464AC161D169126A8262454A4162D1691D
S31508013CE0126A0263434AC16212684263424A12680F
S31508013CF08263424A1268C263414A12680264414AAF
S31508013D0012684264404A12688264404A034610684F
S31508013D103F4AD86411683F4A19651288A3F85420A6
S31508013D203D4A1288A3F856203C4A1288A3F858201F
S31508013D303B4A1288A3F85A203A4A1288A3F85C200B
S31508013D40394A1288A3F85E20384A127883F8602027
S31508013D50374A127883F86120364A127883F8622046
S31508013D60354A127883F86320344A147883F8644014
S31508013D70547883F865409478D27883F86720304A76
S31508013D8083F86640147883F86840547883F8694064
S31508013D909478D27883F86B202A4A83F86A40127895
S31508013DA083F86C20C3E91C0110BD00BF520B00202B
S31508013DB05C3D00206CAA0408BC1A0020D40D002022
S31508013DC0D50D0020304000201404002015040020E1
S31508013DD0D8520020783B0020FC8801205E1D002077
S31508013DE070480020883E0020D03E0020641D002037
S31508013DF0AC1D0020E0080020DC0D0020E40D0020A9
S31508013E00E00D002078090020400A0020E8880120FA
S31508013E10580A0020520700209C0C0020548F0120CC
S31508013E20528F0120DA3C0020DC3C0020A00800204B
S31508013E30900D0020D43C0020D13C00200204002033
S31508013E40FE030020514200202DE9F74FE24FDFF82B
S31508013E50FC83DFF8FC93DFF8FCA3DFF8FCB30C4620
S31508013E60054616463B46DD4ADD4920462DF094FABD
S31508013E702046F4F7D7F933460246214628462AF062
S31508013E80D8FDBB7AD74A414620462DF085FA204609
S31508013E90F4F7C8F933460246214628462AF0C9FDF1
S31508013EA0FB7AD14A414620462DF076FA2046F4F7A8
S31508013EB0B9F933460246214628462AF0BAFD7B7BE4
S31508013EC0CA4A414620462DF067FA2046F4F7AAF970
S31508013ED033460246214628462AF0ABFDBB7BC44A37
S31508013EE0414620462DF058FA2046F4F79BF9334609
S31508013EF00246214628462AF09CFD97F90F30BD4A0D
S31508013F00414620462DF048FA2046F4F78BF9334608
S31508013F100246214628462AF08CFD97F91030B64A02
S31508013F20414620462DF038FA2046F4F77BF9334608
S31508013F300246214628462AF07CFD7B7CAF4A41464B
S31508013F4020462DF029FA2046F4F76CF93346024645
S31508013F50214628462AF06DFD97F91230A84A4146AE
S31508013F6020462DF019FA2046F4F75CF93346024645
S31508013F70214628462AF05DFD97F91330A14A4146A4
S31508013F8020462DF009FA2046F4F74CF93346024645
S31508013F90214628462AF04DFD7B699B4A494620461B
S31508013FA02DF0FAF92046F4F73DF933460246214643
S31508013FB028462AF03EFDBB69944A494620462DF01B
S31508013FC0EBF92046F4F72EF93346024621462846F0
S31508013FD02AF02FFDFB698E4A494620462DF0DCF969
S31508013FE02046F4F71FF933460246214628462AF0A9
S31508013FF020FD3B6A874A494620462DF0CDF92046E1
S31508014000F4F710F933460246214628462AF011FDEF
S315080140107B6A814A494620462DF0BEF92046F4F7C7
S3150801402001F933460246214628462AF002FDBB6AB3
S315080140307A4A494620462DF0AFF92046F4F7F2F8B8
S3150801404033460246214628462AF0F3FCFB6A744A9F
S31508014050494620462DF0A0F92046F4F7E3F8334601
S315080140600246214628462AF0E4FC3B6B6D4A49463E
S3150801407020462DF091F92046F4F7D4F83346024646
S31508014080214628462AF0D5FC7B6B524649462046EE
S315080140902DF082F92046F4F7C5F833460246214643
S315080140A028462AF0C6FCBB6B5F4A494620462DF0D6
S315080140B073F92046F4F7B6F83346024621462846F0
S315080140C02AF0B7FCFB6B5A46494620462DF064F99F
S315080140D02046F4F7A7F833460246214628462AF031
S315080140E0A8FCFB6B5A46494620462DF055F9204651
S315080140F0F4F798F833460246214628462AF099FCF1
S31508014100386CF4F751FA494ACDE900014849204685
S315080141102DF042F92046F4F785F833460246214642
S3150801412028462AF086FC786CF4F73EFA414ACDE92E
S315080141300001414920462DF02FF92046F4F772F87F
S3150801414033460246214628462AF073FC7B6B5246C3
S31508014150494620462DF020F92046F4F763F8334600
S315080141600246214628462AF064FCBB6C334A494676
S3150801417020462DF011F92046F4F754F83346024645
S31508014180214628462AF055FCFB6C2D4A494620460D
S315080141902DF002F92046F4F745F833460246214642
S315080141A028462AF046FC3B6D264A494620462DF00C
S315080141B0F3F82046F4F736F83346024621462846F0
S315080141C02AF037FCB7F954301F4A414620462DF0EC
S315080141D0E3F8204642E000BFBC1A002073AA04088F
S315080141E092AA04089BAA0408BDAA0408D6AA040828
S315080141F0EDAA040803AB040816AB040829AB0408A6
S3150801420044AB04085DAB040870AB04089EAB040814
S31508014210C0AB0408E5AB040808AC04082BAC0408D9
S315080142204CAC04086FAC0408B3AC040815AD04081B
S315080142303AAD040846AD040867AD040873AD040831
S3150801424094AD0408B6AD0408D8AD0408B4AA0408A8
S3150801425094AB040890AC0408E4AC0408F3F7E2FF55
S3150801426033460246214628462AF0E3FBB7F956307B
S315080142709F4A414620462DF08FF82046F3F7D2FF94
S3150801428033460246214628462AF0D3FBB7F9583069
S31508014290984A414620462DF07FF82046F3F7C2FF9B
S315080142A033460246214628462AF0C3FBB7F95A3057
S315080142B0914A414620462DF06FF82046F3F7B2FFA2
S315080142C033460246214628462AF0B3FBB7F95C3045
S315080142D08A4A414620462DF05FF82046F3F7A2FFA9
S315080142E033460246214628462AF0A3FBB7F95E3033
S315080142F0834A414620462DF04FF82046F3F792FFB0
S3150801430033460246214628462AF093FB97F9603040
S315080143107C4A414620462DF03FF82046F3F782FFB6
S3150801432033460246214628462AF083FB97F961302F
S31508014330754A414620462DF02FF82046F3F772FFBD
S3150801434033460246214628462AF073FB97F962301E
S315080143506E4A414620462DF01FF82046F3F762FFC4
S3150801436033460246214628462AF063FB97F963300D
S31508014370674A414620462DF00FF82046F3F752FFCB
S3150801438033460246214628462AF053FB97F96430FC
S31508014390604A414620462CF0FFFF2046F3F742FFCC
S315080143A033460246214628462AF043FB97F96530EB
S315080143B0594A414620462CF0EFFF2046F3F732FFD3
S315080143C033460246214628462AF033FB97F96630DA
S315080143D0524A414620462CF0DFFF2046F3F722FFDA
S315080143E033460246214628462AF023FB97F96730C9
S315080143F04B4A414620462CF0CFFF2046F3F712FFE1
S3150801440033460246214628462AF013FB97F96830B7
S31508014410444A414620462CF0BFFF2046F3F702FFE7
S3150801442033460246214628462AF003FB97F96930A6
S315080144303D4A414620462CF0AFFF2046F3F7F2FEEF
S3150801444033460246214628462AF0F3FA97F96A3096
S31508014450364A414620462CF09FFF2046F3F7E2FEF6
S3150801446033460246214628462AF0E3FA97F96B3085
S315080144702F4A414620462CF08FFF2046F3F7D2FEFD
S3150801448033460246214628462AF0D3FA97F86C3075
S31508014490284A414620462CF07FFF2046F3F7C2FE04
S315080144A033460246214628462AF0C3FA3B6F224A7A
S315080144B0414620462CF070FF2046F3F7B3FE3346FB
S315080144C00246214628462AF0B4FA7B6F1B4A414622
S315080144D020462CF061FF2046F3F7A4FE3346024638
S315080144E02146284603B0BDE8F04F2AF0A2BA00BF1C
S315080144F004AE040825AE040855AE040886AE0408C1
S31508014500A3AE0408C1AE0408E0AE040805AF04086A
S315080145102BAF040849AF040869AF04088AAF040839
S31508014520A9AF0408C8AF0408E9AF04080BB004082A
S315080145302BB004084BB004086DB0040890B0040809
S3150801454010B50446ADF5667D5248FBF7B9FB122254
S3150801455021465AA82AF0B6F8052807D12046FEF7BB
S315080145606FFE0A2221465AA82AF0ACF830B149480A
S31508014570FBF7BCFB00200DF5667D10BD46492246BA
S315080145801AA82CF009FF1AA8F3F74CFE6B46024647
S315080145901AA95AA82AF04DFA6A461AA95AA8FFF77B
S315080145A053FC3E4A3E4901A82CF0F6FE01A8F3F752
S315080145B039FE6B46024601A95AA82AF03AFA6B4611
S315080145C038497C225AA82AF034FA374B93F9003035
S315080145D0022B1DDD354A324901A82CF0DDFE01A862
S315080145E0F3F720FE6B46024601A95AA82AF021FADA
S315080145F02F496B4690225AA82AF01BFA0028B6D1F1
S315080146002C496B4636225AA82AF013FA0028AED14D
S31508014610294A234901A82CF0BFFE01A8F3F702FE97
S315080146206B46024601A95AA82AF003FA23496B46A2
S315080146304FF461425AA82AF0FCF9002897D1204A7A
S31508014640174901A82CF0A8FE01A8F3F7EBFD6B4664
S31508014650024601A95AA82AF0ECF91A496B4645F20D
S3150801466060425AA82AF0E5F9002880D15AA82AF00A
S31508014670F0FA15490B8804460133022205200B80FE
S31508014680F4F702FF002C7FF472AF0248FBF72EFB0A
S31508014690012070E7A5A9040897AA0408B3B004087D
S315080146A0E1A90408BC1A0020900D0020C2B0040834
S315080146B0244300203234012034AA0408DC520020A5
S315080146C030AA040880340120520B00202DE9F04F4E
S315080146D0374E3849DFF81491DFF8148197B0304620
S315080146E0FAF714FF3046FAF7E8FE3046FAF7F6FE0F
S315080146F00321304696F9294096F92AB03588FBF701
S3150801470039F82D4B002211461B693046FAF790FEFF
S3150801471099F90020294B09A853F82210F4F72FFD1F
S3150801472009A92748F6F700F909A8F4F7E3FC254B88
S315080147301B78012B0CBF2449244909A8F4F71FFD4E
S3150801474009A92348F6F7F0F809A8F4F7D3FCD8F82D
S315080147500020204909A82CF01FFE09A906A8F4F78C
S315080147600EFD1D4806A9F6F7DFF806A8F4F7C2FC00
S3150801477099F90030012B40F06781184906A8F4F72A
S31508014780FEFC174806A9F6F7D2F806A8F4F7B2FC14
S31508014790144B1B68B3F5167F2CDA0A2193FBF1F249
S315080147A001FB1233104909A82CF0F6FD40E000BFC1
S315080147B0C0110020BA5A04086C080020000800201D
S315080147C0FC42002030400020D5B00408D9B00408C6
S315080147D0A4420020ECB304087C420020DCB00408A3
S315080147E0D4420020DC0D0020E3BB0408A008002009
S315080147F0E0080020B64B9A6BB3F95810B3F95A3052
S31508014800114419444FF4167048F6A043B1FBF0F76A
S31508014810B1FBF3F203FB121300FB1711B3FBF0F321
S315080148200A2709A8B1FBF7F10091AA492CF0B4FDB2
S3150801483009A906A8F4F7A3FCA74806A9F6F774F888
S3150801484006A8F4F757FCDFF808A3A44B9AF800204A
S315080148501B78002A00F015812BB1A14B93F9003082
S31508014860012B00F016819F4B1B78002B00F0048169
S315080148709D4A9E4B12689E4909A82CF08DFD9D4BB9
S3150801488093F90030002B00F0AB829B4D0424286875
S315080148900621F6F77FF855F8040BF6F7CBF8013C35
S315080148A0F5D196F8294096F82A209448358809A919
S315080148B0A41AFAF719FE99F90030E4B2281A00EB9E
S315080148C0D070A600012BC0F34F01A7B204EB440A2E
S315080148D0B34609AB40F0018288483246FAF7A8FD8B
S315080148E0874B1B78002B00F044818649DFF86492D8
S315080148F009A82CF0C1FD09A98048FAF7F5FD4FEA88
S315080149005508A8EB000000EBD07009ABC0F34F01C6
S3150801491052467A48FAF78CFD7B4909A82CF0ACFD7A
S315080149207A4B05934FF0000B059B13F8012B059362
S31508014930043A012A0CD809A8BBF1000F40F01B81E3
S31508014940F3F770FC462209AB494618442CF024FDBE
S315080149500BF1010BBBF1030FE6D109A8F3F762FCD2
S315080149600B2804D16A490DF12F002CF085FD09A900
S315080149706248FAF7B9FDA8EB000000EBD07008EB26
S31508014980600009AB81B252465C48FAF751FD534BB8
S315080149901B78002B40F0FA805E4B5F4AB3F9008022
S315080149A05E4BD3ED007A5E4BB7EE007A87EE276A47
S315080149B04FF00A0A98FBFAF907EE908AB8EEE77AF9
S315080149C0DFED587A27EE067AF2EE045AC7EE276A21
S315080149D00AFB198892ED007AC3ED006AB8EEC77A28
S315080149E00FFA89F3C7EE257A059367EE867AC7EE3D
S315080149F0A67A17EE900AF3F7D7FD0FFA88F2CDE9F2
S31508014A0002010092484A059BD268484909A82CF038
S31508014A10C3FC09A93948FAF767FD281A00EBD070D3
S31508014A20BA19C0F34F0109AB34480592FAF700FDEC
S31508014A302B4B059A93F90010002940F01C813C4B39
S31508014A402E48FAF7F5FC16E1002B7FF4FCAE39493E
S31508014A5006A8F4F794FB06A91F48F5F768FF06A808
S31508014A60F4F748FB344BB3F900300A2193FBF1F212
S31508014A7001FB12331BB295E6304909A82CF0FCFC60
S31508014A80FDE623B1164B93F90030012B01D02C49D1
S31508014A90F3E72C4F3B7801333B70002AF7D0114BD3
S31508014AA01B78002B58D0104A104B1268264909A8C2
S31508014AB02CF072FC3B78072B7FF6E1AE234B1B7873
S31508014AC0012B04BF00238AF8003000233B70D6E689
S31508014AD0BC1A0020E6B00408D4420020681F002052
S31508014AE0D73C0020211E0020D44700205C3D002031
S31508014AF022B10408D13C002018040020C01100206E
S31508014B003C3800204AB1040871B10408F4030020B6
S31508014B1080B104087C090020DC0D002078090020FA
S31508014B209846002000007A441808002085B1040838
S31508014B30EE510408F3B0040852070020FDB004083A
S31508014B4012B104089F2C00201BB10408500B002049
S31508014B50042A00207DB104088E49059309A82CF082
S31508014B608BFC3A78072A7FF68AAE059B8AF80030CD
S31508014B70ACE78949BAE6BBF1010F03D1F3F752FB5A
S31508014B804922E0E6F3F74EFB5A22DCE6834B93F91A
S31508014B900090B9F1000F6ED1814B8249B3F90080BB
S31508014BA0814BDFF838A2D3ED007A804BB7EE007A55
S31508014BB087EE276A0A2298FBF2FB07EE908AB8EE7F
S31508014BC0E77ADFED7B7A27EE067AF2EE045AC7EE2C
S31508014BD0276A91ED007AC3ED006AB8EEC77A0FFA33
S31508014BE08BF3C7EE257A059367EE867AC7EEA67A22
S31508014BF017EE900AF3F7D8FC0A22CDE9020102FB67
S31508014C001B880FFA88F20092059BDAF80C2069498D
S31508014C1009A82CF0C1FB09A96748FAF765FC281A07
S31508014C2000EBD070C0F34F08BA1909AB4146624888
S31508014C300592FAF7FDFBDAF80C1009A82CF01CFC12
S31508014C4009A95D48FAF750FC58FA80F34946059ACE
S31508014C50594800979BB2FAF777FF49465648FAF73B
S31508014C6089FD4146059A544809ABFAF7E1FB5248D2
S31508014C700321FAF77FFD514B484E1B78002B00F0B4
S31508014C80F28196F90030012B40F0ED814C4B1B78EF
S31508014C90002B40F0E6814B4909A82CF0EDFB09A948
S31508014CA04548FAF721FC281A00EBD07004EB4404B6
S31508014CB0620009ABC0F34F013F480592FAF7B8FB0A
S31508014CC096F90030059A012B04D13F4B3A48002149
S31508014CD0FAF7AEFB17B0BDE8F08F52463648FAF739
S31508014CE0A7FB3A4B3A49B3F90090D8F80030324855
S31508014CF003FB09F9FAF70AFC2F480321FAF73AFDEB
S31508014D004FF4167048F6A043B9FBF0F1B9FBF3F27C
S31508014D104FF00A0A03FB129300FB1199B3FBF0F358
S31508014D20B9FBFAF109A800912A492CF035FB09A922
S31508014D302148FAF7D9FB281A00EBD070BA19C0F343
S31508014D404F0109AB1C48FAF773FBD8F80010182075
S31508014D501E2791FBF0F200FB121391FBF7F60AFBF3
S31508014D6003F307FB161193FBF0F3032709A891FB3D
S31508014D70F7F1CDE9006118492CF00EFB0E4809A997
S31508014D80FAF7B2FB281A00EBD07009AB5A46C0F302
S31508014D904F0155E632B104085EB10408D73C00203C
S31508014DA07C090020DC0D00207809002098460020A7
S31508014DB000007A4485B10408C0110020681F00204C
S31508014DC05C0A0020E4B10408EE51040852070020E9
S31508014DD0BA5A0408ABB10408C0B10408180800207F
S31508014DE0A24F042638680621F5F7D4FD57F8040BB7
S31508014DF0F5F720FE013EF5D109A99D48FAF774FB9E
S31508014E00A4EB0B04281AE4B200EBD07009ABC0F38B
S31508014E104F0104EB44029648FAF70AFB99F9003068
S31508014E20012BA7B240F0C380924BDFF884921B781E
S31508014E30002B54D1904B914AB3F90080904BD3ED96
S31508014E40007A904BB7EE007A87EE276A4FF00A0B85
S31508014E5098FBFBFA07EE908AB8EEE77ADFED8A7AD5
S31508014E6027EE067AF2EE045AC7EE276A0BFB1A8872
S31508014E7092ED007AC3ED006AB8EEC77A0FFA8AF3A3
S31508014E80C7EE257A059367EE867AC7EEA67A17EEF8
S31508014E90900AF3F789FB0FFA88F2CDE9020100922D
S31508014EA07A4A059BD2687A4909A82CF075FA09A9A4
S31508014EB06F48FAF719FB281A00EBD070BA0009AB4C
S31508014EC0C0F34F016A480592FAF7B2FA99F9003028
S31508014ED0059A002B7FF4CFAE6E4B3146B0E599F9B2
S31508014EE00030002B7FF4C7AE634B644AB3F90080E8
S31508014EF0634BDFF89891D3ED007A624BB7EE007AEF
S31508014F0087EE276A4FF00A0B98FBFBFA07EE908AA1
S31508014F10B8EEE77ADFED5C7A27EE067AF2EE045A06
S31508014F20C7EE276A0BFB1A8892ED007AC3ED006A71
S31508014F30B8EEC77A0FFA8AF3C7EE257A059367EEB4
S31508014F40867AC7EEA67A17EE900AF3F72DFBCDE916
S31508014F5002010FFA88F20092059BD9F80C204C49F8
S31508014F6009A82CF019FA09A94148FAF7BDFA281A2D
S31508014F7000EBD070C0F34F08BA0009AB41463C4874
S31508014F800592FAF755FAD9F80C1009A82CF074FA13
S31508014F9009A93748FAF7A8FA58FA80F33146059A63
S31508014FA0334800979BB2FAF7CFFD314656E63A4B9E
S31508014FB03A49B3F90060D8F800302D485E43FAF74C
S31508014FC0A5FA2B480321FAF7D5FB4FF4167148F6D3
S31508014FD0A043B6FBF1F0B6FBF3F24FF00A0903FB67
S31508014FE0126301FB1066B3FBF1F3B6FBF9F62C4924
S31508014FF0009609A82CF0D0F909A91D48FAF774FA00
S31508015000281A00EBD07007EB8702C0F34F0109ABF2
S315080150101748FAF70DFAD8F8001018204FF01E0CA9
S3150801502091FBF0F200FB1213BE0009FB03F391FB9F
S31508015030FCF793FBF0F30CFB171109A84FF0030CCF
S3150801504091FBFCF1CDE9007116492CF0A5F9084848
S3150801505009A9FAF749FA281A00EBD07009AB3246C2
S3150801506095E6114918E6114916E600BF180400200D
S31508015070C0110020681F00207C090020DC0D0020DB
S31508015080780900209846002000007A441808002074
S3150801509085B10408EE51040852070020BA5A0408DB
S315080150A0ABB10408C0B10408EAB10408FEB10408AA
S315080150B0D73C0020F0B58B498B488B4D9FB0FAF74A
S315080150C025FA8A4B1B78002B4BD1894B0822F821EC
S315080150D02846FAF7ADF987498348FAF717FA824855
S315080150E0FAF7EBF98048FAF7F9F995F8294095F8AE
S315080150F02A302E88804D7C480321E41AFAF73AFBB8
S3150801510029780229E4B202D17748FAF733FB2978DC
S31508015110012902D17448FAF72DFB784B93F900203F
S31508015120002A40F02181764B6F485B691146FAF7F0
S315080151307FF9744B1B68162BA4B240F0B280724BF0
S3150801514093F90030022B11AD68D1704B1B78013BE6
S31508015150082B12D8DFE803F00C5356595C111111CC
S315080151605F006B4B1B780BB96A4BAFE76A4BADE730
S315080151706A4B196828462CF07FF9694A0095D2E9E5
S315080151800023684904A82CF007F904AB22460F212D
S315080151905548FAF74DF9644E644F32683B686449DD
S315080151A004A865002CF0F8F804AB2A460F214E48EE
S315080151B0FAF73EF933683968C91A5E4BB3F9003014
S315080151C04FF41670594348F6A043B1FBF0F6B1FB0C
S315080151D0F3F203FB121300FB1611B3FBF0F30A26D5
S315080151E004A8B1FBF6F1009153492CF0D5F83E48D5
S315080151F004AB62190F21FAF71BF91FB0F0BD474B33
S315080152005968B7E7454B9968B4E7444BD968B1E79C
S31508015210424B1969AEE7414B5969ABE7ADDD474BDF
S315080152201B78643B0A2BA8D801A252F823F000BFC9
S31508015230715101085D5201086B5201087352010848
S315080152407B520108835201088B52010893520108C7
S315080152509B5201081152010817520108384B394966
S315080152601A6828462CF098F887E7354B36491A68A4
S31508015270F7E7334B35491A68F3E7314B34491A686E
S31508015280EFE72F4B33491A68EBE72D4B32491A687A
S31508015290E7E72B4B31491A68E3E7294B30491A6886
S315080152A0DFE7172B7FF477AF1D4D2E49AB682A68C8
S315080152B004A82CF071F804AB22460F210A48FAF724
S315080152C0B7F8696904A82CF067F804A90648FAF73B
S315080152D00BF9301A00EBD07004AB3322C0F34F013F
S315080152E056E700BF6C6A0408C01100200A2E002088
S315080152F00FB204080462040815040020A00800205F
S315080153006C080020980C0020900D0020C046002053
S315080153100B2E002011B2040813B204081C0B00203E
S31508015320380B002035B20408242C0020E888012017
S3150801533000B80408520700203DB20408C1460020FF
S31508015340340B002015B2040819B204081DB204086A
S3150801535021B2040825B2040829B204082DB20408AA
S3150801536031B2040811530408012A7FF446AF3C4BB5
S315080153703C481B6A00221146FAF75AF83A4B1B6851
S31508015380162BA4B268D1394B1B78052B48D1384B5B
S31508015390344822460F21FAF74BF8364B364A374935
S315080153A01B681268D1ED007AB2EE047A991A27EED3
S315080153B0877A07EE901AF8EE677A48F6A04567EEFF
S315080153C0277A4FF41676FCEEE77A0A2717EE901A33
S315080153D0B1FBF5F005FB1011B1FBF6F506FB15114E
S315080153E0B1FBF7F607FB1611CDE90005CDE9026118
S315080153F004A8234965002BF0CFFF04AB19482A46B8
S315080154000F21FAF715F81F4B93F90030012B7FF49A
S31508015410F4AE1D4B1D491A8804A82BF0BDFFE6E61C
S31508015420042B07D11A4B1B491A6804A82BF0B4FFA1
S3150801543004ABADE7062B03D1154B17491A68F4E7F8
S31508015440032B03D1124B15491A68EEE7022BA4D197
S315080154500F4B13491A68E8E7172B9ED1114B97E7AB
S315080154606C080020C0110020980C002095460020E9
S3150801547059B20408E8880120242C00207809002064
S31508015480ABB20408D43C0020568F0120CBB20408E5
S31508015490380B002067B2040872B204087EB2040809
S315080154A08CB204089EB204082DE9F74F2D4C2E49FB
S315080154B0DFF8BC90DFF8BC80DFF8BCB02046FAF70D
S315080154C025F82046F9F7F9FF2046FAF707F894F880
S315080154D02A3094F8295003212046ED1AFAF74AF999
S315080154E00022D9F81C3011462046EDB2F9F7A0FF83
S315080154F0ADB2AA46002758F8041B2046F9F7F4FF6F
S31508015500C0F1640086B203212046FAF733F9174B36
S3150801551093F90030BB420DD19BF80010D9B1002197
S315080155202046009564235246FAF70EFB00212046D1
S31508015530FAF720F9524658F8043C31462046013715
S31508015540F9F776FF05EB0A02032F1FFA82FAD2D181
S3150801555003B0BDE8F08FD9F8003052462046F9F776
S3150801556067FFE7E7C011002004620408D33C002066
S315080155706C0800205C080020681F00202DE9F04116
S315080155804A4A1378BBB1012B0AD1494801780B293C
S3150801559008D00C39032903D800211170454A137024
S315080155A0BDE8F08100211170424A1370424B1B7805
S315080155B001330370F4E73E4909780C2963D00E29B3
S315080155C06AD00B29ECD1012111703B4A92F90040AE
S315080155D074BB3A4B3A4E1C703A4B3B4F93F9003029
S315080155E08B4208BF394B3A4908BF1C60394B1868CA
S315080155F0394B06251C68002311F8012B042A10D102
S31508015600A0420CD0024603EB060E944207DD05FBC9
S3150801561002FC33F807802EF80C800132F5E701F811
S31508015620015C0233062BE7D1224B01221A70B7E738
S31508015630012C15D0022CF7D1244A28481360284B8F
S315080156401970F4F7E5FD012803D124482146F4F73A
S31508015650C7FD244B1A78012A0DD000221A700AE0D8
S315080156601A4A116859B91460164B93F90030012B7F
S3150801567004BF00231360114B00221A70D4E70129D5
S3150801568008BF1360F0E70C490A78013A52B2002ABA
S31508015690ACBF0A700B70C7E7074A137801335BB2D0
S315080156A0022BC8BF02231370BEE700BF681F002084
S315080156B069890120CC080020D33C0020022A002059
S315080156C080340120D43C0020683401208C46002017
S315080156D0F4030020242C0020E8880120E03C002067
S315080156E05C0A0020304000202DE9F04190B00024EA
S315080156F006460D4605A82449F3F741FDA04622466C
S31508015700AB68984504F1010725D22E212846039254
S31508015710F3F7E6FD5FFA80F8039A434629460CA893
S31508015720F3F7ECFD0CA905A8F3F77CFD0CA8F3F734
S31508015730E1FC002105A8F3F7A6FD05A8F3F704FE89
S31508015740E4B210AB03EB840408F1010244F8200C1F
S31508015750D2B23C46D4E70B9B01930A9B00930B49B3
S31508015760DDE908230CA82BF017FE0CA92846F3F748
S3150801577061FD29463046F3F732FD05A8F3F7BAFC71
S31508015780304610B0BDE8F081709B0408DFB204080A
S315080157902DE9F0479B4C9C4F002323703B7894B02E
S315080157A006465BB9032840F09C8001233B70974B62
S315080157B09749DA6897482BF0EFFD20703B78012B63
S315080157C013D10D2E40F06A82904A934991480223DB
S315080157D03B7053680093136A52692BF0DDFD8F4ABB
S315080157E02070002313708E4A13703B78022B78D1F0
S315080157F0032E40F053828B490B780D2B40F04E82D5
S315080158004B780A2B40F04A828B782B2B40F0468244
S31508015810CB784F2B40F042820B794B2B40F03E82DE
S3150801582008A8F3F7ACFC0A9BDFF808A2DFF8F091A9
S31508015830023B062208A911A8F3F760FD11A908A8D9
S31508015840F3F7F0FC11A8F3F755FC77490BA8F3F722
S3150801585096FC0025A8460A9B984525D22A462C215E
S3150801586008A8F3F73DFD5FFA80F843462A4608A9DA
S3150801587011A8F3F743FD11A90BA8F3F7D3FC11A857
S31508015880F3F738FC99F8000000EB40000BA90AEB86
S315080158908000F3F7AEFC99F8003008F101050133F1
S315080158A089F80030EDB2D6E75C4A13780133DBB2EA
S315080158B01370013B042B40D8DFE803F0032B303586
S315080158C03A00524A53680093D36C52695249514877
S315080158D02BF062FD20700BA8F3F70CFC08A8F3F770
S315080158E009FC3B78032B40F0D981032E40F0D68181
S315080158F04A4A13780133DBB21370013B052B00F2D8
S315080159009982DFE813F0A401D3014D025C02740207
S315080159108F023E4A53680093136BD6E73B4A536896
S315080159200093136DD1E7394A53680093536DCCE759
S31508015930364A53680093136EC7E73C4B93F80080C9
S31508015940B8F1000FC7D1334B39493A4883F800807B
S3150801595084F80080F3F7A4FC364D8146002879D0F7
S31508015960354B05F10C010EA883F80080F3F750FCBE
S315080159700EA911A8FFF7B8FE11A93048F3F752FC92
S3150801598011A8F3F7B7FB0EA8F3F7B4FB05F1180155
S315080159900EA8F3F73DFC0EA911A8FFF7A5FE11A95C
S315080159A02748F3F73FFC11A8F3F7A4FB0EA8F3F772
S315080159B0A1FB05F124010EA8F3F72AFC0EA911A8EB
S315080159C0FFF792FE11A91F48F3F72CFC11A8F3F76C
S315080159D091FB0EA8F3F78EFB1B4905F13000F3F78F
S315080159E05FFC18B1194B83F8008082E0184905F16C
S315080159F03000F3F755FC002800F0D480134B012240
S31508015A001A7076E004890120B4430020A00400201E
S31508015A1041A90408058901206BB30408E40800209C
S31508015A20E48801209E480020709B0408FA43002060
S31508015A30F3B20408004400207C3C0020703C00209E
S31508015A4028410020082F0020FAB20408203401203A
S31508015A5000B304089E492846F3F722FC002800F003
S31508015A6095809C4B05F10C014FF001080EA883F8AF
S31508015A700080F3F7CDFB0EA911A8FFF735FE11A992
S31508015A809548F3F7CFFB11A8F3F734FB0EA8F3F704
S31508015A9031FB05F118010EA8F3F7BAFB0EA911A8F7
S31508015AA0FFF722FE11A98D48F3F7BCFB11A8F3F7FE
S31508015AB021FB0EA8F3F71EFB05F124010EA8F3F747
S31508015AC0A7FB0EA911A8FFF70FFE11A98448F3F742
S31508015AD0A9FB11A8F3F70EFB0EA8F3F70BFB8149F7
S31508015AE005F13000F3F7DCFB002853D07E4B83F831
S31508015AF000907E48F3F728FC7D4B073818707D48DF
S31508015B00F3F722FC7C4B7D49013818707C48F3F782
S31508015B10C7FB002859D07B4B00221A706B6F7A4954
S31508015B201A1F11A8F3F7EAFB11A97848F3F77AFBCC
S31508015B3011A8F3F7DFFA76497648F3F75AFB76495F
S31508015B407648F3F756FB76497648F3F752FB7649DA
S31508015B507648F3F7A5FB002858D0754B00221A7032
S31508015B6074490EA8F3F754FB0EA911A8FFF7BCFD5B
S31508015B7011A97148F3F756FB11A8F3F7BBFA0EA85A
S31508015B80F3F7B8FA6D496E48F3F733FB6D48F5F745
S31508015B9099FCA0E66C4905F13000F3F781FB002872
S31508015BA07FF420AF694905F13000F3F779FB10B1AD
S31508015BB04D4B022224E7664905F13000F3F770FBE5
S31508015BC0002896D0484B03221AE762494C48F3F756
S31508015BD067FB10B14B4B01229FE75F494848F3F732
S31508015BE05FFB10B1474B022297E75C494448F3F73C
S31508015BF057FB10B1434B03228FE759494048F3F746
S31508015C004FFB00288AD03F4B042286E7554947486F
S31508015C10F3F746FB10B1464B0122A0E75249434828
S31508015C20F3F73EFB10B1424B022298E74F493F4832
S31508015C30F3F736FB10B13E4B032290E74C493B483C
S31508015C40F3F72EFB00288BD0394B042287E7494A04
S31508015C50494853680693494B1B6E0593294B197896
S31508015C60474B53F821300493234B1978454B53F886
S31508015C70213003931E4B1978434B53F82130029375
S31508015C80194B1978414B53F8213001931369009345
S31508015C90D36C3F4952692BF07FFB20702278364935
S31508015CA03C4814B0BDE8F04725F0B4B8314A3A4942
S31508015CB053680393154B1B680293384B0193136979
S31508015CC00093136B52692C482BF066FBE5E700BF7E
S31508015CD049B304087C3C0020703C00202841002080
S31508015CE0082F0020FAB20408203401203C44002081
S31508015CF0F843002048440020FB43002015B304085C
S31508015D0054440020F94300206C44002044420020FA
S31508015D1078440020408F012084440020404600201A
S31508015D2090440020144000202EB304089C4400200F
S31508015D30FC430020A844002064480020B444002005
S31508015D405C3E00208852002000B3040807B304080B
S31508015D500EB304081AB304081EB3040823B30408CF
S31508015D6028B3040833B3040838B304083DB3040858
S31508015D7042B30408A004002005890120004400203C
S31508015D8090C904089CC90408B4C90408A4C904082C
S31508015D904EB304089C94012065B3040872B3040841
S31508015DA0274A284953680393274B1B680293274BB5
S31508015DB01B68019313690093136D526983E7204A9F
S31508015DC0234853680493234B1B680393224B1B6890
S31508015DD00293224B1978224B53F821300193136908
S31508015DE00093136E1F4952692BF0D6FA55E7144AE8
S31508015DF01748536805931C4B1B6804931B4B1B6878
S31508015E0003931B4B1B6802931A4B19781A4B53F8C9
S31508015E102130019313690093136A184952692BF0CB
S31508015E20BBFA3AE7064A164953680948926C2BF0B9
S31508015E30B3FA32E7064A0023137023702EE700BF30
S31508015E40A00400207BB3040840460020408F0120AF
S31508015E50058901205C3E002064480020FC4300209F
S31508015E60BCC9040889B30408082F0020284100206A
S31508015E70703C00207C3C002000CA04089AB3040840
S31508015E80115304082DE9F0418EB0002406460D464B
S31508015E9004A82049F3F773F9A0462246AB6898454A
S31508015EA004F1010724D22E2128460392F3F718FAA2
S31508015EB05FFA80F8039A4346294607A8F3F71EFABC
S31508015EC007A904A8F3F7AEF907A8F3F713F904A885
S31508015ED0F3F73AFAE4B20EAB03EB8404FF2828BFC2
S31508015EE0FF2008F1010244F8100CD2B23C46D5E76E
S31508015EF00D9B01930C9B084900933046DDE90A2363
S31508015F002BF04AFA04A8F3F7F5F830460EB0BDE8C7
S31508015F10F08100BF709B0408DFB2040810B50128A0
S31508015F2088B018D10D4C01A82146F3F771F901A9DA
S31508015F3004A8FFF7A7FF01462046F3F77BF901A856
S31508015F40F3F7D8F8216806482BF096FA04490F2288
S31508015F506020F3F75DFA08B010BD00BF703C002061
S31508015F602134012010B5012888B018D10D4C01A89B
S31508015F702146F3F74DF901A904A8FFF783FF014666
S31508015F802046F3F757F901A8F3F7B4F8216806484C
S31508015F902BF072FA04490F227020F3F739FA08B088
S31508015FA010BD00BF284100202134012010B5012869
S31508015FB088B018D10D4C01A82146F3F729F901A992
S31508015FC004A8FFF75FFF01462046F3F733F901A856
S31508015FD0F3F790F8216806482BF04EFA04490F2288
S31508015FE08020F3F715FA08B010BD00BF082F00206E
S31508015FF0213401202DE9F04F954E9649964D91B0E1
S315080160003046F9F783FA3046F9F757FA3046F9F781
S3150801601065FA03213046F9F7ADFB95F90030348866
S31508016020072B0BD08D493046F9F75EFA201A84B250
S315080160308A4B032221463046F9F7FAF988498448FA
S31508016040F9F752FA013C201A0322854B81B280489E
S31508016050F9F7EEF983497E48F9F758FA7C48F9F7D2
S315080160602CFA7B48F9F73AFA79480321F9F782FBC2
S3150801607096F8294096F82A307B49B6F800900134FB
S3150801608003A8E41A2BF0F8F903A97148F9F72CFAD1
S31508016090E4B2A6B2A9EB000004EB440403AB224622
S315080160A081B26B48F9F7C4F9704903A82BF0E4F9F2
S315080160B003A96748F9F718FAB700A9EB00003A46A9
S315080160C003AB81B26248F9F7B3F9694903A82BF022
S315080160D0D3F903A95E48F9F707FAB846A9EB000010
S315080160E0374403AB81B23A465948F9F7A1F995F90C
S315080160F00030072B6FD8DFE813F00800D300300112
S315080161008D010800D30030018D01DFF884915949CA
S3150801611099F80020584B594D1B68033203A851F8CA
S31508016120222057492BF038F90022114603AB48487B
S31508016130F9F77EF999F8003052494FF01C0A0AFB23
S3150801614003F30A22EB5A53434F4A03A812692BF069
S3150801615023F903AB324664213D48F9F769F999F801
S3150801616000304A490AFB035303A81A892BF014F98C
S3150801617003AB720064213648F9F75AF999F80030E9
S3150801618042490AFB035303A81A7C2BF005F903AB12
S31508016190224664212E48F9F74BF999F800303B4914
S315080161A00AFB035303A81A7D2BF0F6F803AB424604
S315080161B027486421F9F73CF999F800300AFB035599
S315080161C02A7E324903A82BF0E7F8214803AB3A4661
S315080161D06421F9F72DF9DFF8BC901D4DDFF8B8A059
S315080161E0DFF8B8B034464FF0000859F8041B2846C2
S315080161F0F9F77AF9C0F15000C7B203212846F9F731
S31508016200B9FA9AF90030434510D19BF800100029D4
S3150801621000F05D81731C0093002128465023224615
S31508016220F9F792FC00212846F9F7A4FA224659F80B
S31508016230043C3946284608F10108F9F7F9F83444C7
S31508016240B8F1050FA4B2D0D111B0BDE8F08F00BFE7
S31508016250C01100206C6A04088452002018C304087F
S3150801626049B70408BA5A0408AEB30408BDB304080A
S31508016270D1B304086C0C0020040C0020980D0020F2
S3150801628011530408E7B30408883E0020EDB3040857
S315080162902B2C0020800C002085520020681F00202E
S315080162A0DFF864928D4999F800208D4B8D4D5B6816
S315080162B0033203A851F822208B492BF06DF80022EE
S315080162C0114603AB8948F9F7B3F899F800308849BC
S315080162D04FF01C0A0AFB03530A225B885343854A7B
S315080162E003A812692BF058F803AB324664217F489C
S315080162F0F9F79EF899F800307F490AFB035303A87A
S315080163005A892BF049F803AB720064217748F9F7EB
S315080163108FF899F8003078490AFB035303A85A7C89
S315080163202BF03AF803AB224664217048F9F780F856
S3150801633099F8003070490AFB035303A85A7D2BF0DC
S315080163402BF803AB424669486421F9F771F899F8C5
S3150801635000300AFB03556A7E33E7DFF8AC915F49E3
S3150801636099F800205E4B5F4D9B68033203A851F8EC
S3150801637022205D492BF010F80022114603AB5B4839
S31508016380F9F756F899F8003059494FF01C0A0AFBF3
S3150801639003530A229B885343584A03A812692AF0D1
S315080163A0FBFF03AB324664215048F9F741F899F8E7
S315080163B0003051490AFB035303A89A892AF0ECFFD6
S315080163C003AB720064214948F9F732F899F80030AD
S315080163D049490AFB035303A89A7C2AF0DDFF03AB5C
S315080163E0224664214148F9F723F899F800304249D1
S315080163F00AFB035303A89A7D2AF0CEFF03AB424654
S315080164003A486421F9F714F899F800300AFB03555C
S31508016410AA7ED6E6DFF8F090304999F80020304B8D
S31508016420304DDB68033203A851F822202E492AF0A1
S31508016430B3FF0022114603AB2C48F8F7F9FF99F888
S3150801644000302B494FF01C0A0AFB03530A22DB884A
S3150801645053432B4A03A812692AF09EFF03AB32461F
S3150801646064212248F8F7E4FF99F8003022490AFB2B
S31508016470035303A8DA892AF08FFF03AB720064215C
S315080164801A48F8F7D5FF99F800301B490AFB035358
S3150801649003A8DA7C2AF080FF03AB2246642113485D
S315080164A0F8F7C6FF99F8003013490AFB035303A806
S315080164B0DA7D2AF071FF03AB42460C486421F8F7EE
S315080164C0B7FF99F800300AFB0355EA7E79E60D4BCA
S315080164D022461B682846F8F7ABFFA7E66C0C002096
S315080164E0040C0020980D002011530408C011002047
S315080164F0E7B30408D03E0020EDB30408641D00206C
S31508016500AC1D00206C0800202B2C00201C4B1B788E
S315080165105BB91C4B1A780B2A02D00E2A06D0704793
S315080165202A221A70184B01221A707047174A92F9D3
S315080165300020022A04D0164A92F90020032A04D11F
S31508016540144A1C2111600222EEE7134991F9001041
S31508016550012904D10F4A1C2111600422E4E7072A04
S3150801656001D00C2A04D10B4A1C2111600522DBE754
S31508016570052ADAD1074A1C2111600622D4E700BF91
S31508016580681F002069890120CC080020E1890120C3
S31508016590783B0020980C0020302D00202DE9F0478B
S315080165A0AD49AE4898B0F8F7B1FFAC48F8F785FFA2
S315080165B0AA48F8F793FFA9480321F9F7DBF8A84B8E
S315080165C01B78033BDBB2092B05D840F2152222FAC8
S315080165D003F3DB0709D4A34B93F90030092B04D045
S315080165E0A14B93F90030012B05D1A04B9B480522FD
S315080165F0F921F8F71DFF9E4998489E4CF8F786FF42
S315080166009648F8F75FFF9548F9F7C1F89348F8F700
S3150801661065FF97499148F8F779FF97490BA82AF03A
S315080166202BFF002211460BAB8C48F8F701FF2068B7
S3150801663003680021DB689847904902460BA82AF0AF
S31508016640ABFE0A220BAB00218448F8F7F1FE0BA931
S315080166508248F8F749FF0A30C5B220680368012164
S31508016660DB689847864902460BA82AF095FE0A2256
S315080166700BAB29467948F8F7DBFE0BA97748F8F7FB
S3150801668033FF0A300544206803680E211B699847C1
S31508016690EDB202467B490BA82AF07EFE0A2229465C
S315080166A00BAB6E48F8F7C4FE206803680221DB6865
S315080166B09847754902460BA82AF06EFE14220BABC1
S315080166C000216648F8F7B4FE0BA96448F8F70CFFF1
S315080166D00A30C5B2206803680321DB6898476B490D
S315080166E002460BA82AF058FE14220BAB29465B4832
S315080166F0F8F79EFE0BA95948F8F7F6FE0A30054445
S31508016700206803680F211B699847EDB20246604964
S315080167100BA82AF041FE142229460BAB4F48F8F77D
S3150801672087FE206803680121DB699847FDEEC07A78
S31508016730584917EE902A0BA82AF02EFE1E220BABFB
S3150801674000214648F8F774FE206803680221DB69D0
S315080167509847FDEEC07A504917EE902A0BA82AF001
S315080167601BFE0BAB1E2246213C48F8F761FE4FF48F
S3150801677000414A4820F0B2FE4FF48041099047484B
S3150801678020F0ACFE4FF400510890444820F0A6FED4
S315080167904FF480510546414820F0A0FE4FF40061B0
S315080167A006463E4820F09AFE4FF4806107463B486C
S315080167B020F094FE4FF400718046384820F08EFE92
S315080167C04FF480718146354820F088FE8021824643
S315080167D0324820F083FEDDE90832CDE905A03049CB
S315080167E00095CDE90389CDE901670BA82AF0D4FD07
S315080167F00BAB1E228C211948F8F71AFE206803688C
S31508016800002211465B6898470546206803680022FE
S3150801681011469B689847234903462A460BA82AF03E
S31508016820BBFD0BAB282200210C48F8F701FE2068B6
S31508016830036800225B6811469847FF2834D8256803
S315080168402B680022D3E9006311462846984700239E
S31508016850C2B2FF2155E000BF6C6A0408C0110020CE
S31508016860783B0020E1890120302D002078A7040813
S31508016870BA5A0408AC1F0020F0B30408FEB3040892
S315080168800CB404081CB404082BB4040839B404086D
S3150801689049B4040858B4040864B404080010024052
S315080168A06FB404088BB404082068036800225B6887
S315080168B011469847B0F5FF7F0DD825682B68002249
S315080168C0D3E900631146284698470023C0F1FE0024
S315080168D0FF22C1B215E02068036800225B681146F1
S315080168E0984740F2FD2398426ED825682B68002206
S315080168F0D3E900631146284698470230C3B2FF22FE
S3150801690000212846B0472068036800225B680121F8
S31508016910984705462068036800229B680121984725
S315080169204E4903462A460BA82AF036FD0BAB282208
S3150801693064214B48F8F77CFD2068036800221B6A2E
S3150801694011469847474902460BA82AF025FD2822F1
S31508016950C8210BAB4248F8F76BFD20680368DB6B6F
S315080169609847414902460BA82AF016FD32220BAB7D
S3150801697000213B48F8F75CFD206803689B6A984745
S315080169800F28024664D139490BA82AF075FD0BABCD
S3150801699032224B213248F8F74BFD354B1B686421EF
S315080169A0B3FBF1F201FB1233092B94BF314932498A
S315080169B00BA82AF0F1FC0BAB3222AF212848F8F7D5
S315080169C037FD18B0BDE8F0872068036800225B68C8
S315080169D011469847B0F57F7F0CD825682B680022A9
S315080169E0D3E90063114628469847C0F1FC00FF2306
S315080169F0C2B285E72068036800225B68114698479A
S31508016A0040F2FB4398420BD825682B680022D3E94C
S31508016A100063114628469847FF230430002258E7A9
S31508016A202068036800225B681146984740F2FA53CA
S31508016A3098423FF668AF25682B680022D3E90063C0
S31508016A40114628469847C0F1FA00C3B2002200E76A
S31508016A500A490BA82AF0A0FC99E700BF98B40408D4
S31508016A60C0110020A5B40408ADB40408BAB40408DA
S31508016A70DC330120D7B40408E6B40408C9B4040811
S31508016A8070B5A749A74890B0F8F740FDA548F8F7AB
S31508016A9014FDA448F8F722FDA2480321F8F76AFE77
S31508016AA0A149A048F8F720FDC0F1F9009E4B81B233
S31508016AB005229C48F8F7BCFC9C4B93F900300C2B3B
S31508016AC008D023F00203052B04D0994B93F9003023
S31508016AD0012B05D1974B93480522F921F8F7A8FC14
S31508016AE095499048954EF8F711FD8E48F8F7EAFC56
S31508016AF08C48F8F74CFE8B48F8F7F0FC8E49894824
S31508016B00F8F704FD8E4903A82AF0B6FC002203AB68
S31508016B1011468448F8F78CFC72688A4903A82AF05A
S31508016B203BFC03AB0A2200217E48F8F781FC03A946
S31508016B307C48F8F7D9FC0A30C4B23269824903A8FD
S31508016B402AF02AFC03AB0A2221467648F8F770FC9C
S31508016B5003A97448F8F7C8FC328E7C497C4E054671
S31508016B6003A82AF019FC05F10A01214403AB0A22FC
S31508016B70C9B26C48F8F75CFC7268764903A82AF032
S31508016B800BFC03AB142200216648F8F751FC03A954
S31508016B906448F8F7A9FC0A30C4B232696A4903A8FD
S31508016BA02AF0FAFB03AB142221465E48F8F740FCAB
S31508016BB003A95C48F8F798FC328E6449664E054687
S31508016BC003A82AF0E9FB05F10A01214403AB1422C3
S31508016BD0C9B25448F8F72CFC7268604903A82AF030
S31508016BE0DBFB03AB1E2200214E48F8F721FC03A963
S31508016BF04C48F8F779FC0A30C4B23269524903A8FD
S31508016C002AF0CAFB03AB1E2221464648F8F710FCB8
S31508016C1003A94448F8F768FC328E4C49504E05469C
S31508016C2003A82AF0B9FB05F10A01214403AB1E2288
S31508016C30C9B23C48F8F7FCFB72684A4903A82AF02E
S31508016C40ABFB03AB282200213648F8F7F1FB03A971
S31508016C503448F8F749FC0A30C4B232693A4903A8FC
S31508016C602AF09AFB03AB282221462E48F8F7E0FBC7
S31508016C7003A92C48F8F738FC328E3449054603A88F
S31508016C802AF08AFB05F10A01214403AB2822C9B27D
S31508016C902448F8F7CDFB344A3449D37801939378DD
S31508016CA000935378127803A82AF076FB03AB3222B5
S31508016CB000211C48F8F7BCFB03A91A48F8F714FC8D
S31508016CC02B4B2C4A1B6812682B49044601330132A7
S31508016CD003A82AF061FB611D03AB3222C9B2114830
S31508016CE0104CF8F7A5FB254B1B686421B3FBF1F2A1
S31508016CF001FB1233092B94BF2149224903A82AF023
S31508016D004BFB03A920462578F8F7EEFB281AC1B2F2
S31508016D1003AB32222046F8F78BFB10B070BD00BFDB
S31508016D206C6A0408C0110020BF9D0408783B002046
S31508016D30302D002078A70408BA5A0408883E002096
S31508016D40F4B4040800B504080CB5040813B504081E
S31508016D50D03E002019B50408641D002025B5040895
S31508016D60AC1D002031B50408ED3301203DB50408FA
S31508016D70580A0020242C00204FB50408DC330120D2
S31508016D80D7B40408E6B4040810B5214B1B7873B9C7
S31508016D90204C23780B3B042B09D8DFE803F00309C1
S31508016DA0082603002A2323701B4B01221A7010BDE3
S31508016DB01A4B93F90030022B04D0194B93F9003082
S31508016DC0032B05D1174B1C221A6002232370EEE709
S31508016DD0154B18680368DB6B984720B1114B1C22C9
S31508016DE01A600123F2E700BFE1E70D4B93F9003082
S31508016DF0072B01D00C2B04D10A4B1C221A60052340
S31508016E00E4E7052BD3D1074B1C221A600623DDE7DD
S31508016E10681F002069890120CC080020E18901202A
S31508016E20783B0020980C0020AC1F00202DE9F0418A
S31508016E305149524890B0F8F769FB5048F8F73DFBBD
S31508016E404E48F8F74BFB4D480321F8F793FC4C499C
S31508016E504A48F8F749FBC0F1F900494B81B20522C6
S31508016E604648F8F7E5FA474B93F900300C2B03D05F
S31508016E7023F00203052B05D1434B40480522F9218E
S31508016E80F8F7D6FA3D4C4149DFF82881404F414E83
S31508016E902046F8F73BFB2046F8F714FB2046F8F79F
S31508016EA076FC2046F8F71AFB3B4B03A859682AF0EB
S31508016EB0E3FA002203AB11462046F8F7B9FAB8F807
S31508016EC000303288009335493B88258803A82AF083
S31508016ED063FA03A92046F8F707FB281A00EBD070D6
S31508016EE003ABC0F347010A222046F8F7A1FAB8F81E
S31508016EF00230728800932A497B8803A82AF04CFA43
S31508016F0003A92046F8F7F0FA281A00EBD07003AB6C
S31508016F10C0F3470114222046F8F78AFAB8F8043074
S31508016F20B28800931F49BB8803A82AF035FA03A93A
S31508016F302046F8F7D9FA281A00EBD07003ABC0F34C
S31508016F4047011E222046F8F773FA174B1B6864217E
S31508016F50B3FBF1F201FB1233092B94BF1349144910
S31508016F6003A82AF019FA03AB3222AF210348F8F72E
S31508016F705FFA10B0BDE8F0816C6A0408C011002000
S31508016F80BF9D0408783B002078A70408BA5A04086C
S31508016F90840D0020683401207C0B002061B50408AB
S31508016FA088B50408AFB50408DC330120D7B4040852
S31508016FB0E6B404087034012010B5194B1B786BB977
S31508016FC0184C23780B3B032B08D8DFE803F002089B
S31508016FD002272A232370144B01221A7010BD134B62
S31508016FE093F90030012B05D1114B1C221A60042399
S31508016FF02370F3E70F4B93F90030022B03D10C4AA8
S315080170001C211160F4E70C4B18680368DB6B984781
S3150801701020B1074B1C221A600123E9E700BFDDE70F
S31508017020681F002069890120CC080020302D002026
S31508017030980C0020E1890120AC1F002070B58D4C09
S315080170408D4992B02046F8F761FA2046F8F735FAE5
S315080170502046F8F743FA20460321F8F78BFB8749C0
S315080170602046F8F741FAC0F1F900844B052281B2AE
S315080170702046F8F7DDF982492046F8F747FA20460F
S31508017080F8F720FA2046F8F782FB2046F8F726FAA1
S3150801709020467B49F8F73AFA7A4905A82AF0ECF925
S315080170A005A920462578F8F71FFA281A05AB002204
S315080170B0C1B22046F8F7BCF97349744D05A82AF000
S315080170C0DBF9002205AB11462046F8F7B1F97049FC
S315080170D005A82AF0D1F905AB0A2200212046F8F7BE
S315080170E0A7F92A686B4905A82AF056F905AB1422AF
S315080170F000212046F8F79CF9674B68495A6805A8A4
S315080171002AF04AF905AB1E2200212046F8F790F924
S31508017110634905A82AF0B0F905AB0A22552120468C
S31508017120F8F786F96A685B4905A82AF035F905ABC7
S31508017130142255212046F8F77BF95A4B57495A68C4
S3150801714005A82AF029F905AB1E2255212046F8F78C
S315080171506FF9554905A82AF08FF905AB0A22AA2124
S315080171602046F8F765F96A694A4905A82AF014F923
S3150801717005AB1422AA212046F8F75AF94B4B474981
S315080171805A6805A82AF008F905AB1E22AA21204645
S31508017190F8F74EF901212846F2F77AFA0221039007
S315080171A02846F2F775FA032102902846F2F770FA93
S315080171B0042106462846F2F76BFADDE90232CDE9E3
S315080171C000603B4905A82AF0E7F805AB282200210B
S315080171D02046F8F72DF995F83130019395F83030B6
S315080171E0009395F82F3095F82E20324905A82AF0F4
S315080171F0D3F805AB282250212046F8F719F9D5E925
S3150801720003232D4905A82AF0C7F805AB3222002128
S315080172102046F8F70DF995F8273095F826202749DD
S3150801722005A82AF0B9F82046254C05AB3222642177
S31508017230F8F7FEF823686421B3FBF1F201FB123378
S31508017240092B94BF1F49204905A82AF0A5F805ABC3
S315080172503222AF210748F8F7EBF8D4ED007ADFEDD3
S315080172601B6AF8EE677A87EEA67A85ED417A12B03F
S3150801727070BD00BFC01100206C6A0408BF9D0408D8
S31508017280BA5A0408ABA00408D6B50408CC380020BD
S3150801729000B6040808B60408883E002011B604089A
S315080172A019B60408D03E002023B60408641D002040
S315080172B02CB604083EB6040855B6040864B6040894
S315080172C0DC330120D7B40408E6B404080000C84238
S315080172D010B5194B1B7863B9184C23780C2B09D0B8
S315080172E00E2B26D00B2B04D12A232370144B0122F3
S315080172F01A7010BD134B93F90030012B05D1124BAF
S315080173001C221A6004232370F3E7104B93F900300B
S31508017310022B03D10C4A1C211160F4E70C4B1868A7
S315080173200368DB6B984720B1074B1C221A600123BF
S31508017330E9E700BFDDE700BF681F00206989012072
S31508017340CC080020302D0020980C0020E18901206E
S31508017350AC1F002010B565496548664CA8B0F8F71A
S31508017360D5F86348F8F7A9F86148F8F7B7F8604817
S315080173700321F8F7FFF960495D48F8F7B5F8C0F158
S31508017380F9005D4B052281B25948F8F751F85B4976
S315080173905748F8F7BBF85648F8F794F85448F8F7F9
S315080173A0F6F95348F8F79AF854495148F8F7AEF8F8
S315080173B053490FA82AF060F8002211460FAB4C4832
S315080173C0F8F736F84F4A504992F9013092F90020F8
S315080173D00FA829F0E1FF0FAB0A2200214448F8F76C
S315080173E027F84A4A4A49937B0C93537B0B93137BA1
S315080173F00A93D37A0993937A0893537A0793137A5C
S315080174000693D3790593937904935379039313795F
S315080174100293D378019393780093537812780FA83F
S3150801742029F0BAFF0FAB1E2200213148F8F700F800
S31508017430384A3749937B0C93537B0B93137B0A93F7
S31508017440D37A0993937A0893537A0793137A06930F
S31508017450D379059393790493537903931379029313
S31508017460D378019393780093537812780FA829F06B
S3150801747093FF0FAB282200211D48F7F7D9FF226891
S3150801748025490FA829F088FF0FAB19480A227D2143
S31508017490F7F7CEFF23681BB34FF47A721F49B2FB85
S315080174A0F3F20FA829F078FF0FAB14227D211048BB
S315080174B0F7F7BEFF1A4B1B686421B3FBF1F201FB18
S315080174C01233092B94BF174917490FA829F064FFEE
S315080174D00FAB3222AF210648F7F7AAFF28B010BD35
S315080174E012490FA829F0C8FFDEE700BF6C6A040835
S315080174F0C0110020908F0120BF9D0408BA5A0408C4
S315080175006FB60408898F01207EB60408618F0120B1
S315080175108BB60408758F0120C8B60408E0B60408BE
S31508017520DC330120D7B40408E6B40408EAB6040833
S3150801753010B5224B1B7863B9214C23780C2B09D043
S315080175400E2B39D00B2B04D12A2323701D4B012274
S315080175501A7010BD1C4B93F90030052B05D11B4B36
S315080175601C221A6006232370F3E7072B01D00C2B84
S3150801757004D1164B1C221A600523F4E7144B93F920
S315080175800030012B04D1114B1C221A600423EAE7AF
S31508017590104B93F90030022B03D10C4A1C211160C0
S315080175A0E1E70D4B18680368DB6B984720B1074B79
S315080175B01C221A600123D6E700BFCAE7681F00200C
S315080175C069890120CC080020783B0020980C00200E
S315080175D0302D0020E1890120AC1F002030B5644C14
S315080175E06449A9B02046F7F791FF2046F7F765FFEA
S315080175F02046F7F773FF20460321F8F7BBF85E49E3
S315080176002046F7F771FFC0F1F90081B25A4B0522FE
S315080176102046F7F70DFF594B0522F9212046F7F7C2
S3150801762007FF57492046F7F771FF2046F7F74AFF44
S315080176302046F8F7ACF82046F7F750FF20465049A0
S31508017640F7F764FF4F490FA829F016FF0FA920463F
S315080176502578F7F749FF281A0FAB0022C1B2204651
S31508017660F7F7E6FE4849494D0FA829F005FF00221C
S315080176700FAB11462046F7F7DBFE2A7844490FA8D7
S3150801768029F08AFE0FAB0A2200212046F7F7D0FE21
S31508017690404A4149937B0C93537B0B93137B0A9383
S315080176A0D37A0993937A0893537A0793137A0693AD
S315080176B0D3790593937904935379039313790293B1
S315080176C0D378019393780093537812780FA829F009
S315080176D063FE0FAB1E2200212046F7F7A9FE2F4AAB
S315080176E02D49937B0C93537B0B93137B0A93D37A84
S315080176F00993937A0893537A0793137A0693D3795E
S315080177000593937904935379039313790293D37861
S31508017710019393780093537812780FA829F03CFEC9
S315080177200FAB282200212046F7F782FE2A7818494E
S315080177300FA829F031FE0FAB00227D212046F7F76D
S3150801774077FE174B1B686421B3FBF1F201FB123379
S31508017750092B94BF134914490FA829F01DFE0FAB35
S315080177603222AF210248F7F763FE29B030BD00BFC8
S31508017770C01100206C6A0408BF9D040878A7040894
S31508017780BA5A0408F4B60408F3A10408B44300205D
S31508017790F8B604089E4800208BB60408058901201E
S315080177A0DC330120D7B40408E6B404082DE9F04710
S315080177B06A496B486B4FDFF8F491DFF8F4A1A2B080
S315080177C0F7F7A4FE6648F7F778FE6548F7F786FEE9
S315080177D063480321F7F7CEFF63496148F7F784FE4B
S315080177E0C0F1F90081B2604B5D480522F7F720FE2A
S315080177F05E4B5B480522F921F7F71AFE5C495848A2
S31508017800F7F784FE5648F7F75DFE5548F7F7BFFFC9
S315080178105348F7F763FE3A7856490025013209A815
S3150801782029F0BAFD2A46294609AB4D48F7F700FE65
S31508017830514B0FCB05AE86E80F00504909A829F030
S315080178401BFE09A94648F7F74FFE4D4B4D4A93F9DA
S3150801785000304D490446E4B209A829F09DFD09AB5B
S315080178600A2221463E48F7F7E3FD484B484A1B687A
S31508017870454909A829F090FD09AB14222146384843
S31508017880F7F7D6FD434B444A93F900303E4909A818
S3150801789029F082FD09AB1E2221463148F7F7C8FDBA
S315080178A03E4909A829F0E8FD09AB282221462C48BA
S315080178B0F7F7BEFD3B783A49032B9CBFC3F1030397
S315080178C0DDB2384B33F81520254D09A829F064FD9A
S315080178D009A928462F78F7F707FE381AC1B209AB66
S315080178E028222846F7F7A4FD37460026032128460D
S315080178F0F7F740FF334699F9001057F8048B01361C
S3150801790006EB86025200994292B215D19AF80010F6
S31508017910E1B1414628460392F7F7E6FD0A232044DA
S315080179200093002183B2039A2846F8F70DF900213E
S315080179302846F7F71FFF039A434621462846F7F7D5
S3150801794077FD042ED2D122B0BDE8F087164B0392FB
S315080179501B682846F7F76CFDEDE700BF6C6A04085B
S31508017960C01100202A2C0020BF9D040878A704080E
S31508017970BA5A040805B70408CC4F040817B704080F
S31508017980C63800207D9A040898BF0408940D002083
S31508017990839A0408AD5200208D9A0408939A040824
S315080179A01AB70408A45200206C0C0020AC5200201F
S315080179B0681F00202DE9F04F9F4DA04C6D68DFF838
S315080179C0C0C2DFF8C0E2DFF8C082DFED9D5A9FED45
S315080179D09D5A451B002DB8BF6D4225609A4D6D68AD
S315080179E04D1B002DB8BF6D426560984D6D68551BDE
S315080179F0002DB8BF6D42A560954D6D685D1B002DC4
S31508017A0089B0B8BF6D42E560924D0495924D0295D5
S31508017A100194924D0595A1468E4C03944746F2462C
S31508017A20E3460026F6EE004AB0EE006A039C54F8D7
S31508017A30045B03942C8ED5ED0D7A59F8045B07EE99
S31508017A40104AF8EE677AB8EEC77A67EEA57A27EE96
S31508017A50057AB0EE404AC7EE876A029C0136F6B24D
S31508017A60A6EEC64A27EEA67A67EE847A27EE247A28
S31508017A70E4EC017AE7EE067A0294059CEBEC016ADE
S31508017A80FCEEE77AAAEC017AE4EC017A059417EEA2
S31508017A90904AAC4234BF00250125042E07F8015B44
S31508017AA0C4D16F4EDFF89491DFF8A8A19FED6D4A16
S31508017AB0DFF8D8B1DFED6C3A9FED6C3A00253560F9
S31508017AC0002518F8017B8FBB59F8257077B307EEA7
S31508017AD0107A5AF82570DEED007AD7ED0D6AD6EDE3
S31508017AE0002AB8EE477AF8EE666AA7EEC67A66EE17
S31508017AF0A56AC7EE267A9CED007AE7EE067A77EE56
S31508017B00847AF4EEE27AF1EE10FACBED007A0DDD25
S31508017B10B0EEE77AB4EE637AF1EE10FA27D8B4EE4E
S31508017B20437AF1EE10FA22DBC6ED007A0135042D0F
S31508017B300EF1040E0CF1040CC3D1D6ED007A4C4DAE
S31508017B40F5EEC07AF1EE10FA13DD4A4EC5ED007A6C
S31508017B503488B0EE670A01343480FFF72BFF454AB3
S31508017B6013880BB1013B138009B0BDE8F08F00BF44
S31508017B70DCE70023CDE906333F4ADFF8E0C09FED95
S31508017B803F4A85ED000A30EE606A07A906A8012575
S31508017B90019C54F8047B019407EE907AF8EE676A23
S31508017BA0049C86EE867A54F8046B0494348ED6EDDA
S31508017BB00D7AC7EE203AF8EE677A67EEA57AF4EE03
S31508017BC0C77A07EE104AB8EEC77AF1EE10FA27EE31
S31508017BD0057A48BF0570B4EEE37A10F8016BF1EE49
S31508017BE010FA48BF0D700EB90E780EB35CF8236013
S31508017BF0B7420BD1C7EE876AC2ED006A0133042B7F
S31508017C0002F1040201F10101C2D1A8E786EEA77AC1
S31508017C1060EE247A30EE477AB4EEE77AF1EE10FA9E
S31508017C20AABF67EE847A82ED007AC2ED007AE5E7AB
S31508017C30C2ED000AE2E700BF883E0020741F00205B
S31508017C400024743FA5D4E842D03E0020641D0020DC
S31508017C50AC1D0020D0C90408683E0020841F0020FE
S31508017C604C4100206F12833AFFFF7F7F000080009E
S31508017C70D04200205C460020E84700206666E63EC2
S31508017C803C410020CC2D0020D00D00201C340120C1
S31508017C902DE9F04F9B46644B644CD3ED007A644B57
S31508017CA094ED007AD3ED006AB8EE477A77EEE65A94
S31508017CB02DED068B87EE256A924683B08146884666
S31508017CC0B6EE008AC6EE265ADFED5A6ADFED5A8A03
S31508017CD085EEA67AD3ED015A37EE087A37EEE55ADC
S31508017CE0BCEEC77A17EE102A94ED017AB8EE477AF8
S31508017CF097B287EE05AA8AEE255AD3ED025A85EE82
S31508017D00267A37EEE55A37EE087ABCEEC77A17EEC9
S31508017D10102A94ED027AB8EE477A96B2C7EE059A1A
S31508017D2089EEA55AD3ED035A85EE267A77EEE57ADA
S31508017D3037EE087ABCEEC77A17EE102A94ED037A65
S31508017D403E4CB8EE477A204687EE279A95B289EED9
S31508017D50257AC7EE267A77EE887AFCEEE77A17EE69
S31508017D60903AC6EE287A9BB2019377EE887AFCEEB2
S31508017D70E77A17EE901AF8F7D7F9012F3946204610
S31508017D8038BF0121F8F7FCF9CAEE287A2C4F384694
S31508017D9077EE887AFCEEE77A17EE901AF8F7C4F9C7
S31508017DA0012E3146384638BF0121F8F7E9F9C9EEFF
S31508017DB0A87A244E304677EE887AFCEEE77A17EEF3
S31508017DC0901AF8F7B1F9012D2946304638BF012135
S31508017DD0F8F7D6F9C9EE287A1B4D284637EE888A70
S31508017DE0FCEEC87A17EE901AF8F79EF9019B012B5B
S31508017DF038BF012319462846F8F7C2F949462046ED
S31508017E00F8F782F941463846F8F77EF95146304681
S31508017E10F8F77AF95946284603B0BDEC068BBDE852
S31508017E20F04FF8F771B900BFD0420020741F002047
S31508017E30E8470020A5D4E8420024743F883E002084
S31508017E40D03E0020641D0020AC1D00200328F8B593
S31508017E500D4600F20981B94C9FEDB95A54F8203004
S31508017E609FEDB84A5F68D3ED0D7A1B8EDFF84CC3D8
S31508017E70B54EB8EE677A07EE903AF8EEE77A27EE4E
S31508017E80057A67EE847AB14B87EE276A03EB80039E
S31508017E90CA1B002AB8BF524246F820208100F6EED6
S31508017EA0004A67EE066A83ED006A76EE065AA84B23
S31508017EB066EEA46A03EB800370EE657AC3ED006A89
S31508017EC0A44B67EE877A76EEA66A03EB8003C3EDC9
S31508017ED0007A77EEA67AFCEEE77A17EE903A9A429E
S31508017EE04CF820309C4B94BF4FF0010E4FF0000E1A
S31508017EF003F800E0994B54D9AF4252D007EE902AC5
S31508017F00B8EEE76ADFED967A964A76EE666A86EE07
S31508017F10876ADFED956A36EE257A37EE277AF0EE2F
S31508017F20C77AF4EE667AF1EE10FA82ED007A36D85F
S31508017F30DFED8E6AF4EE667AF1EE10FA2FDB83ED49
S31508017F40007A56F82020D3ED006A54F8203007EE5F
S31508017F50902A36EEE07AF8EE675AC5EE877A93EDFF
S31508017F600D7A1B8EC7EEA03A06EE103AB8EEC66A2F
S31508017F70B8EE477A26EE046A27EE057AB4EEE36A86
S31508017F80F1EE10FA7A4B40F1CF805CF82040A2421C
S31508017F900AD1C7EE067A5A18C2ED007A12E000BF76
S31508017FA0CFE783ED000ACCE7C5EE877A5A1836EE95
S31508017FB0E77A66EEA47AB4EEE77AF1EE10FA2CDAED
S31508017FC082ED007A0B44D3ED007A76EEE76A85EE08
S31508017FD0A67AC7EE276AC6EE847A77EEA47AFCEE0D
S31508017FE0E77A17EE903AC7EE057A9CB2012C38BFAC
S31508017FF0012477EEA47AFCEEE77A17EE901A88B98F
S315080180005C48F8F791F85B482146F8F7B9F85948FA
S315080180102946BDE8F840F8F777B89FED577A67EE35
S31508018020877AB9E7012809D15448F8F77DF8534802
S315080180302146F8F7A5F851482946EAE7022809D161
S315080180404F48F8F771F84E482146F8F799F84C4821
S315080180502946DEE74B48F8F767F84A482146F8F714
S315080180608FF848482946D4E706285BD8464B9FED42
S31508018070477A4749474A01241C70474B043883ED20
S31508018080000AFAEE047A454BC0B2E0EE077A187098
S31508018090434B33F8103021F81030FCEEE77A414BA8
S315080180A0B1F9001023F8105017EE903AC0EE807A15
S315080180B09BB213803C4A00261680691A3B4E07EE8E
S315080180C0103AB8EE477A67EE877A07EE101AFCEE91
S315080180D0E77AB8EEC77A17EE902A92B2934219BF99
S315080180E09B1A07EE903ADFED207A314B328014BFA6
S315080180F0F8EEE77A1C60C7EE276A2E4B03EB80037E
S3150801810007EE902AF8EE677AC3ED006A86EEA77A3B
S31508018110294B03EB8000BDE8F84080ED007A1C206E
S315080181201EF0EEBD00BFF8BDB4EEE77AF1EE10FA27
S315080181303FF52BAF5A18C2ED000A43E7D0C9040828
S315080181400024743FA5D4E842741F00203C41002056
S31508018150CC2D0020683E0020D00D0020D042002002
S315080181606F12833A1C340120FFFF7F7F00008000D5
S31508018170E8470020883E00206666E63ED03E00209D
S31508018180641D0020AC1D002030250020000040425F
S315080181906A2F0020EC880120303800205042002048
S315080181A0703401202A250020142F0020363800209B
S315080181B0102E0020481E00203C1E0020841F00208F
S315080181C0F8B504460D4616461F46FFF7F3FB3B4630
S315080181D0204632462946FFF75BFD114B114C1B78A9
S315080181E013B9114B1B7813B1104B22681A601EF094
S315080181F091FA07EE900A94ED007ADFED0D6A0D4BC0
S31508018200F8EE677AE7EE267ADFED0B6A77EEA67A5D
S31508018210FCEEE77AC3ED007A084B83ED007AF8BDE8
S31508018220FF330120D0420020608F01203038002022
S3150801823000007A44C83C00200000C84234410020AE
S31508018240154A137893B1012B25D11449097801F000
S31508018250FD000C2806D00B291DD100211170104AEA
S31508018260137070470E4B01221A7070470B490B7831
S315080182700B3B032B0FD801A050F823F08D82010880
S31508018280658201089382010865820108012313703A
S31508018290E5E72A230B707047681F002069890120CA
S315080182A0CC0800202DE9F0412DED028B7D4C7E494D
S315080182B0DFF824827D4F7E4E94B02046F7F726F9E3
S315080182C02046F7F7FAF82046F7F708F9204603217A
S315080182D0F7F750FA77492046F7F718F92046F7F7DE
S315080182E0ECF82046F7F7FAF820460321F7F742FAA1
S315080182F07149258807A829F0BFF807A92046F7F785
S31508018300F3F8281A00EBD07007AB0022C0F3470137
S315080183102046F7F78DF8694BB3F9023007EE903A24
S31508018320F8EEE77AB2EE048AC7EE887A17EE900A73
S31508018330F0F73AF90B4662490246CDE90423B1F949
S31508018340023007EE903AF8EEE77AC7EE887A17EE2A
S31508018350900AF0F729F9DDE90423CDE90001594925
S3150801836007A829F019F807A92046F7F7BDF8281A2A
S3150801837000EBD07007AB0A22C0F347012046F7F796
S3150801838057F8D8F80000F0F70FF902460B4630689F
S3150801839039680291CDE90423F0F706F9DDE90423EA
S315080183A0CDE90001484907A828F0F6FF07A92046A4
S315080183B0F7F79AF8281A00EBD07007AB1422C0F326
S315080183C047012046F7F734F8D8F80000F0F7ECF83B
S315080183D002460B46706879680291CDE90423F0F7E5
S315080183E0E3F8DDE90423CDE90001384907A828F0B7
S315080183F0D3FF07A92046F7F777F8281A00EBD070BC
S3150801840007AB1E22C0F347012046F7F711F8D8F843
S315080184100000F0F7C9F802460B46B068B968029140
S31508018420CDE90423F0F7C0F8DDE90423CDE900011D
S31508018430274907A828F0B0FF07A92046F7F754F8F7
S31508018440281A00EBD07007AB2822C0F34701204653
S31508018450F6F7EEFFD8F80000F0F7A6F802460B4645
S31508018460F068F9680291CDE90423F0F79DF8DDE992
S315080184700423CDE90001174907A828F08DFF07A9AC
S315080184802046F7F731F8281A00EBD070C0F34701F8
S3150801849007AB32222046F6F7CBFF14B0BDEC028BB0
S315080184A0BDE8F081C01100206C6A0408741F002021
S315080184B0E8470020BA5A04082AB704081206002019
S315080184C01205002031B704084BB7040872B704082F
S315080184D099B70408C0B70408D042002001441944DA
S315080184E0114401EB132303EB12204042C0B270473B
S315080184F001280CD11C4B1A88114409B221EAE171F1
S3150801850042F20F729142A8BF11461980704702289C
S315080185100CD1154B5A88114409B221EAE17142F28C
S315080185200F729142A8BF11465980704703280CD192
S315080185300D4B9A88114409B221EAE17142F20F7290
S315080185409142A8BF11469980704704280BD1064B62
S31508018550DA88114409B221EAE17142F20F729142B5
S31508018560A8BF1146D9807047840D0020024B00220E
S315080185701A705A709A707047E08801202DE9F04107
S31508018580012888B00E464FF0000400F03E8102280B
S3150801859000F05581032800F05481042800F0538126
S315080185A0632800F05281602800F051815F2800F0AD
S315080185B05081082800F04F81092800F04E810A28C9
S315080185C014BF25460F25072E2ED8DFE816F0090019
S315080185D034010C01E900FD0001010401080101252E
S315080185E09F4A92F900301278782A00F2B180421E29
S315080185F09C499D4C31F8121034F81220914240F2F0
S31508018600A28003F5A0618EB2012840F0A380954BA4
S31508018610954A1988B3F90030118042F20F74A342C2
S3150801862001DC23EAE374A4B223463246062128462E
S31508018630FFF754FFDFF858828C4988F800002A466C
S3150801864001A828F0A9FE8A4F0128387004D1894962
S315080186502A4601A828F0A0FE8449062202A828F085
S315080186609BFE012383493B70062202A828F094FE4B
S3150801867032467E4904A828F08FFEC3B203283B7010
S31508018680324640F0B2807B4904A828F085FE774936
S31508018690224606A828F080FEC3B203283B7040F0A4
S315080186A0A9807449224606A828F076FE98F8002083
S315080186B06E4903A828F070FE0128387005D198F88C
S315080186C000206C4903A828F067FE6B493A230B7012
S315080186D09DF804304B709DF805308B709DF8083075
S315080186E0CB709DF809300B719DF810304B719DF8D0
S315080186F011308B719DF81230CB719DF813300B72C6
S315080187009DF818304B729DF819308B729DF81A3006
S31508018710CB729DF81B300B739DF80C304B739DF88B
S315080187200D308B730D23CB730A230B74534B112214
S315080187303A7093F90030012B02D1514822F06AFBB5
S3150801874008B0BDE8F081BFF45FAF03F5B0615AE741
S31508018750002659E7022806D1424B434A59885180D7
S31508018760B3F9023059E7032806D13E4B3E4A9988A8
S315080187709180B3F9043050E7042806D1394B3A4AB7
S31508018780D988D180B3F9063047E7002349E73D4B3D
S315080187901C780125632CA8BF6324A4B2032643E7EA
S315080187A0022802D1374B5C78F4E7032802D1354B0E
S315080187B09C78EFE7042802D1324BDC78EAE70A28ED
S315080187C0FAD00024E9E70125012400262CE7012532
S315080187D00024FAE701250024052625E701250024BA
S315080187E0062621E7012500241EE7022B0CBF264990
S315080187F0264949E7022B02D12349224653E7012B91
S315080188007FF454AF214922464DE7072915D801A31C
S3150801881053F821F0DF85010835880108E587010845
S315080188208F870108C7870108CF870108D5870108FF
S31508018830DD87010801253446F6E60125F4E60546F5
S31508018840C1E60425BFE60825BDE6C925BBE696258A
S31508018850B9E66A25B7E60325B5E60725B3E600BFF7
S31508018860541E0020840D002070340120EAB7040844
S3150801887004890120E9B70408642D0020302D002061
S31508018880E09401208C0D0020E8B70408E7B7040836
S315080188903034012038B5324B1D7845B9314C23782F
S315080188A00E2B30D004D80B2B19D00C2B1DD038BD6C
S315080188B0182B46D02C2BFAD12B4A137883F00103B7
S315080188C013702A4A106802681468D3B114232A4619
S315080188D01146A047BDE838402548F6F717B92A23B7
S315080188E02370244B01221A70E1E7204B18680368AC
S315080188F0DB6B98470028DAD01F4B1C221A6001232C
S315080189000AE0FF22E4E71D4B93F90030012B05D15C
S31508018910194B1C221A6004232370C8E7184B93F9D4
S315080189200030072B01D00C2B04D1134B1C221A60E3
S315080189300523F1E7052BBAD10F4B1C221A60062332
S31508018940EAE7104C23782BB105216320FFF716FEC1
S315080189502570ACE704216320FFF710FECFE700BFBF
S31508018960681F00206989012001340120AC1F0020FD
S31508018970A81E0020CC080020980C0020302D0020CD
S31508018980783B0020882A00202DE9F04F8BB0904BC8
S31508018990009300258F4BDFF85892019383464FF0D9
S315080189A001082C46009B33F8022B0093019B33F8F0
S315080189B0026B0193B24200F0E3800023B8F1010F84
S315080189C0ADF80C308DF80E30ADF810308DF8123048
S315080189D006938DF81C3008938DF82430ADF81430C1
